:100000000C9428170C9461170C9461170C946117C9
:100010000C94C63F0C94C63F0C94C63F0C94C63F4C
:100020000C9461170C9461170C9461170C94611770
:100030000C9461170C9408270C9461170C946117A9
:100040000C9461170C941E250C94FDC20C9461173E
:100050000C942A820C9420820C9461170C946117E2
:100060000C9461170C9461170C9461170C94611730
:100070000C9461170C9461170C9461170C94611720
:100080000C9461170C9461170C9461174E414E4902
:100090004E495459494E46CDCCCC3D0AD7233C1746
:1000A000B7D13877CC2B329595E6241FB14F0A0093
:1000B0000020410000C84200401C4620BCBE4CCA83
:1000C0001B0E5AAEC59D7400407A10F35A00A07200
:1000D0004E18090010A5D4E80000E8764817000083
:1000E000E40B54020000CA9A3B000000E1F5050051
:1000F0000080969800000040420F000000A086019A
:10010000000000102700000000E803000000006469
:1001100000000000000A00000000000100000000D4
:10012000002C76D888DC674F0823DFC1DFAE59E1A9
:10013000B1B796E5E3E453C63AE651997696E8E618
:10014000C28426EB898C9B62ED407C6FFCEFBC9CEB
:100150009F40F2BAA56FA5F490055A2AF75C936BFD
:100160006CF9676DC11BFCE0E40D47FEF520E6B5B8
:1001700000D0ED902E0300943577050080841E0892
:100180000000204E0A000000C80C333333330F98B0
:100190006E12831141EF8D2114893BE65516CFFE77
:1001A000E6DB18D1844B381BF77C1D901DA4BBE403
:1001B00024203284725E228100C9F124ECA1E53D45
:1001C000275045544700504C41005072696E7420CE
:1001D00041626F72746564004D3235005061757311
:1001E000696E672E2E2E004D323400454550524F19
:1001F0004D2056657273696F6E204572726F720082
:10020000454550524F4D20496E64657820457272C5
:100210006F7200454550524F4D2043524320457266
:10022000726F72003F0049676E6F726500526573AE
:10023000657400496E697469616C697A6520454529
:1002400050524F4D0000FE0003FF8007C7C007015A
:10025000E00000E00000F00000700400700E00708C
:100260001F00703F80F00E00E00F01E007C7C003E1
:10027000FF8000FE0000FE0003FF8007C7C00F01E3
:10028000E00E00E03F80F01F00700E007004007070
:100290000000700000F00000E00701E007C7C003A5
:1002A000FF8000FE000E000E000E000E000E000E7D
:1002B000000E000E007FC03F801F000E00040004EF
:1002C000000E001F003F807FC00E000E000E000ECB
:1002D000000E000E000E000E00FFFFFF7F80FFC02B
:1002E000FFC0FFC07F807F80FFC0FFC0FFC03F0016
:1002F0001E000C0050726F6265205A204F666673B4
:1003000065740020082046616374002008204D6158
:1003100078002008204D696E004F6666004F6E0021
:100320004175746F74656D700045207374657073EA
:100330002F6D6D005A2053746570732F6D6D0059C9
:100340002053746570732F6D6D0058205374657061
:10035000732F6D6D00416476616E63656420536533
:100360007474696E67730054656D7065726174753D
:1003700072650053746570732F6D6D00436F6E6608
:10038000696775726174696F6E003F004E657874BD
:1003900020436F726E657200446F6E65004E657823
:1003A0007400486F6D696E672058595A0053746F16
:1003B00072652053657474696E6773004C6F616475
:1003C0002053657474696E677300426564205472CB
:1003D000616D6D696E670050726F6265205A204FC3
:1003E0006666736574004661646520486569676880
:1003F00074004F6666004F6E00426564204C65765F
:10040000656C696E67004C6576656C2042656400BA
:100410004732394E00473239004175746F20486FBA
:100420006D65004D6F74696F6E00526573746F7205
:10043000652044656661756C7473004C6F6164205F
:1004400053657474696E67730053746F72652053DB
:10045000657474696E67730050726F6265205A200C
:100460004F666673657400416476616E63656420EF
:1004700053657474696E6773004D61696E003F0067
:100480004261636B0053746F70004D3232004174EF
:1004900074616368204D65646961004D32310050BC
:1004A00072696E742066726F6D204D6564696100BB
:1004B00052656C65617365204D6564696100436FC9
:1004C0006E66696775726174696F6E0054656D70F0
:1004D00065726174757265004D6F74696F6E00525C
:1004E0006573756D65205072696E740054756E6524
:1004F0000053746F70205072696E74005061757390
:1005000065205072696E7400496E666F2053637285
:1005100065656E000A4D3234004D3233202573007C
:100520003F005374617274205072696E74004361AD
:100530006E63656C005072696E740043616E6E6F1D
:100540007420656E746572207375626469723A20F6
:100550000002202E2E000152656672657368004D00
:1005600061696E002100486F74656E6420746F6F5E
:1005700020636F6C64004261636B0050726F63654F
:100580006564004D6F74696F6E0044697361626CDD
:1005900065205374657070657273004D3834004285
:1005A0006564204C6576656C696E67004175746F93
:1005B00020486F6D6500473238004D61696E00C696
:1005C00001C101436F6F6C646F776E005072656894
:1005D00065617420240046616E2053706565640077
:1005E0004E6F7A7A6C65004D61696E0050726F6271
:1005F00065205A204F666673657400466C6F7700FD
:1006000046616E205370656564004E6F7A7A6C6542
:10061000005370656564004D61696E00486F6D69D7
:100620006E67204661696C6564006F70656E00548A
:100630005249474745524544003A20007A5F70725C
:100640006F6265007A5F6D696E00795F6D696E003B
:10065000785F6D696E005265706F7274696E6720A5
:10066000656E6473746F70207374617475730A00BF
:1006700020746F6F206C6F6E67206578747275736D
:10068000696F6E2070726576656E7465640A00200D
:10069000636F6C6420657874727573696F6E207017
:1006A000726576656E7465640A00486F6D65202515
:1006B0007325732573204669727374005761726ED7
:1006C000696E673A20486F6D696E672042756D707C
:1006D0002044697669736F72203C20310A0002025F
:1006E000040000E0C0000000C0000000000000683E
:1006F000430000634300007A430000A0400000A0D4
:100700004000000040FFFDFCFAF8F6F4F2F0EEECD9
:10071000EAE9E7E5E3E1E0DEDCDAD9D7D5D4D2D007
:10072000CFCDCBCAC8C7C5C3C2C0BFBDBCBAB9B79D
:10073000B6B4B3B2B0AFADACAAA9A8A6A5A4A2A105
:10074000A09E9D9C9A99989795949392908F8E8D48
:100750008B8A8988878684838281807F7E7D7B7A6D
:10076000797877767574737271706F6E6D6C6B6A71
:10077000696867666564636261605F5E5D5C5B5A61
:100780005958585756555453525150504F4E4D4C3E
:100790004B4A4A4948474646454443424241403F06
:1007A0003E3E3D3C3B3B3A393838373635353433BD
:1007B00032323130302F2E2E2D2C2B2B2A29292866
:1007C000272726252524232322212120201F1E1E02
:1007D0001D1C1C1B1B1A1919181817161615151491
:1007E000131312121111100F0F0E0E0D0D0C0C0B16
:1007F0000A0A090908080707060605050404030391
:100800000202010000000000010000000100008061
:1008100000555555000000400033333300AAAA2A82
:10082000004992240000002000C7711C009999190A
:1008300000D1451700555515003BB113002449124E
:100840000011111100000010000F0F0F00E3380E0F
:100850000043790D00CCCC0C00C3300C00E8A20B97
:100860000064210B00AAAA0A00703D0A009DD80965
:1008700000427B090092240900DCD3080088880824
:10088000001042080000000800F0C1070087870739
:100890000075500700711C07003EEB0600A1BC0666
:1008A000006990060066660600703E060061180644
:1008B0000017F4050074D105005BB00500B2900587
:1008C00000627205005555050078390500B81E050F
:1008D00000050505004EEC040087D40400A1BD040A
:1008E0000090A7040049920400C17D0400EE690451
:1008F00000C7560400444404005C3204000821048C
:100900000041100400000004003FF00300F8E00381
:100910000026D20300C3C30300CCB503003AA803EA
:10092000000A9B0300388E0300C08103009F7503FB
:1009300000D0690300505E03001D530300344803D8
:1009400000913D03003333030016290300381F03D1
:100950000097150300300C0300030303000BFA0299
:100960000049F10200BAE802005CE002002DD80262
:10097000002DD0020059C80200B0C0020031B902F7
:1009800000DAB10200AAAA0200A0A30200BC9C02E5
:1009900000FA9502005C8F0200DF8802008282026A
:1009A00000457C02002776020027700200436A029D
:1009B000007C640200D05E02003F590200C853026E
:1009C00000000061430000614300007A430000E042
:1009D000C0000000C00000000053657474696E67B9
:1009E000732053746F72656400290A002062797461
:1009F00065733B20637263200053657474696E678E
:100A0000732053746F726564202800454550524F1F
:100A10004D206461746173697A65206572726F72CA
:100A20002E0A00290A002062797465733B206372E4
:100A30006320002073746F72656420736574746939
:100A40006E6773207265747269657665642028002C
:100A5000202863616C63756C6174656429210A00E8
:100A600020213D2000454550524F4D204352432008
:100A70006D69736D61746368202D202873746F72C3
:100A800065642920002053697A653A2000496E6424
:100A900065783A2000204D61726C696E3D5638369B
:100AA000290A00454550524F4D2076657273696F93
:100AB0006E206D69736D61746368202845455052DE
:100AC0004F4D3D0048617264636F64656420446506
:100AD0006661756C742053657474696E6773204C1D
:100AE0006F616465640A000000FA430000FA430085
:100AF00000A0400000C8410000A0420000A0420049
:100B000000C8430080C043F4010000F40100006409
:100B10000000008813000020286D6D2900203B2074
:100B20004C6576656C696E67200020204D3432304C
:100B30002053004175746F20426564204C657665D2
:100B40006C696E670020460020480020204D31343B
:100B5000352053004D6174657269616C2068656170
:100B600074757020706172616D65746572730020B8
:100B70004A002020473239205720490020204D319B
:100B800034392043203B20556E69747320696E20F0
:100B900043656C736975730A0054656D70657261A5
:100BA0007475726520556E69747300202047323168
:100BB000203B004C696E65617220556E697473004C
:100BC00024F4D43050C38E20C2A24017828B7011FF
:100BD000127A910D816CD90AA861E108C75866079D
:100BE000615143061E4B5D05C145A7041A4111041E
:100BF000093D9803713931034036DB0265339102B8
:100C0000D4305402802E1D02632CEE01752AC501DA
:100C1000B028A001102781018F2564012B244B01EE
:100C2000E0223401AC211F018D200D01801FFC004A
:100C3000841EED00971DDF00B81CD200E61BC60025
:100C4000201BBC00641AB200B219A8000A19A00047
:100C50006A189900D117910040178B00B5168400CF
:100C600031167E00B31579003A157300C7146F0072
:100C700058146A00EE1366008813630025135E00A3
:100C8000C7125B006C12570015125400C1115100BD
:100C900070114F0021114B00D61049008D104700F4
:100CA0004610440002104200C00F4000800F3E007A
:100CB000420F3C00060F3B00CB0E3800930E37006E
:100CC0005C0E3500270E3400F30D3200C10D3100EB
:100CD000900D3000600D2E00320D2D00050D2C0002
:100CE000D90C2B00AE0C2900850C29005C0C2700C8
:100CF000350C27000E0C2600E80B2400C40B240042
:100D0000A00B23007D0B23005A0B2100390B21007F
:100D1000180B2000F80A1F00D90A1E00BB0A1E008B
:100D20009D0A1D00800A1D00630A1C00470A1B0063
:100D30002C0A1B00110A1A00F7091A00DD09190014
:100D4000C4091900AB091900920917007B091800A2
:100D5000630917004C091600360916002009160011
:100D60000A091500F5081500E0081400CC08140065
:100D7000B8081400A4081400900813007D0812009D
:100D80006B081300580812004608120034081100BE
:100D9000230811001208110001081100F0071000CB
:100DA000E0071000D0071000C0071000B0070F00C8
:100DB000A107100091070E0083070F0074070F00B2
:100DC00065070E0057070E0049070E003B070D0090
:100DD0002E070E0020070D0013070D0006070D005B
:100DE000F9060C00ED060D00E0060C00D4060C0020
:100DF000C8060C00BC060C00B0060C00A4060B00D4
:100E000099060C008D060B0082060B0077060B007E
:100E10006C060B0061060A0057060B004C060A0020
:100E200042060A0038060A002E060A0024060A00B6
:100E30001A060A001006090007060A00FD05090047
:100E4000F4050900EB050900E2050900D9050900D0
:100E5000D0050900C7050900BE050900B505080051
:100E6000AD050800A50509009C05080094050800CB
:100E70008C050800840508007C050800740508003E
:100E80006C050700650508005D05070056050800AC
:100E90004E05070047050700400508003805070014
:100EA000310507002A050700230507001C05060079
:100EB000160507000F0507000805060002050700D4
:100EC000FB040600F5040700EE040600E804060033
:100ED000E2040700DB040600D5040600CF04060088
:100EE000C9040600C3040600BD040600B7040600DA
:100EF000B1040500AC040600A6040600A004050029
:100F00009B04060095040500900406008A04050071
:100F100085040500800406007A04050075040500B8
:100F2000700405006B0405006604050061040500FB
:100F30005C04050057040500520405004D0405003B
:100F400048040500430405003E0404003A0405007B
:100F500035040500300404002C04050027040400B7
:100F6000230405001E0404001A04040016040500EE
:100F7000110404000D040400090405000404040025
:100F800000040400FC030400F8030400F40304005C
:100F9000F0030400EC030400E8030400E40304008D
:100FA000E0030400DC030400D8030400D4030400BD
:100FB000D0030400CC030400C8030300C5030300EE
:100FC00024F404D9201BC40C5C0E9804C4095F02ED
:100FD00065077101F405F900FB04B30048048700BC
:100FE000C10369005803550003034500BE023A00DF
:100FF0008402310053022A00290225000402200045
:10100000E4011C00C8011900AF0117009801140089
:1010100084011300710110006101100051010E00E4
:1010200043010D0036010B002B010B0020010B00CA
:10103000150109000C01090003010800FB0008006C
:10104000F3000800EB000700E4000600DE000600E5
:10105000D8000600D2000600CC000500C70005003D
:10106000C2000500BD000400B9000400B500040082
:10107000B1000400AD000400A9000400A5000300B5
:10108000A20003009F0004009B00030098000300DF
:101090009500020093000300900003008D00020001
:1010A0008B00030088000200860002008400030019
:1010B000810002007F0002007D0002007B00020030
:1010C000790002007700010076000200740002003F
:1010D00072000100710002006F0002006D0001004B
:1010E0006C0002006A000100690002006700010054
:1010F000660001006500010064000200620001005A
:1011000061000100600001005F0002005D0001005D
:101110005C0001005B0001005A0001005900010061
:101120005800010057000100560001005500010061
:101130005400010053000000530001005200010060
:1011400051000100500001004F0001004E0000005E
:101150004E0001004D0001004C0001004B0000005A
:101160004B0001004A000100490001004800000056
:101170004800010047000100460000004600010051
:10118000450000004500010044000100430000004C
:101190004300010042000000420001004100000045
:1011A00041000100400001003F0000003F0001003D
:1011B0003E0000003E0001003D0000003D00010037
:1011C0003C0000003C0000003C0001003B0000002F
:1011D0003B0001003A0000003A0001003900000025
:1011E000390001003800000038000000380001001C
:1011F0003700000037000100360000003600000014
:101200003600010035000000350000003500010007
:1012100034000000340000003400010033000000FE
:1012200033000000330001003200000032000000F3
:1012300032000100310000003100000031000100E7
:101240003000000030000000300001002F000000DE
:101250002F0000002F0000002F0001002E000000D2
:101260002E0000002E0001002D0000002D000000C7
:101270002D0000002D0001002C0000002C000000BB
:101280002C0000002C0001002B0000002B000000AF
:101290002B0000002B0001002A0000002A000000A3
:1012A0002A0000002A000100290000002900000097
:1012B000290000002900000029000100280000008A
:1012C000280000002800000028000000280001007D
:1012D0002700000027000000270000002700000072
:1012E0002700010026000000260000002600000064
:1012F0002600000026000100250000002500000057
:101300002500000025000000250000002500010048
:10131000240000002400000024000000240000003D
:10132000240001002300000023000000230000002F
:101330002300000023000000230000002300010020
:101340002200000022000000220000002200000015
:101350002200000022000100210000002100000006
:1013600021000000210000002100000021000000F9
:1013700021000100200000002000000020000000EB
:1013800020000000200000002000000020000000DD
:10139000200001001F0000001F0000001F000000CF
:1013A0001F0000001F0000001F0000001F000100C0
:1013B0001E0000001E0000001E0000001E000000B5
:1013C000393000003325000087190000B00F0000FD
:1013D000DB080000BD040000740200003F010000B3
:1013E00020436F756E7420583A0045310045002C3B
:1013F0002073797374656D2073746F7070656421E8
:10140000204865617465725F49443A20004865610F
:1014100074696E67204661696C6564004865617433
:10142000696E67206661696C6564004572723A2076
:101430004D415854454D50004D415854454D502054
:10144000747269676765726564004572723A204D0F
:10145000494E54454D50004D494E54454D50207411
:10146000726967676572656400202F0020403A004A
:101470007C3C3E5E2B3D3F2F5B5D3B2C2A225C007B
:10148000434F4D4D554E49434154494F4E004452F0
:101490005952554E004552524F525300494E464FF5
:1014A000004543484F0053544F505045442E2000B0
:1014B0005072696E7465722073746F707065642009
:1014C00064756520746F206572726F72732E20468A
:1014D000697820746865206572726F7220616E642D
:1014E00020757365204D39393920746F207265730A
:1014F000746172742E202854656D70657261747504
:1015000072652069732072657365742E205365744B
:1015100020697420616674657220726573746172EB
:1015200074696E67290A004E6F20436865636B73A8
:10153000756D2077697468206C696E65206E756DB5
:101540006265722C204C617374204C696E653A2080
:10155000004E6F20436865636B73756D2077697407
:1015600068206C696E65206E756D6265722C204C0A
:10157000617374204C696E653A2000636865636B23
:1015800073756D206D69736D617463682C204C6197
:101590007374204C696E653A20004C696E65204E6C
:1015A000756D626572206973206E6F74204C617373
:1015B00074204C696E65204E756D6265722B312CFE
:1015C000204C617374204C696E653A20004D3131B6
:1015D000300053657269616C207374617475732097
:1015E0006D69736D617463680A00534420726561AC
:1015F00064206572726F720A002121204B494C4CA5
:101600002063617573656420627920746F6F206D4B
:1016100075636820696E6163746976652074696DAD
:1016200065202D2063757272656E7420636F6D6D19
:10163000616E643A20004D6564696120496E73658E
:101640007274656400627573793A207061757365B0
:101650006420666F7220696E7075740A006275731B
:10166000793A2070617573656420666F72207573B6
:1016700065720A00627573793A2070726F636573E0
:1016800073696E670A00506C6561736520526573FB
:101690006574005052494E5445522048414C5445BF
:1016A000440025533A202553004B494C4C45442EC9
:1016B00020005072696E7465722068616C74656494
:1016C0002E206B696C6C28292063616C6C65642129
:1016D0000A006563686F3A004572726F723A004F94
:1016E0004646004F4E0042696C696E656172204C3F
:1016F0006576656C696E6720477269643A0A0050C6
:10170000726F62696E6720506F696E740025532096
:1017100025692F2569002E0A002F0050726F62691B
:101720006E67206D65736820706F696E742000208D
:101730002844525952554E29004732392041757478
:101740006F20426564204C6576656C696E67003F6A
:1017500020284C2C522C462C4229206F7574206F67
:101760006620626F756E64732E0A003F28562965E5
:1017700072626F7365206C6576656C20696D706C44
:1017800061757369626C652028302D34292E0A003A
:10179000426164205A2076616C75650A004E6F20A4
:1017A00062696C696E65617220677269640A0047DC
:1017B00032384C300020204D3230312058004D61FD
:1017C0007820416363656C65726174696F6E20286F
:1017D000756E6974732F7332290020204D323033B7
:1017E0002058004D61782066656564726174657388
:1017F0002028756E6974732F7329002052002020F1
:101800004D323034205000416363656C6572617401
:10181000696F6E2028756E6974732F7332292028C2
:10182000503C7072696E742D616363656C3E20522A
:101830003C726574726163742D616363656C3E20F4
:10184000543C74726176656C2D616363656C3E29EE
:1018500000204A0020540020530020204D32303513
:10186000204200416476616E6365642028423C6DCD
:10187000696E5F7365676D656E745F74696D655FD2
:1018800075733E20533C6D696E5F66656564726179
:1018900074653E20543C6D696E5F74726176656C50
:1018A0005F66656564726174653E204A3C6A756E68
:1018B000635F6465763E29002044002049002020B3
:1018C0004D333031205000486F74656E64205049AC
:1018D00044002E0A00206E6F742064697361626C8C
:1018E00065642E20536861726564207769746800AE
:1018F00020496E76616C69642065787472756465E0
:10190000722000536C6565702E2E2E005A20507286
:101910006F62652050617374204265640A005A202A
:1019200050726F62652050617374204265640020BC
:101930005A3A200020593A200042656420583A2043
:10194000004D65736820706F696E74206F75742028
:101950006F662072616E67650A00436C69636B2075
:10196000746F20526573756D652E2E2E00616C7339
:101970006F20656E61626C6564290A004E6F204DB0
:101980006F76652E004E6F206D656469610A0045B3
:101990006E642066696C65206C6973740A00426528
:1019A00067696E2066696C65206C6973740A00282B
:1019B0006E6F2066696C6529004E6F742053442059
:1019C0007072696E74696E670A00534420707269A0
:1019D0006E74696E67206279746520004375727257
:1019E000656E742066696C653A20002E0A004465B5
:1019F0006C6574696F6E206661696C65642C204645
:101A0000696C653A200046696C652064656C657494
:101A100065643A002569730025696D2025697300A6
:101A20002569682025696D20256973002569642072
:101A30002569682025696D2025697300256979204D
:101A4000256964202569682025696D202569730052
:101A50005072696E742074696D653A20006F6B0076
:101A60006F666600A1149C1495148E14801444456E
:101A70004255473A004D3131322053687574646FD6
:101A8000776E004D3131332053004D656761205A28
:101A900065726F204F46462E00434F4E4649475FC2
:101AA0004558504F5254004D4541545041434B000E
:101AB000434F4F4C45525F54454D5045524154554C
:101AC0005245004348414D4245525F54454D5045B3
:101AD0005241545552450042414259535445505089
:101AE000494E470041524353004D4F54494F4E5FBA
:101AF0004D4F44455300544845524D414C5F505260
:101B00004F54454354494F4E00455854454E444563
:101B1000445F4D3230004C4F4E475F46494C454E76
:101B2000414D45004155544F5245504F52545F531B
:101B3000445F5354415455530053445F57524954E2
:101B400045005245504541540053444341524400DE
:101B500050524F4D50545F535550504F52540048BF
:101B60004F53545F414354494F4E5F434F4D4D4196
:101B70004E445300454D455247454E43595F5041F1
:101B80005253455200434153455F4C494748545FC7
:101B90004252494748544E45535300544F47474CCF
:101BA000455F4C494748545300534F4654574152A0
:101BB000455F504F574552004255494C445F504590
:101BC0005243454E54004C4556454C494E475F44A0
:101BD000415441005A5F50524F42450052554E4FBA
:101BE0005554004155544F4C4556454C00505249B0
:101BF0004E545F4A4F420050524F47524553530094
:101C00004155544F5245504F52545F54454D50002A
:101C10004155544F5245504F52545F504F53005608
:101C20004F4C554D455452494300454550524F4D38
:101C30000042494E4152595F46494C455F5452411A
:101C40004E534645520053455249414C5F584F4E02
:101C50005F584F4646004649524D574152455F4EE8
:101C6000414D453A4D61726C696E20322E302E39ED
:101C70002E332D6B61643120284465632032372078
:101C8000323032312031333A35303A323229205332
:101C90004F555243455F434F44455F55524C3A6759
:101CA00069746875622E636F6D2F6B61642F4D616F
:101CB000726C696E2050524F544F434F4C5F5645E3
:101CC0005253494F4E3A312E30204D414348494EF0
:101CD000455F545950453A4D656761205A65726FAA
:101CE0002045585452554445525F434F554E543A3F
:101CF0003120555549443A64626663636435352D35
:101D0000656262612D343631352D616264372D3163
:101D100039366161343338663330340A002F2F008E
:101D20004D31343520533C696E6465783E206F75C3
:101D300074206F662072616E67652028302D31290E
:101D40000A003F4A206F7574206F662072616E67CB
:101D5000652028302E303120746F20302E33290A30
:101D60000020580020204D61783A200020002020DB
:101D70004D696E3A2000203B200020204D32313149
:101D800020530046523A0020466C6F773A200050AC
:101D9000726F6265204F6666736574205A005072D8
:101DA0006F6265204F6666736574205A00646973BC
:101DB00000656E0043290A0061626C656420286D2D
:101DC000696E2074656D702000436F6C64206578C7
:101DD0007472756465732061726520004F46460A0F
:101DE0000046616465204865696768742000426543
:101DF00064204C6576656C696E6720004661696C8D
:101E0000656420746F20656E61626C652042656454
:101E1000204C6576656C696E670A00496E76616C68
:101E20006964206D6573682E0A004D343231206973
:101E30006E636F727265637420706172616D657438
:101E400065722075736167650A004D65736820705F
:101E50006F696E74206F7574206F662072616E6793
:101E6000650A00454550524F4D204F4B0A00290A44
:101E70000020746F20003F5A206F7574206F662019
:101E800072616E6765202800290A0020746F2000A7
:101E90003F59206F7574206F662072616E676520F0
:101EA000282D00290A0020746F20003F58206F75EC
:101EB00074206F662072616E676520282D004D3892
:101EC0003400446F6E65207072696E74696E6720AD
:101ED00066696C650A004D3737004D333100496E35
:101EE00076616C69642065787472756465720A0045
:101EF0004361703A00203B0020204D383531205896
:101F0000005A2D50726F6265204F666673657400CB
:101F1000436F6F6C696E672E2E2E00486561746981
:101F20006E672E2E2E0045312025530020573A0093
:101F300023646566696E652044454641554C545F8F
:101F4000004B6420004B6920004B70200050494436
:101F5000204175746F74756E652066696E6973686B
:101F60006564212050757420746865206C617374F9
:101F7000204B702C204B6920616E64204B642063E1
:101F80006F6E7374616E74732066726F6D2062651C
:101F90006C6F7720696E746F20436F6E666967752A
:101FA000726174696F6E2E680A0050494420417551
:101FB000746F74756E65206661696C656421207448
:101FC000696D656F75740A00504944204175746FDE
:101FD00074756E65206661696C6564212054656D59
:101FE000706572617475726520746F6F20686967BF
:101FF000680A00504944204379636C657300255397
:102000002025692F256900204B643A2000204B6968
:102010003A2000204B703A200020436C61737369B2
:102020006320504944200A002054753A2000204B78
:10203000753A2000206D61783A2000206D696E3A73
:10204000200020643A200020626961733A20005722
:1020500061697420666F7220686561742075702EE6
:102060002E2E00504944204175746F74756E6520A2
:1020700073746172740A00504944204175746F741E
:10208000756E65206661696C6564212054656D70AC
:102090006572617475726520746F6F206869676816
:1020A0000A00504944204175746F74756E6520664E
:1020B00061696C65642120426164206865617465B2
:1020C000722069640A00504944204175746F747528
:1020D0006E65004572723A207574663820666F6EC0
:1020E00074206E6F7420696E697469616C697A65B9
:1020F000642E004572723A207574663820666F6EE1
:1021000074206E6F7420696E697469616C697A6598
:10211000642E004572723A207574663820666F6EC0
:1021200074206E6F7420696E697469616C697A6578
:10213000642E002568753A253032687500253032E6
:1021400068753A2530326875002530326875272564
:102150003032687500256875642025303268753A1C
:1021600025303268750042656400456E636C6F739C
:1021700075726500202020202020200020202020B3
:1021800000453A00523A00657272001FE0201020AC
:102190001020101020102020102010303008400493
:1021A0008003001FE03FF03FF03FF01FE01FE03FE3
:1021B000F03FF03FF00FC0078003003FFFF0380012
:1021C0007030FC3020FC102078102030102C00D013
:1021D0002E31D02F7BD02F7BD02E31D02C00D02091
:1021E000301020781020FC1030FC303800703FFF99
:1021F000F03FFFF03800703186302387102787903A
:102200002F87D02F03D02030102078102078102076
:1022100030102F03D02F87D0278790238710318647
:10222000303800703FFFF0001DC43F0000000C86F6
:10223000198000000D0E198000000F0B198000009E
:102240000D9F198000000DD3998000001CFBFF003A
:1022500000000000000000000000000000F380000B
:102260001F80007700001980005B1CF6131DAE5B19
:1022700035AB0635FB5B3DA70CBD9B4B30EB19B175
:102280009BE39D8E9F9D8E0001E0000000000120D9
:102290000000000001E0000000000C0F00FE07023B
:1022A0002503BB017FFE08FE08FE050808060000A6
:1022B00040F0C88888987810050808060000C0F823
:1022C0008888888888F80505050600012030F830E0
:1022D000200508080600002070F820202020E005D6
:1022E00009090600FF2070A8A8B888887020070593
:1022F00005070001D86C366CD80509090600FFF8FF
:10230000A88888888888A8F8050A0A0600FE205050
:1023100050505088A8A8887003030306000340A00B
:1023200040FFFFFFFFFFFFFFFFFFFFFFFFFFFFFF7C
:10233000FFFFFFFFFFFFFF0000000605FF0107078B
:102340000602008080808080008003030306010570
:10235000A0A0A005060606000050F85050F8500551
:1023600009090600FF2070A8A07028A870200507A2
:1023700007060000C8C81020409898050707060007
:102380000040A0A040A890680103030602058080D9
:10239000800309090601FF204040808080404020E2
:1023A0000309090601FF80404020202040408005AD
:1023B000070706000020A8702070A8200505050664
:1023C00000012020F820200203030601FFC0408006
:1023D000050101060003F8020202060100C0C00563
:1023E0000707060000081010204040800507070678
:1023F0000000708898A8C88870030707060100408D
:10240000C040404040E00507070600007088081003
:102410002040F8050707060000F80810300888700B
:1024200005070706000010305090F8101005070748
:10243000060000F880F0080888700507070600000D
:10244000304080F0888870050707060000F8081003
:1024500010202020050707060000708888708888F3
:10246000700507070600007088887808106002056C
:1024700005060100C0C000C0C00206060601FFC07C
:10248000C000C040800305050601012040804020B7
:10249000050303060002F800F803050506010180A4
:1024A00040204080050707060000708810202000AB
:1024B000200507070600007088B8A8B880700507D7
:1024C00007060000708888F88888880507070600D6
:1024D00000F04848704848F005070706000070887B
:1024E0008080808870050707060000F0484848484B
:1024F00048F0050707060000F88080F08080F805A6
:102500000707060000F88080F08080800507070636
:102510000000708880809888700507070600008892
:102520008888F8888888030707060100E040404053
:102530004040E005070706000038101010109060BA
:102540000507070600008890A0C0A090880507072F
:10255000060000808080808080F805070706000064
:1025600088D8A8888888880507070600008888C852
:10257000A8988888050707060000708888888888DA
:1025800070050707060000F08888F0808080050746
:102590000706000070888888A8906805070706006D
:1025A00000F08888F0A09088050707060000708872
:1025B0008070088870050707060000F8202020209A
:1025C000202005070706000088888888888870050D
:1025D00007070600008888888850502005070706EE
:1025E000000088888888A8A850050707060000888A
:1025F00088502050888805070706000088885020EA
:10260000202020050707060000F80810204080F869
:102610000309090601FFE080808080808080E0055A
:102620000707060000804040201010080309090633
:1026300001FFE020202020202020E00503030600E9
:10264000052050880501010600FEF803030306017A
:10265000058040200505050600007008788878058B
:1026600007070600008080F0888888F005050506C9
:102670000000708080887005070706000008087851
:10268000888888780505050600007088F080700548
:102690000707060000304840E040404005070706B5
:1026A00000FE70888888780870050707060000809B
:1026B00080F0888888880307070601004000C04032
:1026C0004040E00409090601FE100030101010100F
:1026D000906005070706000080808890E0908803DE
:1026E0000707060100C04040404040E005050506E0
:1026F0000000D0A8A8A8A8050505060000B0C88855
:102700008888050505060000708888887005070719
:102710000600FEF0888888F080800507070600FE26
:1027200078888888780808050505060000B0C88004
:10273000808005050506000078807008F005070711
:102740000600002020F820202018050505060000BE
:1027500088888898680505050600008888885020C4
:102760000505050600008888A8A85005050506008F
:102770000088502050880507070600FE888888508A
:10278000204080050505060000F8102040F80309E8
:10279000090601FF204040408040404020010909D7
:1027A0000602FF8080808080808080800309090687
:1027B00001FF804040402040404080050303060068
:1027C0000248A890FF43616E6E6F74206F70656E53
:1027D00020737562646972200053442063617264DF
:1027E000206F6B0A006F70656E526F6F74206661A8
:1027F000696C65640A00766F6C756D652E696E692B
:1028000074206661696C65640A004E6F2053442031
:10281000636172640A002E0A006F70656E20666143
:10282000696C65642C2046696C653A200046696CC9
:10283000652073656C65637465640A002053697A6A
:10284000653A200046696C65206F70656E65643A74
:102850002000454E4420535542524F5554494E4551
:102860000A002220706F73002220706172656E74FE
:102870003A2200535542524F5554494E4520434148
:102880004C4C207461726765743A22005375626320
:10289000616C6C204F766572666C6F77004578636B
:1028A0006565646564206D617820535542524F55CB
:1028B00054494E452064657074683A0066726573C9
:1028C0006800646F696E67002066696C653A200075
:1028D0004E6F77200057726974696E6720746F209D
:1028E00066696C653A20006D61726C696E66772E60
:1028F0006F726700322E302E392E332D6B616431AA
:10290000001FFFFFFFFFFFFF600000000001FF400E
:102910000000000000FF8000000000007F83CF0067
:10292000000C303F87FF80000C301F867980000C40
:10293000000F8C30C7838C30E78C30CFC7CC31F39D
:102940008C30DCECEC33B98C30D86C6C33198C30B7
:10295000D06C0C33198C30D86C0C33198C30DC6C87
:102960000E3B198C30CF7C079F198C30C77C038FAE
:102970001940000000000002600000000000061F77
:10298000FFFFFFFFFFF870012C0190012701B0014C
:102990002201C0011D01F0011801100213013002D3
:1029A0000E016002090190020401C002FF00000351
:1029B000FA004003F5008003F000D003EB00200490
:1029C000E6007004E100E004DC004005D700C0052B
:1029D000D2004006CD00D006C8008007C3003008F2
:1029E000BE00F008B900C009B400B00AAF00B00BD7
:1029F000AA00D00CA500000EA000500F9B00C01034
:102A000096005012910000148C00C0158700B0177A
:102A10008200B0197D00D01B7800001E730040209A
:102A20006E0090226900F024640040275F00902926
:102A30005A00E02B5500102E500020304B00103271
:102A40004600E033410090353C00103737007038C5
:102A50003200A0392D00B03A2800A03B2300603C92
:102A60001E00103D1900903D1400103E0F00703EF6
:102A70000A00C03E0500003F0000403FFBFF803FD2
:102A8000F6FFC03FF1FF2020506C616E6E65724210
:102A9000756666657242797465733A2000204672E5
:102AA0006565204D656D6F72793A200020436F6D2A
:102AB00070696C65643A2044656320323720323097
:102AC00032310A00204C6173742055706461746562
:102AD000643A20323032312D30392D3033207C2091
:102AE000417574686F723A20286B61642C20416EC6
:102AF000796375626963204D656761205A65726FFD
:102B00002041424C20313256290A004D61726C69D5
:102B10006E20322E302E392E332D6B6164310A0037
:102B200020536F6674776172652052657365740A0D
:102B300000205761746368646F6720526573657421
:102B40000A002042726F776E206F75742052657391
:102B500065740A002045787465726E616C20526558
:102B60007365740A00506F77657255700A0073744C
:102B70006172740A004732385859004D3130303193
:102B8000006572726F722077726974696E67207463
:102B90006F2066696C650A00446F6E65207361760C
:102BA000696E672066696C652E0A004D32390045F2
:102BB0006E6473746F707300255320256320256342
:102BC0002025632025630020503A00205A3A002037
:102BD000593A0020583A00656E6473746F70732020
:102BE0006869743A2000000000010200090A000030
:102BF00000000403080700000000000000000000BF
:102C0000000000000000004D6F76652025736D6D9B
:102C1000004D6F766520302E316D6D004D6F7665FD
:102C200020316D6D004D6F76652031306D6D004D3A
:102C30006F76652041786973004D6F766520457821
:102C4000747275646572004D6F7665205A004D6F21
:102C500076652059004D6F76652058005072696E78
:102C6000742066726F6D204D6564696100FFFFFF1F
:102C7000205A3A200020593A200042656420583AF0
:102C800020004D656761205A65726F20526561644E
:102C9000792E005072696E74696E672E2E2E005068
:102CA00072696E742050617573656400220A005564
:102CB0006E6B6E6F776E20636F6D6D616E643A2020
:102CC00022006F6B00204500205A00205900202070
:102CD0004D3932205800537465707320706572202E
:102CE000756E6974003B2000DB0FC93F45BCDA3FBD
:102CF0008FB30240FCF0274056946140FE4B9B404E
:102D000084A5D840E0231841346A5641E8599741D8
:102D100064DBD5416E271742B4B75542CE1A9742AD
:102D2000C8AED542B5885A43D40684BFA65FA7BFB4
:102D30007443E0BF10B11AC01C2C58C0E8F697C00D
:102D4000B849D6C04E4E17C124D355C1802497C16F
:102D5000A0B5D5C1121A17C244AE55C2781797C292
:102D60006CACD5C267885AC320746F6F206C6F6ECD
:102D70006720657874727573696F6E2070726576FE
:102D8000656E7465640A0020636F6C6420657874F6
:102D9000727573696F6E2070726576656E746564A6
:102DA0000A006F6B0A00526573656E643A2000205A
:102DB000453A00205A3A0020593A00583A0000009B
:102DC0002200250028002B000000210024002700FD
:102DD0002A000202020202020202040404040404A1
:102DE00004040303030303030303010101010101BD
:102DF0000101010204081020408001020408102093
:102E00004080010204081020408080402010080407
:102E100002014572726F722077726974696E672061
:102E2000746F20454550524F4D210A005448455279
:102E30004D414C2052554E415741590054686572DE
:102E40006D616C2052756E6177617900D0D028D7A2
:102E500011241FBECFEFD0E4DEBFCDBF84B7809377
:102E6000331514BE0FB6F894A89580916000886160
:102E700080936000109260000FBE12E0A0E0B1E00D
:102E8000EEE7FAEC01E00BBF02C007900D92AC3800
:102E9000B107D9F725E1ACE8B2E001C01D92A33338
:102EA000B207E1F717E1C7E2D7E104C02197FE01BD
:102EB0000E9487E2C632D107C9F70E947AD10C94EA
:102EC00033E50C940000A0E1B0E0E9E6F7E10C94F2
:102ED000B6E28C01DC01ED91FC910280F381E02DE2
:102EE000BE016F5F7F4F0995882309F45DC089811A
:102EF000807C91F56F81637070E0762F6627770F85
:102F0000770F8885B4E08B9FC0011124682B792B43
:102F100089858295869586958370682B6F5F7F4F34
:102F200090E080E02A852370220F3B8537FB332712
:102F300030F9232B3E813F70230F3327331F275057
:102F4000310904C0660F771F881F991F2A95D2F791
:102F50006096E4E00C94D2E2803419F568856695B9
:102F6000669570E090E080E0CB01772766272A85A0
:102F7000622B098510E0102F0027012E000C220B78
:102F8000330B602B712B822B932B6F5F7F4F8F4FF7
:102F90009F4F4AE0660F771F881F991F4A95D1F708
:102FA000D7CF8BE0F801848360E070E0CB01D0CF15
:102FB0000895FC0182810895FC0190E1A1E7B4E04D
:102FC00001900D929A95E1F70895EF92FF920F9379
:102FD0001F93E0929003F092910300939203109359
:102FE0009303B62F172F022FF32E242F582FB093B1
:102FF000940310939503509396036FEFFF27B01B34
:103000001F09520B30F450951095B195160B560BC5
:10301000662760939204A6E0BA9F00928604712D01
:10302000EE271A9F700DE11D5A9FE00D70938704E3
:10303000E0938804AFE0BA9F00928A04712DEE27D6
:103040001A9F700DE11D5A9FE00D70938B04E09361
:103050008C04AAE0BA9F00928E04712DEE271A9F6D
:10306000700DE11D5A9FE00D70938F04E093900462
:103070001F910F91FF90EF900895A5E0B0E0E3E479
:10308000F8E10C94AFE26F3671058105910578F493
:10309000FB01EE0FFF1FEE0FFF1FEB5FF74F659178
:1030A0007591859194912596EBE00C94CBE2F62EE8
:1030B000E72E282FE5E0F7E00027BB275F2D8E2DB8
:1030C000922F992341F4982F852FB85F992319F4F3
:1030D000982F8827B85F903138F482959295582FB1
:1030E0005F70807F952BBC5F903428F4880F991F08
:1030F000880F991FBE5F903818F4880F991FB395F9
:10310000880F991FE90FF01F549181E09927B8505B
:1031100079F1C0F0B0FF02C0550F881FB1FF04C0A5
:10312000550F881F550F881FB2FF06C08295529514
:10313000152F1F70507F812BB3FF1AC0982F852F3A
:10314000552716C0B195B0FF02C085955795B1FFC0
:1031500004C08595579585955795B2FF05C0829512
:10316000507F5295582B8F70B3FF02C0582F88277D
:10317000BB247727AA27B2E0F59EB0187109A00BEF
:10318000B00BE59E7019A109B00B259FA019B109DC
:10319000F89E7019A109B00BE89EA019B109289FEB
:1031A000B019F99EA019B109E99EB0195B9DA12C37
:1031B00099244427662733278B9DA00C911C401F20
:1031C000601F301F9B9D900C411D601F301F579F3B
:1031D000A00C911C401F601F301F879F900C411D49
:1031E000601F301F979F400D611D301F5A9F900C2C
:1031F000411D601F301F8A9F400D611D301F9A9F27
:10320000600D311D5B9F400D611D301F8B9F600D58
:10321000311D9B9F300DB1E0AA277727BB24F49E78
:10322000B0187109A00BB00BE49E7019A109B00B86
:10323000249FA019B109F69E7019A109B00BE69E52
:10324000A019B109269FB019F39EA019B109E39EF8
:10325000B019BF187E09A20B20F0B1E04B0F601F20
:10326000301F1124762F642F90E0832F1CCFFC0198
:103270007081472F50E0062E02C0559547950A945D
:10328000E2F740FF14C04091090450E0062E02C04E
:10329000559547950A94E2F740FF09C021E030E0D8
:1032A00001C0220F6A95EAF720952723208308950D
:1032B0008F929F92AF92BF92CF92DF92EF92FF9246
:1032C000FC01C080D180E280F38020E030E048EC57
:1032D00052E4C701B6010E9427DC4B015C0120E0EB
:1032E00030E0A901C701B6010E94C2DB20E030E056
:1032F00040EA50E487FF04C020E030E040EA50ECB0
:10330000C501B4010E94E0E22DEC3CEC4CEC5DE325
:103310000E9427DC0E94BFE39B018BE237FF05C0C0
:1033200022273327261B370B8DE280939602C90193
:1033300068EE73E00E9458E2CB01EAE0F0E0BF01E2
:103340000E9458E2805D80939702C90164E670E0B4
:103350000E9458E2CB01BF010E9458E2805D809339
:103360009802C901BF010E9458E29C01CB01BF0134
:103370000E9458E2805D809399028EE280939A02C7
:10338000205D20939B0286E992E0FF90EF90DF9012
:10339000CF90BF90AF909F908F9008954F925F9283
:1033A0006F927F928F929F92AF92BF92CF92DF9255
:1033B000EF92FF92FC01C080D180E280F38020E098
:1033C00030E04AE754E4C701B6010E9427DC4B0114
:1033D0005C0120E030E040E251ECC701B6010E9400
:1033E000C2DB181654F420E030E048EC52E4C70188
:1033F000B6010E9443E487FD8AC020E030E0A901C5
:10340000C701B6010E94C2DB87FF72C060E070E0B6
:1034100080EA90ECA50194010E94E0E22DEC3CECE6
:103420004CEC5DE30E9427DC0E94BFE36B017C0152
:10343000F7FC63C020E137E240E050E00E946BE21D
:10344000CA01B9012AE030E040E050E00E946BE29E
:10345000605D60939602C701B60128EE33E040E05C
:1034600050E00E946BE29AE0892E912CA12CB12CA5
:10347000CA01B901A50194010E946BE2605D6093ED
:103480009702C701B60124E630E040E050E00E9418
:103490006BE2CA01B901A50194010E946BE2605D73
:1034A000609398028EE280939902C701B601A5014C
:1034B00094010E946BE26B01CA01B901A50194015C
:1034C0000E946BE2605D60939A02F0E3CF0EC092BF
:1034D0009B0286E992E0FF90EF90DF90CF90BF9043
:1034E000AF909F908F907F906F905F904F900895D6
:1034F00060E070E080EA90E48DCFF094E094D094A6
:10350000C094C11CD11CE11CF11C6DE2A2CF20E0D3
:1035100030E0A901C701B6010E94C2DB87FF6BC082
:1035200060E070E080EA90ECA50194010E94E0E286
:103530002DEC3CEC4CEC5DE30E9427DC0E94BFE3E9
:103540004B015C0120E030E0A901C701B6010E94F7
:10355000C2DB87FD0BC020E030E040E251E4C70150
:10356000B6010E9443E460E287FD13C0B7FC48C087
:10357000C501B40128EE33E040E050E00E946BE268
:10358000CA01B9012AE030E040E050E00E946BE25D
:10359000605D60939702C501B40124E630E040E02D
:1035A00050E00E946BE28AE0482E512C612C712C75
:1035B000CA01B901A30192010E946BE2605D6093B0
:1035C00098028EE280939902C501B401A301920191
:1035D0000E946BE26B01CA01B901A30192010E9432
:1035E0006BE2605D60939A0280E3C80EC0929B021A
:1035F00087E992E070CF60E070E080EA90E494CFD9
:10360000B094A09490948094811C911CA11CB11C36
:103610006DE2BFCF282F81E3243609F080E280934A
:10362000980290E22A3040F03AE0822F632F0E9405
:103630002BE20E942BE2905D90939902822F6AE028
:103640000E942BE2905D90939A0285E280939B0208
:1036500088E992E0089560912C0170912D01072E68
:10366000000C880B990B0E94C8DB2AE037ED43E27F
:103670005CE30E9427DC60936C0170936D01809382
:103680006E0190936F010895CF93DF93EC01CB010E
:10369000BA010E94C8DB23E333E343E250E40E9413
:1036A00027DC20E030E040E05FE30E94E0E20E949F
:1036B000C4E36883DF91CF9108950E94C8DB23E3C0
:1036C00033E343E250E40E9427DC20E030E040E0B6
:1036D0005FE30E94E0E20E94C4E324E6629FC0012F
:1036E000112481589F4F6FEF70E00E9458E2862F9F
:1036F00091CF80914907811104C080912007809368
:103700007D070895809178148823C1F081508093BB
:103710007814EFECF2E1882351F08150990B2BE102
:10372000289FF001299FF00D1124E659FC4E8BE1F2
:10373000A4EBB2E101900D928A95E1F72091781403
:10374000211105C08091821480648093821481E0ED
:1037500090E0A0E0B0E0211103C080E090E0DC0147
:1037600080933F0790934007A0934107B09342078F
:1037700010923A0781E080933C0783E080936701D1
:103780000895CF93DF93EC01CB01BA010E94C8DB0F
:10379000688379838A839B83DF91CF910895CF9348
:1037A000DF93EC01CB01BA010E94C8DB2DEC3CECAD
:1037B0004CEC5DE30E9427DC688379838A839B83DA
:1037C000DF91CF910895CF93DF93EC01CB01BA0144
:1037D0000E94C8DB2AE037ED43E25CE30E9427DC6D
:1037E000688379838A839B83DF91CF910895CF92F9
:1037F000DF92EF92FF92CF93DF9300D000D0CDB74E
:10380000DEB70E94C8DB2AE037ED43E25CE30E94AA
:1038100027DC6B017C0120E030E0A9010E94C2DBC3
:103820002DEB37E346E055E387FF04C02DEB37E38C
:1038300046E055EBC701B6010E94E0E269837A8356
:103840008B839C83CE010196A9DD0F900F900F9082
:103850000F90DF91CF91FF90EF90DF90CF90089580
:10386000CF93DF93EC01CB01BA010E94C8DB0E9429
:10387000BFE379836883DF91CF9108958F929F9200
:10388000AF92BF92CF92DF92EF92FF92FC01C08085
:10389000D180E280F38020E030E0A901C701B601C9
:1038A0000E94C2DB87FD99C06DEB77E386E095E36C
:1038B000A70196010E94E0E29F7720E030E048EC0B
:1038C00052E40E9427DC20E030E040EA50E40E940D
:1038D000E0E22DEC3CEC4CEC5DE30E9427DC0E9426
:1038E000BFE36B017C0180E28093950260E2F0E12E
:1038F000CF16F7E2DF06E104F1048CF0C701B60150
:1039000020E137E240E050E00E946BE2CA01B901D9
:103910002AE030E040E050E00E946BE2605D60939E
:10392000960260E288EEC81683E0D806E104F1044E
:103930008CF0C701B60128EE33E040E050E00E9471
:103940006BE2CA01B9012AE030E040E050E00E9499
:103950006BE2605D6093970260E2E4E6CE16D1040C
:10396000E104F1048CF0C701B60124E630E040E048
:1039700050E00E946BE2CA01B9012AE030E040E069
:1039800050E00E946BE2605D609398028AE0882EAE
:10399000912CA12CB12CC701B601A50194010E9464
:1039A0006BE26B01CA01B901A50194010E946BE2AF
:1039B000605D609399028EE280939A02F0E3CF0EED
:1039C000C0929B0285E992E0FF90EF90DF90CF904C
:1039D000BF90AF909F908F9008956DEB77E386E056
:1039E00095EB66CFA4E0B0E0E8EFFCE10C94B8E220
:1039F0000E94C8DB2DEC3CEC4CEC5DE30E9427DC24
:103A000069837A838B839C83CE01019637DF24966A
:103A1000E2E00C94D4E2CF93DF93EC018D810E941D
:103A2000608260E08B810E940BC1DF91CF9108958D
:103A3000CF92DF92EF92FF920F931F93CF938C015F
:103A4000C62F69017A01E7DF0E94DDC28C2F8064F6
:103A50000E9454828F2D0E9454828E2D0E94548287
:103A60008D2D0E9454828C2D0E94548287E8C111B2
:103A700001C085E90E945482CC3011F40E94598221
:103A8000C0E00E945982F801868387FF04C0CF3FBF
:103A900011F0CF5FF6CFCF911F910F91FF90EF9074
:103AA000DF90CF90089561E0FC0183810E940BC1FB
:103AB0008FEF0C9454820F931F93CF938C01ABDF45
:103AC0000E94DDC2C82F882369F08DEF0E945482C6
:103AD0000E94DDC2C82FC801E6DF8C2FCF911F9155
:103AE0000F91089582E1F8018483F5CFB0E0A0E062
:103AF000ECE7FDE10C94AEE2EC016A017B014801C8
:103B0000590120E030E0A90167E392DFA5019801A7
:103B100067E1CE018DDF81111DC08F81833039F0C7
:103B200089E0CC0CDD1CEE1CFF1C8A95D1F7A701A7
:103B3000960169E1CE017CDF11E0882319F010E0E5
:103B400087E08C83CE01AFDF812FCDB7DEB7ECE00D
:103B50000C94CAE289E08C8310E0F4CFCF93DF931A
:103B6000EC016EBDFA01CA019E5F0DB407FEFDCFE8
:103B700020812EBD0DB407FEFDCF21812EBD3296D2
:103B8000E817F90791F70DB407FEFDCF8FEF0E94FC
:103B900054828FEF0E9454820E9459828E838F71CB
:103BA000853041F083E18C83CE017DDF80E0DF91C1
:103BB000CF91089581E0FBCF0F931F93CF93DF93B5
:103BC000EC018B0128DF0E94DDC281110BC085E171
:103BD0008C8310E0CE0167DF812FDF91CF911F91A1
:103BE0000F910895A8016CEFCE01B8DF182F88233C
:103BF00071F3F0CF0F931F93CF93DF93EC01890103
:103C00008F81833039F089E0440F551F661F771F7D
:103C10008A95D1F79A01AB0168E1CE0109DF8111E4
:103C200027C0A8016EEFCE0199DF182F8823A9F0D5
:103C30000E94DDC2182F8823C1F020E030E0A901E6
:103C40006DE0CE01F5DE882321F086E18C8310E063
:103C500004C00E9459828111F8CFCE0124DF812F48
:103C6000DF91CF911F910F91089587E18C83F5CF5C
:103C700086E0ECCF1F93CF93DF93EC01CCDE20E006
:103C800030E0A9016CE0CE01D3DE11E0882319F009
:103C900010E083E08C83CE0106DF812FDF91CF918E
:103CA0001F9108951F93CF93DF93EC018F81833091
:103CB00039F089E0440F551F661F771F8A95D1F7A9
:103CC0009A01AB0162E1CE01B3DE11E0882319F065
:103CD00010E085E08C83CE01E6DE812FDF91CF916D
:103CE0001F9108958F929F92AF92BF92EF92FF9291
:103CF0000F931F93CF93DF938C01EB017A010E9406
:103D0000F3C14B015C012CE2820E21E0921EA11C4A
:103D1000B11C0E945982F80186838F3F69F40E948A
:103D2000F3C1681979098A099B0997FDF2CF81E1EE
:103D3000F8018483C0E021C08E3F69F5F1E0EF1AFD
:103D4000F1088FEF8EBDFE012FEF0DB407FEFDCF02
:103D50008EB581932EBDCF018C1B9D0B8E159F05BB
:103D6000A0F30DB407FEFDCF8EB5CE0DDF1D888309
:103D70000E9459820E945982C1E0C80194DE8C2FB2
:103D8000DF91CF911F910F91FF90EF90BF90AF9077
:103D90009F908F9008958FE0CBCF0F931F93CF9379
:103DA000DF93EC018B0137DE40E052E0B801CE0139
:103DB00099DFDF91CF911F910F9108950F931F937A
:103DC000CF93DF93EC0189018F81833039F089E053
:103DD000440F551F661F771F8A95D1F79A01AB01D3
:103DE00061E1CE0125DE882351F084E08C83CE0191
:103DF0005ADE80E0DF91CF911F910F91089540E04E
:103E000052E0B801CE016EDFF5CFB0E0A0E0EBE00C
:103E1000FFE10C94AEE2EC01162F1F821C824B8353
:103E20000E94F3C16B017C0120EDC20E27E0D21E7F
:103E3000E11CF11CA89561E08B810E940BC18B8174
:103E40000E94BFA7249A2C9A279A2698259A81E047
:103E50000E94608285E08D830E9460820AE08FEF7D
:103E60000E9454820150D9F7A89520E030E0A901C2
:103E700060E0CE01DDDD8E83813079F00E94F3C1F8
:103E80006C197D098E099F0997FDEFCF81E08C8326
:103E9000CE0109DE1A8280E065C0A8952AEA31E0E9
:103EA00040E050E068E0CE01C3DD853031F581E0CF
:103EB0008F83A8958F81812C912C5401823029F415
:103EC000812C912CA12C80E4B82E20E030E0A901B7
:103ED00067E3CE01ADDDA501940169E2CE01A8DD65
:103EE0008E838823F1F00E94F3C16C197D098E093D
:103EF0009F0997FDEACF8AE0CACF04E00E94598269
:103F00008E830150D9F78A3A11F482E0D1CF0E9412
:103F1000F3C16C197D098E099F0997FDBFCF82E01F
:103F2000B6CF8F818230B9F420E030E0A9016AE396
:103F3000CE017EDD882311F088E0A9CF0E9459824E
:103F4000807C803C11F483E08F830E9459820E9420
:103F500059820E945982CE01A6DD81E08A83173002
:103F600030F41D83CDB7DEB7ECE00C94CAE288E1F3
:103F70008C8391CF0F931F93CF93DF93EC018B0131
:103F800020E030E0A90169E053DD882351F080E1B1
:103F90008C83CE0188DD80E0DF91CF911F910F915E
:103FA000089540E150E0B801CE019CDEF5CFCF93FB
:103FB000C82FCB010E94B27B89E396E00E94B27BBE
:103FC0008AE296E0CC2311F08FE296E00E94B27B69
:103FD0008AE00E94917BCF9108950C94FFC140919B
:103FE0008E0321E042276CE070E00C9493A740918F
:103FF0008E0321E0422764E070E00C9493A7409187
:104000008E0321E0422761E070E00C9493A7409179
:104010008E0321E0422761E070E00C9493A7409169
:104020008E0321E0422768E070E00C9493A7409152
:104030008E0321E042276CE070E00C9493A741E0EE
:1040400061E070E00C9493A740918E0321E0422739
:104050000C9493A76CE070E00C949AC161E070E05E
:104060000C949AC16CE070E00C949AC164E070E02A
:104070000C949AC19091B90281E089270C949073B5
:1040800061E080E297E00C941C7420E030E0A9012C
:10409000BC0182E791E00C94CDB780E090E0A0E80D
:1040A000B0E480937A0190937B01A0937C01B0935C
:1040B0007D0187E192E0E9DF80E090E0A0EFB1E4EC
:1040C0008093720190937301A0937401B093750172
:1040D0008093760190937701A0937801B093790152
:1040E000E091E603EE0FFF0BE950FE4F80819181D6
:1040F0008330910539F184309105C9F1029761F45B
:1041000080E090E0A3E4B3E48093720190937301A4
:10411000A0937401B09375018FEF91E0B6DF109218
:104120007A0110927B0110927C0110927D0187E14F
:1041300092E0ABDF8091E6038F5F8430ECF48093F4
:10414000E603089580E090E0A3E4B3E48093720175
:1041500090937301A0937401B093750180937601DD
:1041600090937701A0937801B0937901D5CF80E047
:1041700090E0A3E4B3E4F2CF1092E6030895B0E038
:10418000A0E0E5ECF0E20C94B8E220E24F81588523
:104190006E818D810E94BEBCE2E00C94D4E28091DD
:1041A0002007909121070C9434C262E97AE482E0FE
:1041B0000C94CCBE66E97AE481E00C94CCBE6AE94A
:1041C0007AE480E00C94CCBE6EE97AE483E00C944F
:1041D000CCBE10923A070C9413CD4FE350E06AE83E
:1041E00074E08FED96E00C9419E5809104139091A2
:1041F0000513891B8F7011F40C94707581E008957C
:1042000080916701882341F06091DE037091DF03A4
:1042100041E081E00C945EBC0895CF93DF93EC0104
:104220000E94C5C91B82DF91CF910895CF93DF9380
:10423000EC01462F41706C857D858E859F850E949F
:10424000D6C6882351F0888920E2829FC0011124BC
:1042500085599F4EDF91CF91089590E080E0FACF8D
:10426000CF93DF93EB01FC012381211104C080E097
:10427000DF91CF9108952250223028F48FE2888375
:10428000198281E0F5CF60E0D1DF009781F3DC0196
:1042900060E080E09EE22D91203299F0883031F488
:1042A0009E01260F311DF90190836F5F9E01260F3D
:1042B000311DAD0141505109FA014081F90140839E
:1042C0006F5F8F5F8B3039F7FE01E60FF11D1082B3
:1042D000D8CFACE0B0E0EFE6F1E20C94A9E25C01EB
:1042E000DC0159968D909C90F40181859285A3857F
:1042F000B4859C01AD012F5F3F4F4F4F5F4F298722
:104300003A874B875C87D50114964D905D906D90F0
:104310007C901797411451046104710409F459C049
:10432000BFEF4B1A5B0A6B0A7B0A312C73016201E7
:104330001D821E821F821886F40181859285A385C5
:10434000B4852D813E814F815885281739074A074A
:104350005B0708F056C089859A85AB85BC858C15AE
:104360009D05AE05BF0550F482E0C82ED12CE12C8E
:10437000F12C92E0492E512C612C712C9E012F5F63
:104380003F4FB701A601C4010E94E0C88823C9F1CC
:1043900089819A81AB81BC81892B8A2B8B2B01F17E
:1043A000260137019FEF491A590A690A790A2D81B6
:1043B0003E814F8158852F5F3F4F4F4F5F4F2D8379
:1043C0003E834F8358873FEFC31AD30AE30AF30AA9
:1043D000B3CF408051806280738033243394A6CF62
:1043E000C414D504E604F70411F70FEF1FEF2FEF05
:1043F0003FE0B701A601C4010E9466C8782E811172
:1044000006C0712C872D2C96E1E10C94C5E2F501D4
:10441000448155816681778141155105610571059A
:1044200039F097018601C4010E9466C8882349F3C8
:10443000D5011496CD92DD92ED92FC921797332020
:1044400051F0D701C6010196A11DB11DF401808371
:104450009183A283B383F50185899689A789B08D5D
:10446000892B8A2B8B2B71F6C58AD68AE78AF08E28
:10447000818180688183C6CF40E050E0BA010C940E
:104480000ECA4F925F926F927F92AF92BF92CF927D
:10449000DF92EF92FF920F931F93CF93DF931F92C0
:1044A000CDB7DEB78C017B015A01C22EDB015996D4
:1044B0008D919C91F801928F818FCB01DDDF712C62
:1044C000F70180859185A285B385418952896389E9
:1044D000748984179507A607B70708F052C055E0FE
:1044E000B695A795979587955A95D1F7F82FFF70B0
:1044F000DF2ED70113968C91823010F480E0DAC061
:1045000041E050E0BE016F5F7F4FC7010E9409CBC1
:104510000197A1F7F70180859185A285B3854F9614
:10452000A11DB11D80879187A287B387F0E2DF9E2E
:10453000B001112465597F4E61157105F9F2DB0157
:104540008C91882341F0853E09F04BC0772029F0FB
:1045500077247394B5CF71100EC080916B12909137
:104560006C12A0916D12B0916E12F801848795873C
:10457000A687B787D08ADB018C918111E9CF772498
:1045800073948C2D8274823409F0B8CF772009F4AB
:10459000A1C0F801D08861E0C80148DE009709F4A5
:1045A000ADCF20E2DC011D922A95E9F72BE0F50161
:1045B000DC0101900D922A95E1F721E238E2FC013D
:1045C000318B208B40E058E057874687338B228B16
:1045D000318F208F578B468B0E948DC6811109C069
:1045E0008DCF4BE050E0C5010E94C9E4892B09F052
:1045F00067CFF0E2DF9ED00111249D0125593F4E87
:10460000F9018385817121F08C2D827109F000C13F
:10461000F801818D928D40916B1250916C126091D6
:104620006D1270916E124487558766877787D08A9E
:10463000FD01E559FF4E44885588712C612C3201EB
:1046400055244424D80155964D925D926D927C92EA
:104650005897428D538D70E060E0442955296629B2
:10466000772955964D935D936D937C935897D90117
:104670001B962C91287109F0BDC0848D958DA68D57
:10468000B78DF801818B928BA38BB48B81E08383F0
:104690008C2D8F70F8018183148215821682178207
:1046A000108611861286138681E0C4FE03C0C801FD
:1046B0000E9493CA0F90DF91CF911F910F91FF90AD
:1046C000EF90DF90CF90BF90AF907F906F905F9012
:1046D0004F900895D70113968C911397823009F467
:1046E0000DCF51968D919D910D90BC91A02D803E46
:1046F0009F4FAF41B10508F001CFC701EADD882324
:1047000009F4FCCE0E948DC6882309F4F7CED701A8
:104710005996ED91FC915A9714964D905D906D903D
:104720007C901797B2E04B1A510861087108858593
:1047300004C0440C551C661C771C8A95D2F78685EC
:104740009785A089B189480E591E6A1E7B1E81E09B
:1047500080936F1240926B1250926C1260926D12A5
:1047600070926E12EBE6F0E180E092E0DF019C01D6
:104770001D9221503040E1F7DD24D394D7015996A2
:10478000ED91FC918481D816C0F4809170129091C3
:104790007112DC01ED91FC910288F389E02D2BE68A
:1047A00030E1B301A2014D0D511D611D711D09952F
:1047B000882309F4A3CED394E1CF258580E092E04D
:1047C000A0E0B0E004C0880F991FAA1FBB1F2A9564
:1047D000D2F7F7014189528963897489840F951F43
:1047E000A61FB71F818B928BA38BB48B8BE690E1B6
:1047F000D12CD7CE203161F498012F5E3F4F0E941B
:104800005CC9882329F084E0D80113968C9340CFAB
:10481000D80113961C9272CEFC0123812111FDCC8C
:104820000895A1E4B0E0E7E1F4E20C94A8E24C01C1
:104830005B017A01222E19821C821C8E1F8E61154B
:10484000710569F410E0CE014C96E6DFCE010196C9
:10485000E3DF812FCF5BDF4FE2E10C94C4E2FC0188
:1048600083818111EFCFFA0180818F3251F18B0169
:10487000CE0101966C012C0180E2382E3601229681
:104880003FAE229721963FAE21973FAE3EAE3DAE62
:104890003CAE3BAE3AAE39AE38AE3FAA970190E09F
:1048A00047E0D9018D91882309F447C08F3209F47C
:1048B00044C08E3209F54A3029F298E04AE09D0161
:1048C000F0CFFB01838182508230A0F0618D728D28
:1048D000CE014C960E94C4CC882309F4B3CF8E013C
:1048E000045E1F4FC7017C010196F70120812F3222
:1048F000D1F3BECF8B01F6CFE0E7F4E12491222380
:1049000021F031968213FACF9DCF491708F49ACF40
:10491000813208F497CF8F3709F494CF3FE9380FED
:104920003A3108F420EEE7E3F0E0EC0FFD1FE90F69
:10493000F11D820F80839F5FC2CF8FA9803209F45F
:1049400081CF7901F90180812F5F3F4F8F32C9F309
:104950008823C1F021E0AE01495C5F4FB801C60178
:1049600090DD882309F46ECF0A151B0511F0C801EC
:1049700054DCCE014C964C145D0409F0C301860151
:104980006C017DCF222DAE01495C5F4FB801C4019F
:1049900078DD182F58CF8F929F92AF92BF92CF920F
:1049A000DF92EF92FF920F931F93CF93C82F00E8EF
:1049B00012E1F80160857185072E000C880B990BB8
:1049C0000E94C8DB6B017C01F80184809580A68081
:1049D000B78080E20E94917B84E50E94917B8AE30C
:1049E0000E94917B42E0C501B4010E94DEA789E6E6
:1049F00094E10E94B27B42E0C701B6010E94DEA7AB
:104A000062E070E080E090E00E9467C187E1C80248
:104A1000F0011124E058FD4E628570E08CE694E1CF
:104A20000E947681CF911F910F91FF90EF90DF90C0
:104A3000CF90BF90AF909F908F9008950F930FB736
:104A40000F9300916E000B7F00936E0078940F938C
:104A50000BB70F930CB70F921F922F933F934F9367
:104A60005F936F937F938F939F93AF93BF93EF93D6
:104A7000FF9311240E945D58FF91EF91BF91AF9178
:104A80009F918F917F916F915F914F913F912F9166
:104A90001F900F900CBF0F910BBF0F910460F89403
:104AA00000936E000F910FBF0F911895CF93DF9376
:104AB00010929803C0E8D2E1198618860E94FFC1BF
:104AC0001A865D98DF91CF910895EF92FF920F9330
:104AD0001F93CF93C82F7B018A0180911F078330DA
:104AE000E0F00E940D81C7010E94B27B8FEE93E13E
:104AF0000E94B27BC7FD0EC08DEE93E10E94B27B97
:104B00006C2FCC0F770B880B990B0E9494A58AE031
:104B10000E94917B8AE00E94917BC8DFA8958091DA
:104B20008104811128C081E08093810482E0809318
:104B30001F07BCDFC5E1C150149AB9F069E170E00C
:104B400080E090E00E9467C1A895149868E270E048
:104B500080E090E00E9467C1A89568E270E080E084
:104B600090E00E9467C1A895E6CF40E06AEE73E14D
:104B7000C8010E948381CF911F910F91FF90EF9008
:104B80000895CF93DF93A89580918212909183121C
:104B90000E940CA7609384127093851280938612F2
:104BA00090938712C0918212D091831280916001FC
:104BB00090916101C817D90734F44BE254E168E3DE
:104BC00074E180E082DF809188129091891218163A
:104BD00019066CF480915E0190915F018C179D071E
:104BE00034F44AE454E167E574E180E06EDFDF917C
:104BF000CF9108958F929F92AF92BF92CF92DF9202
:104C0000EF92FF92CF93DF9300D000D0CDB7DEB705
:104C100080911F07811110C0A8950F900F900F90E1
:104C20000F90DF91CF91FF90EF90DF90CF90BF90EA
:104C3000AF909F908F900895809182048111EDCF65
:104C400081E08093820480919903811103C01092C6
:104C50008204E3CF96DF109299030E94F3C16B01A7
:104C60007C010E94AFA54B015C01609164017091D1
:104C70006501072E000C880B990B0E94C8DB9B0175
:104C8000AC01C501B4010E9443E418160CF469C0DC
:104C90006091881270918912072E000C880B990B75
:104CA0000E94C8DB69837A838B839C83CE01019643
:104CB0000E943EC28090841290908512A09086122D
:104CC000B09087126091620170916301072E000C11
:104CD000880B990B0E94C8DB9B01AC01C501B40194
:104CE0000E9443E41816CCF4609164017091650150
:104CF000072E000C880B990B0E94C8DB9B01AC01AE
:104D0000C501B4010E94C2DB87FF07C00E94B8A59D
:104D10000E94BFE37595679501C060E060938A12B9
:104D200080917C1290917D12A0917E12B0917F12A1
:104D30000097A105B10509F48ACFC81AD90AEA0A71
:104D4000FB0AF7FC84CF0E94AFA50E94BFE320912D
:104D50007A1230917B126217730754F00E94FFC1E0
:104D600076CF4BE254E168E374E180E0AEDE90CFB1
:104D70004DE054E16CE174E180E0A7DE68CFCF92B2
:104D8000DF92EF92FF92CF93DF93EC01C880D9803E
:104D9000EA80FB8080EE93E10E94B27BC701B601FE
:104DA0000E94D76FCC80DD80EE80FF8087EB9DE294
:104DB0000E94B27BC701B6010E94D76FC884D98414
:104DC000EA84FB8483EB9DE20E94B27BC701B601BB
:104DD0000E94D76F8AE00E94917BDF91CF91FF9074
:104DE000EF90DF90CF900895BC0120916204309144
:104DF000630440916204509163042417350731F431
:104E000081E02617370709F080E008959A01F1CF75
:104E10000F930FB70F9300916E000F930B7F0093CA
:104E20006E0000916F000D7F00936F000F930BB722
:104E30000F930CB70F921F922F933F934F935F9353
:104E40006F937F938F939F93AF93BF93EF93FF9352
:104E50001124D7D5FF91EF91BF91AF919F918F9181
:104E60007F916F915F914F913F912F911F900F9084
:104E70000CBF0F910BBF0F910260F89400936F006D
:104E80000F9100936E000F910FBF0F91189500C006
:104E900000C08091DB0680FF1FC0459A8FEF809392
:104EA0001B048091DB0681FF1AC0479A8FEF809325
:104EB0001C048091DB0682FF15C02A988FEF809337
:104EC0001D048091DB0683FF10C028988FEF80932C
:104ED0001E0400C000C00895459881E0E0CF4798C7
:104EE00081E0E5CF2A9A81E0EACF289A81E0EFCFEE
:104EF00080918F03982F977F90938F03982F9370B3
:104F000081E011F080E008955E9A08955E988091A6
:104F10008F03886080938F030895E82FF0E021E0ED
:104F200030E0082E02C0220F331F0A94E2F72095CA
:104F3000309590918F03922390938F03ED50FE4F05
:104F40002081922321E019F020E0822F0895813002
:104F500079F038F08230C9F7159A90914D079B7F10
:104F600004C05E9A90914D079E7F90934D07EDCFC0
:104F70005E9A90914D079D7FF8CF80E0CEDF81E073
:104F8000CCDF82E0CADFB4CF813079F070F08230BC
:104F900071F021E030E001C0220F8A95EAF780919C
:104FA0008F03822B80938F0308955E98F2CF15981C
:104FB000F0CFB0E0A0E0EFEDF7E20C94B2E2C82F42
:104FC00063EB7BE00E940BB8C11102C00E9410810C
:104FD0008BEA9BE00E94B27B87E19BE00E94B27B60
:104FE0008AE00E94917B69E97BE08C2F0E940BB8DC
:104FF000C11102C00E9410818CE79BE00E94B27B2D
:105000008C2F0E942BB88C2F0E944E808C2F0E94D8
:1050100075808C2F0E942E808C2F0E94FA7F63E374
:105020007BE08C2F0E9422B8D091B9028AE29BE0EB
:105030000E94B27B6D2F70E090E080E00E9494A50A
:105040004091B5025091B6026091B7027091B802DA
:1050500088EC9CE20E94DD7B8DE19BE00E94B27BAC
:105060008091B9020E94038120E030E0A9016091A3
:10507000BA027091BB028091BC029091BD020E9465
:10508000C2DB8823A1F18AECE82E82E0F82E10E042
:10509000670100E0C11102C00E94108182E79BE01D
:1050A0000E94B27B802F0E94B3718FE69BE00E942A
:1050B000B27B812F0E94B37188EC9CE20E94B27B8C
:1050C000F601608171818281938145E00E94DEA7B3
:1050D0008AE00E94917B0F5FFCE1CF0ED11C07306C
:1050E000C9F61F5F84E0E80EF11C173089F664E50D
:1050F0007BE08C2F0E940BB802EC12E0D0E0C111D3
:1051000002C00E9410818BE49BE00E94B27B8D2F35
:105110000E94B371F80160817181072E000C880B29
:10512000990B0E94C8DBAB01BC0188E49BE00E94A4
:10513000DD7BF801E280F38085E49BE00E94B27B96
:10514000C7010E946B758AE00E94917B0C5F1F4F24
:10515000D13059F48C2F0E9438818C2F0E94EE7B25
:10516000CDB7DEB7E8E00C94CEE2D1E0C8CFB0E036
:10517000A0E0EDEBF8E20C94B0E2CFE3DDE005E671
:1051800017E08FE4A82E8DE0B82EC12CD12C76012B
:10519000C39469917991899199910E94C6DB28897C
:1051A00039894A895B890E9427DC0E94C4E3F8019F
:1051B00061937193819391938F01C616D706E80688
:1051C000F90610F46B017C01AC16BD0611F76FEF08
:1051D0007FEFCB01A70196010E94F0E120937507B4
:1051E000309376074093770750937807CDB7DEB7B3
:1051F000EAE00C94CCE20F931F93CF93DF9303E587
:105200001DE0CEE7D7E0F801219131914191519114
:105210008F0160E070E080E89FE30E9457E36993AC
:10522000799389939993F7E0CE38DF0761F70E946D
:10523000F0B79DDFDF91CF911F910F910895DBCFE4
:10524000DACFD9CFD8CF909104138091051398135A
:1052500006C08091870D9091880D892B21F080E008
:105260000E947182F0CF08959091041380910513EC
:10527000981307C08091870D9091880D892B09F4B0
:105280007CCE80E00E947182EFCFCF92DF92EF92CE
:10529000FF92CF93DF932091B902222319F1EC0101
:1052A00008960E943B716B017C0120E030E0A9016F
:1052B0000E94C2DB20E030E0A901882349F0CE0142
:1052C0000E94B971A70196010E9427DC9B01AC01E5
:1052D000688579858A859B850E94DFE26887798762
:1052E0008A879B87DF91CF91FF90EF90DF90CF90DF
:1052F0000895CF92DF92EF92FF92CF93DF932091A8
:10530000B902222319F1EC0108960E943B716B014E
:105310007C0120E030E0A9010E94C2DB20E030E007
:10532000A901882349F0CE010E94B971A701960115
:105330000E9427DC9B01AC01688579858A859B8565
:105340000E94E0E2688779878A879B87DF91CF9107
:10535000FF90EF90DF90CF900895AEE1B0E0E3EBE7
:10536000F9E20C94AAE29E8F8D8F5B018A01FC0109
:10537000EA5BFF4F2081318142815381298B3A8B37
:105380004B8B5C8BCA01B9010E94C6DB6B017C01AF
:10539000D5012D913D914D915C910E9427DC0E9499
:1053A00044E32B013C01F80120813181428153818A
:1053B000C701B6010E9427DC0E9444E34B015C0157
:1053C000C301B2010E94C4E36D8B7E8B8F8B988FDB
:1053D000683771058105910540F428E730E040E029
:1053E00050E02D8B3E8B4F8B588FC501B4010E942E
:1053F000C4E3698F7A8F8B8F9C8F68377105810525
:10540000910540F488E790E0A0E0B0E0898F9A8FA2
:10541000AB8FBC8FED8DFE8DEE5AFF4F2081318119
:105420004281538129873A874B875C87CA01B9013A
:105430000E94C8DB2B013C016D897E898F89988D84
:105440000E94C6DB6D837E838F83988720E030E0E7
:10545000A901C301B2010E94C2DB882309F4BBC1C8
:10546000A7019601C701B6010E9427DC4B015C0130
:105470002D813E814F815885CA01B9010E9427DCE8
:105480009B01AC01C501B4010E94DFE24B015C014C
:10549000A3019201C301B2010E94E0E29B01AC01B1
:1054A000C501B4010E9457E30E9444E30E94C4E393
:1054B00069837A838B839C8369857A858B859C85B8
:1054C00090958095709561957F4F8F4F9F4F0E946B
:1054D000C8DB4B015C01698D7A8D8B8D9C8D0E94A0
:1054E000C6DB69877A878B879C8720E030E0A9013B
:1054F000C501B4010E94C2DB882309F470C129856B
:105500003A854B855C85CA01B9010E9427DC6D870D
:105510007E878F87988BA7019601C701B6010E94ED
:1055200027DC9B01AC016D857E858F8598890E9463
:10553000DFE26B017C01A5019401C501B4010E9469
:10554000E0E29B01AC01C701B6010E9457E30E9453
:10555000F0E3AD8DBE8D95962D913D914D915C9171
:1055600098972D873E874F87588B69017A0129814B
:105570003A814B815C81C21AD30AE40AF50A0E947F
:10558000C4E3C61AD70AE80AF90AF7FE8CC02D81CF
:105590003E814F815885CA01B9010E9427DC6B0109
:1055A0007C0120E030E0A901C301B2010E94C2DB0E
:1055B000882309F418C16D857E858F8598890E949E
:1055C000C6DB9B01AC010E94E0E2A30192010E94B4
:1055D00027DC4B015C0129853A854B855C85CA0136
:1055E000B9010E9427DC9B01AC01C501B4010E94F6
:1055F000E0E2A70196010E94DFE24B015C0120E09E
:1056000030E040E850E4C301B2010E9427DC9B0176
:10561000AC01C501B4010E9457E30E9444E34B0171
:105620005C0120E030E0A9010E9443E487FF03C051
:10563000812C912C5401C501B4010E94C4E36983FB
:105640007A838B839C832D853E854F8558892617C9
:1056500037074807590720F429833A834B835C8333
:1056600069817A818B819C810E94C6DB4B015C0140
:10567000A3019201C301B2010E94E0E29B01AC01CF
:10568000C501B4010E9427DCA70196010E94E0E257
:105690000E947CE40E94C4E3698B7A8B8B8B9C8B89
:1056A000C12CD12C760169897A898B899C892D89B5
:1056B0003E894F89588D621B730B840B950B0E949A
:1056C000C6DBA30192010E9457E320E034E244EFDD
:1056D00059E40E9427DC0E94C4E34B015C01698904
:1056E0007A898B899C89298D3A8D4B8D5C8D621BC3
:1056F000730B840B950B0E94C6DBA30192010E94E1
:1057000057E320E034E244EF59E40E9427DC0E9492
:10571000C4E36D837E838F839887C501B4010E94A3
:105720003D182B013C016D817E818F8198850E94FF
:105730003D1829813A814B815C81AD8DBE8D999652
:105740002D933D934D935C939C9789019A010C0D89
:105750001D1D2E1D3F1DFD0105A716A727A730AB58
:10576000E65BFF4F2D893E894F89588D2083318319
:1057700042835383D5968D929D92AD92BC92D897D9
:105780002D813E814F815885D9962D933D934D9320
:105790005C93DC973D97408251826282738234969B
:1057A000608371838283938329893A894B895C89D9
:1057B000D1962D933D934D935C93D4973D96298D2F
:1057C0003A8D4B8D5C8D20833183428353836E965B
:1057D000E0E10C94C6E260E070E0CB0165CE60E0F1
:1057E00070E0CB01B4CE60E070E0CB0116CF9091B9
:1057F0006F0081E091FD02C080E0089590916F00FC
:105800009D7F90936F000895EFE6F0E080818260C5
:1058100080830895CF93C82FEADF94E0C99F900159
:105820001124F901EB59FB4F2F583B4FD9014D91F2
:105830005D916D917C91408351836283738391E08C
:10584000909364048111E0DFCF910895CF93DF93AB
:105850008091DA06811105C08091DC06882309F465
:1058600064C08091F603329B63C081608093F6032D
:105870008091F603339B5EC082608093F603809133
:10588000F603349B59C084608093F6038091F6033D
:10589000029B54C088608093F603C0915504C0FFFA
:1058A0000FC08091DB0680FF0BC08091F60380FF64
:1058B00007C080914C07816080934C0780E0AADF8D
:1058C000C1FF0FC08091DB0681FF0BC08091F60302
:1058D00081FF07C080914C07826080934C0781E074
:1058E00099DFC2FF22C08091DB0682FF1EC080913B
:1058F000DC0681110BC08091F60382FF07C0809106
:105900004C07846080934C0782E084DF8091DC0642
:10591000882359F08091F60383FF07C080914C07DC
:10592000886080934C0782E075DFDF91CF91089506
:105930008E7F9CCF8D7FA1CF8B7FA6CF877FABCF74
:1059400056DF1092790710927A0710927B07109217
:105950007C07811159CF08950F931F9380910413F1
:1059600090910513891B8F7009F449C09091011320
:10597000992361F0833040F48FEF890F29F08093F1
:10598000011390E080E038C010920113809105135C
:105990002BE5829FC00111248257984FFC01208182
:1059A00020FDEFCF4091790750917A0760917B07F6
:1059B00070917C07E95AFF4F008111812281338168
:1059C000401B510B620B730B4093790750937A077E
:1059D00060937B0770937C07209105132F5F2F70D6
:1059E000209302133091051320910313321304C046
:1059F00020910213209303131F910F910895A0DFAC
:105A0000C0CFA3E1B0E0E7E0FDE20C94A8E28FEFA5
:105A10009FEF90938900809388002AE02983312C9E
:105A2000212C789480915E0490915F04A091600491
:105A3000B0916104892B8A2B8B2B09F0C2C1809114
:105A400064048823D1F080916204909163041092E1
:105A50006404892B91F010926304109262041092F6
:105A600055049091041380910513981731F080919B
:105A700005138F5F8F70809305138091620490915E
:105A80006304892B09F49DC140915A0450915B0431
:105A900060915C0470915D0480915604909157046C
:105AA000A0915804B091590400914C0410E030E0EA
:105AB00020E0841B950BA60BB70B081719072A07C4
:105AC0003B0710F4D901C8018A8B840F951FA61FCC
:105AD000B71F80935A0490935B04A0935C04B09327
:105AE0005D04E1E0C0902304D0902404E0902504FC
:105AF000F09026048091330490913404A0913504F1
:105B0000B0913604C80ED91EEA1EFB1EC0923304A3
:105B1000D0923404E0923504F0923604F7FC33C09E
:105B200040911B04042E000C550B660B770B8091E3
:105B3000710490917204A0917304B0917404840F65
:105B4000951FA61FB71F8093710490937204A093B2
:105B50007304B093740480911F0490912004A09169
:105B60002104B0912204B701A601481B590B6A0B0E
:105B70007B0BDB01CA018093330490933404A09320
:105B80003504B09336040091270410912804209125
:105B9000290430912A048091370490913804A0910F
:105BA0003904B0913A04080F191F2A1F3B1F0093B4
:105BB0003704109338042093390430933A0437FDA6
:105BC00033C040911C04042E000C550B660B770B60
:105BD0008091750490917604A0917704B091780437
:105BE000840F951FA61FB71F8093750490937604AA
:105BF000A0937704B093780480911F0490912004BF
:105C0000A0912104B091220428013901481A590AAF
:105C10006A0A7B0AD301C201809337049093380447
:105C2000A0933904B0933A0440912B0450912C0472
:105C300060912D0470912E0480913B0490913C045E
:105C4000A0913D04B0913E04480F591F6A1F7B1F6D
:105C500040933B0450933C0460933D0470933E0496
:105C600077FD33C080901D04082C000C9908AA0809
:105C7000BB088091790490917A04A0917B04B09143
:105C80007C04880D991DAA1DBB1D809379049093F7
:105C90007A04A0937B04B0937C0480911F049091BC
:105CA0002004A0912104B09122043A014B01681A0A
:105CB000790A8A0A9B0AD401C30180933B0490931A
:105CC0003C04A0933D04B0933E0480902F04909038
:105CD0003004A0903104B090320480913F04909140
:105CE0004004A0914104B0914204880D991DAA1D61
:105CF000BB1D80933F0490934004A0934104B09354
:105D00004204B7FD33C040901E04042C000C55081B
:105D10006608770880907D0490907E04A0907F04B0
:105D2000B0908004840C951CA61CB71C80927D0446
:105D300090927E04A0927F04B092800480901F0411
:105D400090902004A0902104B09022042C013D01E9
:105D5000481859086A087B085301420180923F04A1
:105D600090924004A0924104B0924204E11104C018
:105D7000E0918400F0918500F7FE5F9A37FF469A24
:105D800077FF2B9AB7FF299AE0918400F091850064
:105D9000E0918400F0918500F7FE5F9837FF469808
:105DA00077FF2B98B7FF29985A88552021F08091CA
:105DB0008400909185002A8921502A8BE0E02111EE
:105DC00091CE80915E0490915F04A0916004B091A7
:105DD0006104892B8A2B8B2B09F0B0C6409062049A
:105DE000509063045B8A4A8A4114510409F402C743
:105DF00080915A0490915B04A0915C04B0915D0481
:105E00004091560450915704609158047091590480
:105E100084179507A607B70708F449C010926304D2
:105E2000109262041092550490910413809105130E
:105E3000981709F4DFC6809105138F5F8F708093E8
:105E40000513A0EDCA2EA7E0DA2EE12CF12C8091EB
:105E5000620490916304892B09F068C67DDD9093FC
:105E6000630480936204892B09F460C64090620445
:105E7000509063045B8A4A8AD2018C9183FF08C5E3
:105E8000C20145960E94DC171092630410926204CE
:105E90001092550490910413809105139817F1F214
:105EA000809105138F5F8F7080930513D7CF40913A
:105EB0005104509152046091530470915404481756
:105EC00059076A077B0708F40FC240914D045091AF
:105ED0004E0460914F0470915004EA89FB8985A9B2
:105EE00096A9A7A9B0AD481759076A077B0708F01C
:105EF000D0C1411551056105710509F066C080905A
:105F0000940390909503A0909603B090970380EC33
:105F100093E1A1E0FC0105911591259134910815BB
:105F200019052A053B0558F4B694A79497948794CD
:105F3000AA0F0496ECEDF3E1E817F90759F7A093DF
:105F40004C04F0E28F169104A104B10428F4E0E2BD
:105F50008E2E912CA12CB12C20E2821A9108A1083E
:105F6000B108811438E09306A104B10408F49AC181
:105F7000A4E09A9EC00111248054904FFC013296F7
:105F800025913491B82DEE27B39F8001B29F010D6A
:105F90001E1F06940E1F1E1F112430E020E0FC017E
:105FA000C590D490F12CE12CC01AD10AE20AF30A70
:105FB0004C0D5D1D6E1D7F1D40934D0450934E048E
:105FC00060934F047093500442CF10E00A81942FE5
:105FD000852E862FBC81AD81FE81EF813885298594
:105FE0004B80E0919003E99FA12DFF273091910311
:105FF000399FA00DF11D10909203199EF00DE89DA0
:10600000A00DF11D389DF00DE89FF00D4A2EBF2F19
:106010004A9EE12D332722274F9EE00D311D211F7F
:10602000BA9FE00D311D211FBF9F300D211D432E52
:10603000B22F4A9E012D332722274F9E000D311D7E
:10604000211FBA9F000D311D211FBF9F300D211D43
:10605000432EB22FEE279091940380909503809168
:10606000960300909204012A09F483C030918E04B3
:10607000349DE119910B810A810B20918F04249D9D
:10608000E0199109810A810B00919004049D9019F7
:106090008108810B3B9FE0199109810A810B2B9F9D
:1060A00090198108810B0B9F801881094A9E012D50
:1060B000332722274F9E000D311D211FBA9F000D4F
:1060C000311D211FBF9F300D211D432EB22F309156
:1060D0008A04349DE10D911F811E811F20918B0444
:1060E000249DE00D911D811E811F00918C04049D53
:1060F000900D811C811F3B9FE00D911D811E811F12
:106100002B9F900D811C811F0B9F800C811D4A9E2F
:10611000012D332722274F9E000D311D211FBA9FCD
:10612000000D311D211FBF9F300D211D432EB22FA9
:1061300030918604349DE119910B810A810B2091E5
:106140008704249DE0199109810A810B009188043C
:10615000049D90198108810B3B9FE0199109810AE8
:10616000810B2B9F90198108810B0B9F801881094F
:1061700082C030918E04349DE10D911F811E811FDC
:1061800020918F04249DE00D911D811E811F00919F
:106190009004049D900D811C811F3B9FE00D911D7B
:1061A000811E811F2B9F900D811C811F0B9F800CD6
:1061B000811D4A9E012D332722274F9E000D311D40
:1061C000211FBA9F000D311D211FBF9F300D211DC2
:1061D000432EB22F30918A04349DE119910B810A2C
:1061E000810B20918B04249DE0199109810A810B78
:1061F00000918C04049D90198108810B3B9FE0194C
:106200009109810A810B2B9F90198108810B0B9FAB
:10621000801881094A9E012D332722274F9E000DA9
:10622000311D211FBA9F000D311D211FBF9F300D51
:10623000211D432EB22F30918604349DE10D911F14
:10624000811E811F20918704249DE00D911D811ED8
:10625000811F00918804049D900D811C811F3B9F2C
:10626000E00D911D811E811F2B9F900D811C811FB0
:106270000B9F800C811D11244B820A83BC83AD834C
:10628000FE83EF8338872987982C892EB12CA82E7E
:106290003ECEAA89BB89D1968D909D90AD90BC9041
:1062A000D49735CED501C401B695A7959795879516
:1062B0008C7F8054944FFC01C590D490FC013296A1
:1062C00025913491E82DE7708E2EE29FC001E39F67
:1062D000900D112433E0969587953A95E1F7C81A09
:1062E000D90AF12CE12C64CE409148045091490424
:1062F00060914A0470914B04481759076A077B075D
:1063000008F030C28090430490904404A09045046B
:10631000B090460480914704EA89FB8981117CC0D2
:10632000EF5BFF4FE080F18002811381EA89FB89F6
:10633000E25BFF4F2081318142815381AA89BB8971
:10634000D1966D917D918D919C91D4970E94E51786
:10635000B1E0B0934704EA89FB8941A952A963A936
:1063600074A980EC93E1A1E0FC01059115912591C0
:106370003491041715072607370758F47695679563
:1063800057954795AA0F0496ECEDF3E1E817F90746
:1063900059F7A0934C04403251056105710520F472
:1063A00040E250E060E070E040525109610971093B
:1063B0004115F8E05F076105710508F4B3C124E0F9
:1063C000529FC00111248054904FFC0132962591B8
:1063D0003491AA27439FF001429FE10DFA1F0694D2
:1063E000EA1FFA1F1124AF0170E060E0FC01C590C4
:1063F000D490F12CE12CC41AD50AE60AF70A8C0CC9
:106400009D1CAE1CBF1C8092430490924404A09239
:106410004504B09246041BCD81AD92ADA3ADB4ADA1
:1064200088169906AA06BB0608F072C18114910469
:10643000A104B10449F440919403509195036091F3
:106440009603709197038DCFA0E0BA85982D492DC2
:106450008A2DFB85EC857D856E855F853889298948
:1064600050919003599F712D662730919103399F68
:10647000700D611D10909203199E600D549F700D58
:10648000611D349F600D589F600DF72FE62FF79F19
:10649000512D33272227F69F500D311D2A1FE79FCC
:1064A000500D311D2A1FE69F300D211DF32FE22FC5
:1064B000F79FB12D33272227F69FB00D311D2A1FDC
:1064C000E79FB00D311D2A1FE69F300D211DF32FD0
:1064D000E22F552790919403409195038091960364
:1064E000009092040A2A09F483C030918E043F9FE1
:1064F00051199A0B4A0B8A0B20918F042F9F501928
:1065000091094A0B8A0BB0919004BF9F90194109E1
:106510008A0B3E9F501991094A0B8A0B2E9F9019A6
:1065200041098A0BBE9F40198109F79FB12D33277E
:106530002227F69FB00D311D2A1FE79FB00D311D98
:106540002A1FE69F300D211DF32FE22F30918A0480
:106550003F9F510D9A1F4A1F8A1F20918B042F9F26
:10656000500D911D4A1F8A1FB0918C04BF9F900D42
:10657000411D8A1F3E9F500D911D4A1F8A1F2E9F4D
:10658000900D411D8A1FBE9F400D811DF79FB12DAB
:1065900033272227F69FB00D311D2A1FE79FB00D2C
:1065A000311D2A1FE69F300D211DF32FE22F309160
:1065B00086043F9F51199A0B4A0B8A0B209187043E
:1065C0002F9F501991094A0B8A0BB0918804BF9FE5
:1065D000901941098A0B3E9F501991094A0B8A0B69
:1065E0002E9F901941098A0BBE9F4019810982C0D4
:1065F00030918E043F9F510D9A1F4A1F8A1F209190
:106600008F042F9F500D911D4A1F8A1FB091900437
:10661000BF9F900D411D8A1F3E9F500D911D4A1F27
:106620008A1F2E9F900D411D8A1FBE9F400D811D08
:10663000F79FB12D33272227F69FB00D311D2A1F5A
:10664000E79FB00D311D2A1FE69F300D211DF32F4E
:10665000E22F30918A043F9F51199A0B4A0B8A0B03
:1066600020918B042F9F501991094A0B8A0BB091EE
:106670008C04BF9F901941098A0B3E9F50199109C4
:106680004A0B8A0B2E9F901941098A0BBE9F401915
:106690008109F79FB12D33272227F69FB00D311DB9
:1066A0002A1FE79FB00D311D2A1FE69F300D211DC7
:1066B000F32FE22F309186043F9F510D9A1F4A1FFE
:1066C0008A1F209187042F9F500D911D4A1F8A1FFA
:1066D000B0918804BF9F900D411D8A1F3E9F500DB1
:1066E000911D4A1F8A1F2E9F900D411D8A1FBE9F1C
:1066F000400D811D1124BA87FB87EC877D876E874B
:106700005F87388B298B542F492F70E0682F29CE53
:106710002A893B89225B3F4FD9014D915D916D9153
:106720007C911FCEDB01CA01B695A79597958795F9
:106730008C7F8054944FFC01C590D490FC0132961C
:10674000259134914770429FC001439F900D1124C1
:10675000A3E096958795AA95E1F7C81AD90AF12C76
:10676000E12C4DCE80912E0190912F01A09130010E
:10677000B0913101B7FF61C0EA89FB89EA5BFF4F45
:10678000C080D180E280F38080EC93E121E0FC01C5
:1067900045915591659174914C155D056E057F0588
:1067A00058F4F694E794D794C794220F04964CEDCE
:1067B00053E14817590759F720934C0450E2C51686
:1067C000D104E104F10428F470E2C72ED12CE12CAD
:1067D000F12C60E2C61AD108E108F108C11478E092
:1067E000D706E104F10408F431C0A4E0DA9EC00148
:1067F00011248054904FFC01329625913491BC2D88
:106800006627B39FA001B29F410D561F0694461FF5
:10681000561F112470E060E0FC0185919491B0E076
:10682000A0E0841B950BA60BB70B80932E019093D1
:106830002F01A0933001B0933101C0902E01D09070
:106840002F01E0903001F090310101CBD701C6015A
:10685000B695A795979587958C7F8054944FFC01AA
:1068600025913491FC01329645915491EC2DE770BD
:10687000E49FC001E59F900D112463E096958795F4
:106880006A95E1F7281B390BC901B0E0A0E0CDCF34
:10689000EA89FB8985889688A788B08C81E0811475
:1068A0009104A104B10409F480E0AA89BB89599636
:1068B000CD90DD90ED90FC905C97C114D104E10483
:1068C000F10409F08260EA89FB89458D568D678D58
:1068D00070A1411551056105710509F0846080932F
:1068E00055041092430410924404109245041092EF
:1068F000460410924D0410924E0410924F041092D0
:106900005004EA89FB8985A196A1A7A1B0A580932F
:10691000560490935704A0935804B0935904442408
:1069200055243201481A590A6A0A7B0A40923304F4
:1069300050923404609235047092360440923704C9
:10694000509238046092390470923A0440923B04A9
:1069500050923C0460923D0470923E0441A052A0CB
:1069600063A074A0440C551C661C771C880C991CF1
:10697000AA1CBB1C8092230490922404A09225049C
:10698000B0922604CC0CDD1CEE1CFF1CC092270428
:10699000D0922804E0922904F0922A04440F551F53
:1069A000661F771F40932B0450932C0460932D0493
:1069B00070932E0440922F04509230046092310460
:1069C00070923204880F991FAA1FBB1F80931F0467
:1069D00090932004A0932104B093220410925A04AF
:1069E00010925B0410925C0410925D0481A592A544
:1069F000A3A5B4A58093510490935204A09353048B
:106A0000B093540485A596A5A7A5B0A98093480482
:106A100090934904A0934A04B0934B04EB5BFF4F5F
:106A200080819091DB06891721F08093DB060E941C
:106A300047270E94262C44244A94542C3201409229
:106A40002E0150922F016092300170923101EA893B
:106A5000FB89FD96E080F18002811381AA89BB89C0
:106A6000D1962D913D914D915C91D4976D01BAE4F1
:106A7000CB0ED11CF60160817181828193810E94CD
:106A8000E51710924704D6014D915D916D917C916F
:106A900080EC93E1A1E0FC010591159125913491E1
:106AA000041715072607370758F476956795579505
:106AB0004795AA0F0496ECEDF3E1E817F90759F7AB
:106AC000A0934C04403251056105710520F440E269
:106AD00050E060E070E040525109610971094115D0
:106AE000F8E05F076105710508F462C024E0529F79
:106AF000C00111248054904FFC01329625913491AD
:106B0000AA27439FF001429FE10DFA1F0694EA1F56
:106B1000FA1F1124AF0170E060E0FC01C590D49031
:106B2000F12CE12CC41AD50AE60AF70AC0925E04D9
:106B3000D0925F04E0926004F092610480915E0460
:106B400090915F04A0916004B0916104AC01BD011B
:106B5000009731E0A307B10520F04FEF5FEF60E051
:106B600070E0841B950BA60BB70B80935E0490938B
:106B70005F04A0936004B0936104F8948091840052
:106B8000909185004096A981A150A983AA2381F103
:106B9000240E351E2816390610F40C94112D30924F
:106BA00089002092880078946396E2E10C94C4E214
:106BB000DB01CA01B695A795979587958C7F805480
:106BC000944FFC01C590D490FC01329625913491EC
:106BD0004770429FC001439F900D112433E096956A
:106BE00087953A95E1F7C81AD90AF12CE12C9ECF86
:106BF0001C01D5CF80EDC82E87E0D82EE12CF12CDA
:106C00002DC9CF93DF938091041390910513891BB5
:106C100080958F7019F40E947182F5CF80910413D2
:106C20008F5F8F70A09104139BE5A99FD001112461
:106C3000FD01E257F84FEF0119929A95E9F798E0B4
:106C40009083AD55B84F90E1E6E0F3E101900D92ED
:106C50009A95E1F72091041390910513291303C02D
:106C600094E690930113809304130E94042CDF9107
:106C7000CF910895FC01208131814281538160913F
:106C80005F0D7091600D8091610D9091620D0E9479
:106C900027DC0E9448E460931213709313138093CF
:106CA0001413909315139091041380910513981762
:106CB00009F0A7CF0E9423290E94F72B40911213BD
:106CC00050911313609114137091151340937D0428
:106CD00050937E0460937F047093800481110C9420
:106CE000042C08954F925F926F927F928F929F92A1
:106CF000AF92BF92CF92DF92EF92FF92CF93DF934A
:106D0000EC0120915F0D3091600D4091610D50912B
:106D1000620D6C857D858E859F850E9427DC0E9493
:106D200048E46B017C0120915B0D30915C0D40913A
:106D30005D0D50915E0D688579858A859B850E94E1
:106D400027DC0E9448E44B015C012091570D3091F3
:106D5000580D4091590D50915A0D6C817D818E8155
:106D60009F810E9427DC0E9448E42B013C01209176
:106D7000530D3091540D4091550D5091560D688131
:106D800079818A819B810E9427DC0E9448E460937C
:106D9000061370930713809308139093091340927E
:106DA0000A1350920B1360920C1370920D13809281
:106DB0000E1390920F13A0921013B0921113C09261
:106DC0001213D0921313E0921413F09215139091B2
:106DD000041380910513981781F013DFDF91CF9191
:106DE000FF90EF90DF90CF90BF90AF909F908F90EB
:106DF0007F906F905F904F9008950E9423290E948A
:106E0000F72BC82F86E093E10E94DC17CC2331F3E7
:106E10000E94042CE3CFCF92DF92EF92FF92CF93A8
:106E2000DF93C82F0E94F72B94E0C99FE001112443
:106E3000FE01EF58FB4FC080D180E280F3808111CA
:106E40000E94042CC258D84FC701B6010E94C8DB6B
:106E5000288139814A815B810E9427DCDF91CF91B3
:106E6000FF90EF90DF90CF900895CF92DF92EF9256
:106E7000FF92CF93DF93C82F0E94F72B94E0C99F16
:106E8000E0011124FE01EB59FB4FC080D180E2806C
:106E9000F38081110E94042CC258D84FC701B6015B
:106EA0000E94C8DB288139814A815B810E9427DCEE
:106EB000DF91CF91FF90EF90DF90CF900895A1E008
:106EC000B0E0E5E6F7E30C94B8E2898360E0CE0138
:106ED00001960E94371961E0CE0101960E94371990
:106EE00062E0CE0101960E94371989812196E2E085
:106EF0000C94D4E2A2E1B0E0E0E8F7E30C94B4E251
:106F0000DEDF8823C1F1EDB6FEB64AE852E082FF2B
:106F100002C041E852E02AE832E081FF02C023E8E3
:106F200032E080FD25C08AE892E05F934F933F9363
:106F30002F939F938F938AEA96E09F938F938E016E
:106F40000F5F1F4F1F930F930E945BDB0E94108106
:106F5000C8010E94A37BC8010E9439B70FB6F894FC
:106F6000DEBF0FBECDBF81E06296E6E00C94D0E2BA
:106F700085E892E0DACF80E0F7CFA0E2B0E0E3EC82
:106F8000F7E30C94A8E280911201882309F4BEC0B3
:106F900080910904082F10E080FF3CC0C0901401CC
:106FA000D0901501E0901601F090170120919D02FC
:106FB00030919E0240919F025091A002C701B601FC
:106FC0000E9443E4181644F4C0929D02D0929E029F
:106FD000E0929F02F092A002C0902001D090210187
:106FE000E0902201F090230120919D0230919E02B9
:106FF00040919F025091A002C701B6010E94C2DBDE
:1070000087FF08C0C0929D02D0929E02E0929F022C
:10701000F092A00201FF3CC0C0901801D09019016D
:10702000E0901A01F0901B012091A1023091A20280
:107030004091A3025091A402C701B6010E9443E40B
:10704000181644F4C092A102D092A202E092A302C8
:10705000F092A402C0902401D0902501E090260176
:10706000F09027012091A1023091A2024091A30249
:107070005091A402C701B6010E94C2DB87FF08C07D
:10708000C092A102D092A202E092A302F092A402C6
:1070900002FF3CC0C0901C01D0901D01E0901E0179
:1070A000F0901F012091A5023091A6024091A70205
:1070B0005091A802C701B6010E9443E4181644F497
:1070C000C092A502D092A602E092A702F092A80276
:1070D000C0902801D0902901E0902A01F0902B0166
:1070E0002091A5023091A6024091A7025091A802DA
:1070F000C701B6010E94C2DB87FF08C0C092A5028B
:10710000D092A602E092A702F092A80280913E0DD2
:1071100083FD61C020917E0130917F01409180010B
:10712000509181016091A9027091AA028091AB02F5
:107130009091AC020E94C2DB882309F44CC00E94EB
:107140008CA8182F882331F00E9410818FE896E0D8
:107150000E94B27B20917E0130917F01409180019D
:10716000509181016091A9027091AA028091AB02B5
:107170009091AC020E94DFE29F7720916C013091E8
:107180006D0140916E0150916F010E9427DC20E05B
:1071900030E046E154E40E9443E41816D4F40E941F
:1071A000108180E796E00E94B27B8091A9029091C5
:1071B000AA02A091AB02B091AC0280937E019093A1
:1071C0007F01A0938001B093810189EA92E052DDB2
:1071D00002C01111EACF2AE037ED43E25CE360918F
:1071E0000C0170910D0180910E0190910F010E9490
:1071F00027DC6B017C016091100170911101072E59
:10720000000C880B990B0E94C8DB9B01AC01C701E5
:10721000B6010E9427DC698B7A8B8B8B9C8B8091CB
:10722000B902882309F18090B5029090B602A0902F
:10723000B702B090B802C090A502D090A602E0902C
:10724000A702F090A80220E030E0A901C501B40136
:107250000E94C2DB8823F9F0A7019601C501B401A1
:107260000E9443E41816BCF020E030E0A901BE0102
:107270006F5E7F4F8DE992E00E94CDB780E1EDE92E
:10728000F2E0A2E7B1E001900D928A95E1F7A096B5
:10729000E2E10C94C4E220917201309173014091BB
:1072A00074015091750160919D0270919E028091D0
:1072B0009F029091A0020E94DFE24B015C012091AD
:1072C0007601309177014091780150917901609178
:1072D000A1027091A2028091A3029091A4020E9447
:1072E000DFE26D8B7E8B8F8B988F20917A013091AE
:1072F0007B0140917C0150917D01C701B6010E9444
:10730000DFE26D8F7E8F8F8F98A320917E01309169
:107310007F0140918001509181016091A90270919B
:10732000AA028091AB029091AC020E94DFE2698FC9
:107330007A8F8B8F9C8F20E030E0A901C501B401CA
:107340000E94C2DB81110CC020E030E0A9016D89F0
:107350007E898F89988D0E94C2DB882309F484CFAF
:10736000A5019401C501B4010E9427DC6B017C01D9
:107370002D893E894F89588DCA01B9010E9427DCA9
:107380009B01AC01C701B6010E94E0E26B017C01E8
:107390002D8D3E8D4F8D58A1CA01B9010E9427DC69
:1073A0009B01AC01C701B6010E94E0E26B017C01C8
:1073B000298D3A8D4B8D5C8DCA01B9010E9427DC65
:1073C0009B01AC01C701B6010E94E0E26B017C01A8
:1073D0000E947CE42B013C012CEC3CEB4CE85BE292
:1073E000C701B6010E94C2DB87FF06C0498C5A8CD8
:1073F0006B8C7C8CE89477F82DEB37E346E855E30B
:10740000C301B2010E94C2DB87FD38CF2DEC3CECFA
:107410004CE45EE3C301B2010E9427DC0E94C4E396
:107420001B01672B19F422242394312CB10190E025
:1074300080E00E94C6DB9B01AC0160E070E080E868
:107440009FE30E9457E36B017C01AC019B01C301E8
:10745000B2010E9427DC2B013C01A7019601C50166
:10746000B4010E9427DC4B015C01A70196016D89E4
:107470007E898F89988D0E9427DC6D8B7E8B8F8B08
:10748000988FA70196016D8D7E8D8F8D98A10E949A
:1074900027DC6D8F7E8F8F8F98A3A7019601698D52
:1074A0007A8D8B8D9C8D0E9427DC698F7A8F8B8FD4
:1074B0009C8F80E1E2E7F1E08E010F5F1F4FD80162
:1074C00001900D928A95E1F70E94F3C16B017C0156
:1074D00028ECC20ED11CE11CF11C81E0281A3108F5
:1074E00009F454C00E94F3C19B01AC012C193D0961
:1074F0004E095F0957FD4DC06B017C0128ECC20E9F
:10750000D11CE11CF11C80E00E947182A501940154
:1075100069817A818B819C810E94E0E269837A8310
:107520008B839C832D893E894F89588D6D817E8107
:107530008F8198850E94E0E26D837E838F83988798
:107540002D8D3E8D4F8D58A169857A858B859C85C3
:107550000E94E0E269877A878B879C87298D3A8D24
:107560004B8D5C8D6D857E858F8598890E94E0E2CC
:107570006D877E878F87988BA3019201BE016F5E16
:107580007F4FC8010E94CDB78111A7CFA3019201FF
:107590006ECE0E94FA25BACF809105049091060420
:1075A000A0910704B091080480930C0190930D0101
:1075B000A0930E01B0930F018091030490910404F5
:1075C0009093110180931001089580910C01909186
:1075D0000D01A0910E01B0910F01809305049093CD
:1075E0000604A0930704B0930804809110019091C1
:1075F0001101909304048093030484E690E0909337
:107600001101809310010895ACE0B0E0EAE0FBE3E3
:107610000C94AAE22B013C0129873A874B875C87AF
:1076200047015801D601CD90DD90ED90FC9020E00F
:1076300030E0A901C701B6010E94C2DB811171C00F
:107640008091680190916901A0916A01B0916B01EC
:1076500089839A83AB83BC8320E030E0A901C70112
:10766000B6010E94C2DB811106C0C12CD12C80E87A
:10767000E82E80E4F82ECD82DE82EF82F886A50126
:10768000940160917A0170917B0180917C019091CD
:107690007D010E94C2DB87FF0CC080927A0190922C
:1076A0007B01A0927C01B0927D01CE0105960E94E3
:1076B0004520409272015092730160927401709261
:1076C000750189859A85AB85BC85809376019093F9
:1076D0007701A0937801B0937901CE0101960E94C1
:1076E0004520A501940160917A0170917B01809100
:1076F0007C0190917D010E9443E4181664F480920D
:107700007A0190927B01A0927C01B0927D01CE0122
:1077100005960E9445200E9423292C96E0E10C94B6
:10772000C6E2D701C60194CFCF92DF92EF92FF92CB
:107730000F931F936B01FC01E080F18002811381A4
:10774000E2E7F1E0248135814681578160817181D2
:107750008281938159DF1F910F91FF90EF90DF900D
:10776000CF9008958F929F92AF92BF92CF92DF9267
:10777000EF92FF921F93CF93DF93CDB7DEB7609761
:107780000FB6F894DEBF0FBECDBF182F80E043DBED
:107790004B015C018092F7039092F803A092F903E9
:1077A000B092FA0381E037DB6B017C01C092FB03EE
:1077B000D092FC03E092FD03F092FE0382E02BDB0B
:1077C0006093FF037093000480930104909302047C
:1077D0001D861E861F86188A89829A82AB82BC8289
:1077E000CD82DE82EF82F88669877A878B879C87D5
:1077F00083E011DB6D877E878F87988BCE010196A2
:107800000E9445291E3FD9F480E1FE013196A2E78E
:10781000B1E001900D928A95E1F760960FB6F89469
:10782000DEBF0FBECDBFDF91CF911F91FF90EF90D4
:10783000DF90CF90BF90AF909F908F90089584E09D
:10784000189FF0011124DF01AE58BE4F81E090E097
:107850008C0F9D1FE80FF91F408151816281738158
:107860004D935D936D937C931397D7CF0C94F0B7A2
:10787000CF930E94F72BC82F809105138093041398
:10788000809303138093021384E6809301130E9474
:10789000A02C80ED93E09093880D8093870DC1110B
:1078A0000E94042C81E0809364040E9423298EEFBF
:1078B00059DFDCDFCF910895ACE0B0E0E2E6FCE315
:1078C0000C94B8E20E944BA80E94F72B9CE0E1E7E1
:1078D000F4E0DE01119601900D929A95E1F7811185
:1078E0000E94042CCE0101960E94BF262C96E2E055
:1078F0000C94D4E2B0E0A0E0E0E8FCE30C94AAE24F
:107900004090720150907301609074017090750105
:107910008090760190907701A0907801B0907901E5
:10792000C0907A01D0907B01E0907C01F0907D01C5
:107930000E94B72860912C0170912D01072E000C38
:10794000880B990B0E94C8DB2AE037ED43E25CE329
:107950000E9427DC60936C0170936D0180936E012F
:1079600090936F0104E111E0D0E0C0E0CE018353B9
:10797000964F0E943571F8016193719381939193B1
:107980008F01CE018F53964F0E943571F8016087A9
:107990007187828793872496CC30D10539F760E0D0
:1079A00087E194E00E941C740E94E9740E94FB2805
:1079B000A301920160917201709173018091740131
:1079C000909175010E94C2DB81111BC0A501940139
:1079D00060917601709177018091780190917901A1
:1079E0000E94C2DB81110DC020917A0130917B0190
:1079F00040917C0150917D01C701B6010E94C2DB1C
:107A000081115ADFCDB7DEB7E0E10C94C6E286E51E
:107A100096E00E94B27B86B160E576E082FB882723
:107A200080F90E94D71F86B16AE476E083FB88273D
:107A300080F90E94D71F86B164E476E08295817058
:107A40000E94D71F80B16CE376E082FB882780F923
:107A50000C94D71F8091DA06811103C08091DC0657
:107A600081110C94262C0895ACE0B0E0EAE3FDE32C
:107A70000C94B8E2AFE3BDE090E080E0FC01E95F88
:107A8000F44F45915591659174914D935D936D932C
:107A90007D93FC01E950F54F4591559165917491A5
:107AA00050964D935D936D937C935397FC01E951F0
:107AB000F54F459155916591749190964D935D93D5
:107AC0006D937C939397049680319105B9F680E28B
:107AD0009EE4A0E0B0E080934F0D9093500DA093F2
:107AE000510DB093520D80E090E0AAEFB3E4809383
:107AF000730D9093740DA093750DB093760D8093D4
:107B0000770D9093780DA093790DB0937A0D8093B3
:107B10007B0D90937C0DA0937D0DB0937E0D109204
:107B20007F0D1092800D1092810D1092820D109297
:107B3000830D1092840D1092850D1092860D8AE0AF
:107B400097EDA3EABDE38093610790936207A0934A
:107B50006307B093640780E090E0A0E2B1E4809313
:107B6000170490931804A0931904B0931A040E9468
:107B7000D2738CE0E2E8F1E0DE01119601900D9203
:107B80008A95E1F789819A81AB81BC818093F31258
:107B90009093F412A093F512B093F6128D819E810A
:107BA000AF81B8858093F7129093F812A093F912E1
:107BB000B093FA1289859A85AB85BC858093FB12B8
:107BC0009093FC12A093FD12B093FE128EEB90E006
:107BD0009093C3028093C2021092C5021092C40215
:107BE00086EE90E09093C7028093C6021092C9027D
:107BF0001092C8028FE892ECADE8B1E480938B124A
:107C000090938C12A0938D12B0938E128CE998EF02
:107C1000A5E4BEE380938F1290939012A0939112EB
:107C2000B093921281E49CEBABECB3E4809393129B
:107C300090939412A0939512B09396121092DA0634
:107C40001092D90607DF56DE0E94108184EC9AE07C
:107C50000E94B27B2C96E2E00C94D4E2A4E0B0E067
:107C6000E4E3FEE30C94B1E29091DC06981709F48A
:107C70004FC0B82E882349F180E090E0A0E2B1E443
:107C800089839A83AB83BC83C090FB12D090FC1293
:107C9000E090FD12F090FE1220E030E0A901C70153
:107CA000B6010E94C2DB87FF0CC0A701960160E00D
:107CB00070E080E291E40E94DFE269837A838B8343
:107CC0009C83CE0101960E946BB860917201709105
:107CD000730180917401909175012091760130912A
:107CE0007701409178015091790119821A821B82A3
:107CF0001C82E0907A01F0907B0100917C01109150
:107D00007D01FE0131966F017FDCB092DC06A2DEC0
:107D100080E02496E9E00C94CDE24F925F926F925E
:107D20007F928F929F92AF92BF92DF92EF92FF92DB
:107D30000F931F93CF93DF93D82EC82FD0E0FE016F
:107D4000E359F34DF49082E0D81609F4E3C06F2DA7
:107D5000FF0C770B880B990B0E94C8DB2B013C01B1
:107D6000CE01880F991F880F991F8750994F0E9445
:107D700035714B015C01A3019201C501B4010E9460
:107D800027DC4B015C017E01EE0CFF1CEE0CFF1C9E
:107D9000C7018351994F0E9435719B01AC01C3010A
:107DA000B2010E9427DC20E030E040EC5FE30E945B
:107DB00027DCAB01BC0100E010E098018D2D0E9492
:107DC000B1BB20E030E0A901C501B4010E94C2DBD3
:107DD000882309F440C082E000E010E020E830E4AD
:107DE000D81619F000E010E09801B501A401705810
:107DF0008D2D0E94B1BBA5019401C501B4010E9463
:107E0000E0E24B015C0182E000E010E020E030E4C1
:107E1000D816E1F0FE01E252F94F6491611107C0FA
:107E20000E9410818CEB96E00E94B27B6AE070E0C9
:107E300090E080E00E94C6DB9B01AC0161E070E055
:107E400088E492E40E9457E38B019C01B501A401F0
:107E50008D2D0E94B1BB81E090E00D2C01C0880FF8
:107E60000A94EAF790914D07982B90934D079091C3
:107E70000904892B80930904C7018F51994F0E94EF
:107E80003571F701EE58FE4F6083718382839383CF
:107E900082E0D8121AC02091FB123091FC1240915E
:107EA000FD125091FE1260917A0170917B018091D8
:107EB0007C0190917D010E94DFE260937A017093D2
:107EC0007B0180937C0190937D01D0DCF701E35628
:107ED000FD4FD701AE58BE4F8D919D910D90BC9135
:107EE000A02D80839183A283B38382E0D81202C045
:107EF00080E0B4DEDF91CF911F910F91FF90EF9062
:107F0000DF90BF90AF909F908F907F906F905F9029
:107F10004F90089581E0A2DE8111ECCF81E097E0DF
:107F20000E94357120E030E0A9010E94C2DB882365
:107F300009F40DCF6F2DFF0C770B880B990B0E9466
:107F4000C8DB2B013C0181E097E00E9435714B01B9
:107F50005C0120E030E040EA50E40E9443E487FF07
:107F60000ACF812C912C90EAA92E90E4B92E03CF50
:107F700080914C07882319F010924C07089540E037
:107F800070E060E08CE196E00E9483811F920F9286
:107F90000FB60F9211240BB60F922F933F934F936E
:107FA0005F936F937F938F939F93AF93BF93EF9361
:107FB000FF930E94262CFF91EF91BF91AF919F916B
:107FC0008F917F916F915F914F913F912F910F9082
:107FD0000BBE0F900FBE0F901F9018950F931F931D
:107FE00080915D07813019F50E94F3C10091EE0385
:107FF0001091EF032091F0033091F103601B710B9E
:10800000820B930B28EE33E040E050E00E94F0E159
:108010006091EA037091EB038091EC039091ED0382
:10802000620F731F841F951F1F910F910895609118
:10803000F2037091F3038091F4039091F503D6CF8E
:1080400010925D071092EE031092EF031092F0036E
:108050001092F1031092F2031092F3031092F403C2
:108060001092F5031092EA031092EB031092EC03C6
:108070001092ED03089580915D078130E1F0823028
:10808000C1F4ACDF6093EA037093EB038093EC03DD
:108090009093ED0381E080935D070E94F3C16093AC
:1080A000EE037093EF038093F0039093F10381E06C
:1080B0000895C6DFEFCF80E008950E94B9B80E940E
:1080C0008375882351F08091821482FD06C087EE6B
:1080D00091E09093DE068093DD06CDCF80915D0721
:1080E000813079F482E080935D070E94F3C1609350
:1080F000F2037093F3038093F4039093F50381E00C
:10810000089580E0089580915D078150823070F479
:1081100010925D070E94F3C16093F2037093F30322
:108120008093F4039093F50381E0089580E008952F
:108130009C0197FF26C0EE27FF27E81BF90B2D397E
:108140008FEF38070CF05DC08DE280939802CF016D
:1081500064E670E00E9458E2CB012AE030E0B90109
:108160000E9458E2805D80939902CF01B9010E947C
:1081700058E2CB01B9010E9458E2805D80939A02D7
:108180002AC0283E83E03807B4F1C90168EE73E0E5
:108190000E9458E2CB01EAE0F0E0BF010E9458E201
:1081A000805D80939802C90164E670E00E9458E205
:1081B000CB01BF010E9458E2805D80939902C90102
:1081C000BF010E9458E2CB01BF010E9458E2805DCE
:1081D00080939A02F901CF016AE070E00E9458E2B0
:1081E000805D80939B0288E992E008958DE237FDDF
:1081F000C5CF80E2C3CFF90180E2243631050CF00F
:10820000A4CF80E28093980280939902EA30F1052E
:108210006CF38DE237FF80E280939902CF016AE030
:1082200070E00E9458E2605D60939A02D4CF9C0196
:1082300097FD2DC080E2243631055CF0C90164E66B
:1082400070E00E9458E2CB016AE070E00E9458E2C0
:10825000805D8093990280E22A3031055CF0EAE08B
:10826000F0E0C901BF010E9458E2CB01BF010E94AA
:1082700058E2805D80939A02C9016AE070E00E9432
:1082800058E2805D80939B0289E992E008953195E0
:10829000219531098DE2DDCFCF92DF92EF92FF92EF
:1082A000FC01C080D180E280F38020E030E0A901B1
:1082B000C701B6010E94C2DB87FD26C06DEB77E3E4
:1082C00086E095E3A70196010E94E0E26B017C0144
:1082D00020E030E0A9010E94C2DB20E030E040E075
:1082E0005FE387FF04C020E030E040E05FEBC701C0
:1082F000B6010E94E0E20E94BFE3CB0198DFFF904D
:10830000EF90DF90CF9008956DEB77E386E095EBEB
:10831000D9CFA4E0B0E0EFE8F1E40C94B8E20E9419
:10832000C8DB69837A838B839C83CE010196B4DF9B
:108330002496E2E00C94D4E2FC0160817181828198
:1083400093810E94BFE3CB0172CFA4E0B0E0EBEADF
:10835000F1E40C94B8E20E94C8DB69837A838B83D2
:108360009C83CE010196E8DF2496E2E00C94D4E2EF
:108370000F931F930E94F3C10091D5061091D6066A
:108380002091D7063091D806011511052105310538
:10839000D9F5209118132223A1F1E0911613215051
:1083A0002093181321E02E0F2093161330911913E8
:1083B000231302C01092161324E0E29FF00111244F
:1083C000E65EFC4E00811181228133810093D1064B
:1083D0001093D2062093D3063093D406600F711FFA
:1083E000811D911D6093D5067093D6068093D706A4
:1083F0009093D8068091D3069091D406892B09F0EA
:10840000149A1F910F910895601B710B820B930BAF
:1084100097FDF7CF14981092D5061092D6061092B9
:10842000D7061092D806EDCF0F931F93CF93DF930B
:108430008C01EB019091181320911913921304C031
:1084400097DF0E94FA25F6CF8091171334E0839FBF
:10845000F0011124E65EFC4E11830083D383C283B6
:108460009F5F909318138F5F281739F0809317132D
:10847000DF91CF911F910F91089510921713F8CFAC
:10848000882351F063E972E084E690E0CDDF6AEB87
:1084900072E084E690E0C8CF68EB71E084E190E0A0
:1084A000FACFE2DA81E0ECCF8F929F92AF92BF9247
:1084B000EF92FF920F931F93CF93DF93EC018B0109
:1084C000E42EF22E80912A1390912B138C179D0786
:1084D000C9F125E5CE3AD20709F03FC08159954749
:1084E00071F40E94F3C16E517B4F8F4F9F4F609389
:1084F000DA037093DB038093DC039093DD03D09366
:108500002B13C0932A1330E020E000933F07109311
:1085100040072093410730934207E0923A07F092D8
:108520003B07C159D54721F4109294021092D90308
:1085300082E08093670181E080933C071092930270
:108540001092E503DF91CF911F910F91FF90EF9073
:10855000BF90AF909F908F90089525E7C139D207C3
:1085600071F68E5A9545D9F40E94F3C18090DA03D2
:108570009090DB03A090DC03B090DD0368197909CB
:108580008A099B0997FF0BC080914D078770873040
:1085900031F40E94F520C7E5DEE48111B0CFC1E9D6
:1085A000D5E7ADCF20E040E070E060E084EE90E2FF
:1085B0007BCF0E948CA8882339F020E040E070E057
:1085C00060E089E79DE470CFEDCF21E02093940235
:1085D000FC0180819181A281B381809308019093F5
:1085E0000901A0930A01B0930B0120E040E070E084
:1085F00060E08091290790912A0756CFA4E0B0E06F
:10860000E4E0F3E40C94B8E28DEC9CECACECBCE35D
:1086100089839A83AB83BC83CE010196D6DF2496EF
:10862000E2E00C94D4E2A4E0B0E0E9E1F3E40C94DD
:10863000B8E28DEC9CECACECBDE389839A83AB8310
:10864000BC83CE010196C1DF2496E2E00C94D4E213
:10865000A4E0B0E0EEE2F3E40C94B8E280E090E055
:10866000A0E8BFE389839A83AB83BC83CE010196E4
:10867000ACDF2496E2E00C94D4E2A4E0B0E0E3E4C2
:10868000F3E40C94B8E280E090E0A0E2B1E48983E6
:108690009A83AB83BC83CE01019697DF2496E2E0F8
:1086A0000C94D4E281E08093940280914D0787700E
:1086B000873051F010924D071092090486EB95E037
:1086C0009093DE068093DD068091B9028093E703E4
:1086D00080E00E94907320E040E070E060E082E77C
:1086E00093E4E2CE80916701882331F041E062EAB1
:1086F00073E082E00E945EBC80910904877087303D
:1087000071F41092E60320E040E070E060E089EF51
:108710009DE4CADE81E08093E5030C944D2008952A
:1087200020E040E070E060E081E995E7BDCE109286
:108730007D070E945625F4CFCF93DF93C091200789
:10874000C7FD1FC084E0C802E0011124FE01EE5302
:10875000FD4F80819181181619063CF4863F9105E2
:1087600014F085EF90E00E9434C2CE53DD4F8A8131
:108770009B818F3F910519F010F08FEF90E080936F
:108780007D07CEDFDF91CF910895B0E0A0E0EBEC64
:10879000F3E40C94B2E2CDB6DEB6E0E5F7E0DF013B
:1087A0000D900020E9F7CD01885497402DB73EB7D2
:1087B000281B390B0FB6F8943EBF0FBE2DBF0DB767
:1087C0001EB70F5F1F4FFF93EF9389E195E09F93D3
:1087D0008F931F930F930E945BDB780134E0E30ECD
:1087E000F11C0F900F900F900F900F900F90D701EA
:1087F0008D917D01882349F0082E000C990B0E9471
:10880000C1E4F70131978083F2CF64E175E0C801DC
:108810000E94F4DA4FE350E0B8018FED96E00E9439
:1088200019E50FB6F894DEBE0FBECDBE79DF0E940B
:10883000B9B8E8E00C94CEE28093200720E040E055
:1088400070E060E087E19EE42FCECF93DF93C0918C
:10885000D903CC23B1F0C150C093D90389E0C89F9C
:10886000E0011124CD55DC4F6A817B812F814E813F
:108870008881998119DE888580939402DF91CF9158
:1088800008954EDFFBCFA4E0B0E0E9E4F4E40C94FB
:10889000ACE20E9472BDF0903A0785E0782E7F0C22
:1088A00085E0E82EEF1884E0D82EDF18AA24AA94D9
:1088B000B12C83E0C82ECF1882E0982E9F1881E05B
:1088C000882E8F186F2C6194F11027C080913D077E
:1088D0008823A1F080916701882359F081E090916D
:1088E0003D07911180E024E047E156E0662D0E94AB
:1088F000BEBC80917D078093200768C080912407CB
:1089000010922407882331F3A0DF80913C0788234D
:1089100009F32496EEE00C94C8E221E0F21276C04E
:1089200080913D07813009F458C080916701882308
:1089300001F311E080913D07813009F010E0609172
:10894000100170911101072E000C880B990B0E94E9
:10895000C8DB69837A838B839C83CE010196ECDC30
:1089600000E09C0141E156E0682D812F0E94396FA3
:1089700080917D078093200723E0F2129CC0109223
:10898000490780913D07833009F482C080916701D7
:108990008823E1F011E080913D07833009F010E079
:1089A0008091200724E6829FC001112481589F4FA7
:1089B000B5010E9458E2862F0E940A1B00E09C012C
:1089C00040E056E06C2D812F0E94396FF394F71030
:1089D0007BCF86E080933B079CCF80912407109249
:1089E0002407882309F4A1CF10E000E027EE33E04C
:1089F0004AE050E060E171E081E196E00E9437BE1C
:108A000080913C07882309F490CF83CF82E0F8124D
:108A1000AFCF80913D07823011F1809167018823AB
:108A200009F467CF11E080913D07823009F010E032
:108A30006091881270918912072E000C880B990B97
:108A40000E94C8DB69837A838B839C83CE01019665
:108A500073DC00E09C014AE056E0692D86CF8091EE
:108A60002407109224078823C1F20E9466BD0DEEF0
:108A70001FE125EF30E050E040E068E872E18AE075
:108A800096E00E9437BE80913C07882331F241CFA7
:108A90008091240710922407882309F477CF0E943D
:108AA00066BD80E096E00E94ACC080913C078823C0
:108AB00009F46CCF2ECF84E0F8123DC080913D07C1
:108AC000843011F180916701882309F47FCF11E090
:108AD00080913D07843009F010E060912C01709185
:108AE0002D01072E000C880B990B0E94C8DB6983AF
:108AF0007A838B839C83CE0101961EDC00E09C016F
:108B00004BEF55E06D2D5FCF809124071092240725
:108B10008823C1F20BE21BE127EE33E04AE050E08C
:108B20006CE271E08BEF95E00E9437BE80913C07CC
:108B3000882341F2EECE25E0F21248CF80913D0726
:108B4000853091F080916701882309F43FCF81E05F
:108B500090913D07953009F080E023E04CEE55E020
:108B60006E2D0E94BEBC32CF809124071092240744
:108B7000882341F387E59EE40E94C8BD80913C07AD
:108B8000882301F3C6CEA7E0B0E0E9ECF5E40C944D
:108B9000A8E2A0908812B09089120E9472BD7090D5
:108BA0003A077E8225E0270D2D8388248A94912C14
:108BB00082E087198F8381E0682E6718472C4194E3
:108BC0005CE9E52E53E4F52E6CECC62E65E0D62E5E
:108BD00085E0582E5718711015C080913D078823E5
:108BE00009F4DBC080916701882309F433C181E077
:108BF00090913D07911180E024E047EE55E0642D0F
:108C00000E94BEBC80918812909189129093210796
:108C10008093200781E0781229C080913D07813040
:108C200009F4CCC080916701882309F44DC011E09C
:108C300080913D07813009F010E06091200770912C
:108C40002107072E000C880B990B0E94C8DB698353
:108C50007A838B839C83CE0101966EDB00E09C01BE
:108C600040EE55E0662D812F0E94396F80917D077F
:108C70008093200792E0791227C0109249078091D3
:108C80003D07823009F4B5C0809167018823E1F087
:108C900011E080913D07823009F010E080912007BB
:108CA00024E6829FC001112481589F4FB4010E9485
:108CB00058E2862F0E940A1B00E09C0146ED55E019
:108CC0006F81812F0E94396F10E000E033E0332E76
:108CD000272C8E81281A00932007731027C0F801D3
:108CE000EE0FFF1FE154FA4F8591949190934B073B
:108CF00080934A0780913D07871509F48DC08091C4
:108D00006701882399F0FF92EF92DF92CF922F9222
:108D100081E090913D07931180E08F930E94BF20E6
:108D20000F900F900F900F900F900F90832D0F5F6B
:108D30001F4F94E0392E843071F6A114B10409F468
:108D400087C095E0791221C080913D07853009F4F4
:108D500071C0809167018823C1F087E993E49F93F4
:108D60008F9383EC95E09F938F935F9281E0909136
:108D70003D07953009F080E08F930E94BF200F904F
:108D80000F900F900F900F900F9086E073942D81AD
:108D9000271121CF80933B070DC0809124071092AB
:108DA0002407882309F41ECF50DD80913C078823D7
:108DB00009F418CF2796E2E10C94C4E280912407CD
:108DC00010922407882309F42DCF0E9466BD0FEC72
:108DD00010E225EF30E050E040E060E277E080EE26
:108DE00095E00E9437BE80913C07882309F41ACF92
:108DF000E1CF8091240710922407882309F444CFFF
:108E00000E9466BD86ED95E00E94ACC080913C0753
:108E1000882309F439CFCECF8091240710922407FC
:108E2000882309F46CCF88DC80913C07882309F4FF
:108E300066CFC0CF8091240710922407882309F4BD
:108E400088CF75DC80913C07882309F482CFB2CFAC
:108E500085E09CCF80918812909189129093210790
:108E60008093200703CFB0E0A0E0E9E3F7E40C949F
:108E7000AFE20E9472BDC0913A0785E0E82EEC0E89
:108E80009BE9C92E95E0D92ED4E0DC1B13E01C1B16
:108E900026EBA22E25E0B22E02E00C1B81E0F82E7C
:108EA000FC1A9C2E9194C1112AC080913D07882301
:108EB000B1F080916701882359F081E090913D07DE
:108EC000911180E024E04AEB55E0692D0E94BEBC80
:108ED000CF5FEC12E8CF85E080933B070BC0809119
:108EE000240710922407882321F3AFDC80913C07EC
:108EF0008823F9F2CDB7DEB7EBE00C94CBE2C130BA
:108F000011F580913D07813079F0809167018823C8
:108F1000F9F281E090913D07913009F080E023E083
:108F20004FE25CE26F2DD2CF80912407109224078C
:108F3000882359F380E198E40E94C8BD80913C07E2
:108F4000882319F3D7CFC23009F053C090913D0761
:108F5000923071F080916701882309F4B9CF81E0E4
:108F6000923009F080E020E24CEA55E0602FAECF6D
:108F70008091240710922407882361F3B092DE06C3
:108F8000A092DD0680913C07882321F3B3CF809126
:108F90003D07833081F080916701882309F498CFE1
:108FA00081E090913D07933009F080E023E04FE9A4
:108FB00055E0612F8BCF80912407109224078823DE
:108FC00051F38FEA9CE50E94C8BD80913C0788233D
:108FD00011F390CF8091240710922407882391F0F9
:108FE000D092DE06C092DD0680913C07882351F0C6
:108FF00081CFC33061F2C43009F06ACF90913D0750
:10900000943041F380916701882309F461CF81E0B6
:10901000943009F080E020E24AE855E06D2F56CF09
:10902000B0E0A0E0E6E1F8E40C94B3E20E9472BD87
:10903000C0913A0785E0E82EEC0ED4E0DC1B13E08B
:109040001C1B02E00C1B81E0F82EFC1ADC2ED194D4
:10905000C1112AC080913D078823B1F0809167013A
:10906000882359F081E090913D07911180E024E040
:1090700043E855E06D2D0E94BEBCCF5FEC12E8CFF7
:1090800085E080933B070BC0809124071092240752
:10909000882321F3DADB80913C078823F9F2CDB7EE
:1090A000DEB7E7E00C94CFE2C13011F580913D07C7
:1090B000813079F0809167018823F9F281E0909105
:1090C0003D07913009F080E023E045E55CE26F2D3B
:1090D000D2CF8091240710922407882359F38FED73
:1090E00090E20E94C8BD80913C07882319F3D7CF36
:1090F000C23009F055C080913D07823081F08091E7
:109100006701882309F4B9CF81E090913D0792303F
:1091100009F080E023E04EE45CE2602FACCF809168
:10912000240710922407882351F38AED90E20E94CD
:10913000C8BD80913C07882311F3B1CF80913D07D2
:10914000833081F080916701882309F496CF81E014
:1091500090913D07933009F080E023E047E45CE222
:10916000612F89CF8091240710922407882351F31F
:1091700085ED90E20E94C8BD80913C07882311F3E1
:109180008ECF8091240710922407882391F089EDD7
:1091900092E40E94C8BD80913C07882351F07FCFA4
:1091A000C33061F2C43009F068CF80913D0784304C
:1091B00041F380916701882309F45FCF81E09091AA
:1091C0003D07943009F080E023E049E35CE26D2F35
:1091D00052CFACE0B0E0EFEEF8E40C94A9E29C874B
:1091E0008B87362E8091240710922407882339F02C
:1091F000109294022ADB2C96E1E10C94C5E2609176
:109200003F07709140078091410790914207611597
:1092100071058105910509F45CC02091120122239A
:1092200009F4AEC0209113012111AAC021E0321629
:1092300009F484C0E2E03E1609F491C0C090140124
:10924000D0901501E0901601F09017014090200198
:109250005090210160902201709023010E94C8DB90
:10926000209108013091090140910A0150910B01B0
:109270000E9427DC6F83788789879A87F4E03F9E76
:1092800080011124C8018E589E4F9E838D83FC015E
:1092900020813181428153816F81788589859A85CA
:1092A0000E94E0E24B015C01A3019201C701B601FB
:1092B0000E94C2DB811173C0F801EE58FE4F80821C
:1092C0009182A282B382832D0E94E26781E0809323
:1092D000670110923F0710924007109241071092C9
:1092E000420780916701882309F485CF24E0329EEC
:1092F000F0011124EE58FE4FC080D180E280F3804F
:10930000C982DA82EB82FC822DEC3CEC4CEC5DE312
:10931000609108017091090180910A0190910B01FF
:109320000E9443E487FD65C0CE0101960E94581952
:10933000BC018B859C850E94D26E5DCFC0901801C8
:10934000D0901901E0901A01F0901B014090240187
:109350005090250160902601709027017FCFC0902A
:109360001C01D0901D01E0901E01F0901F01409063
:1093700028015090290160902A0170902B016ECF36
:10938000412C20E5522E23EC622E27E4722EC12CB4
:1093900030E5D32E33ECE32E37ECF32E5FCF20E015
:1093A00030E0A9016F81788589859A850E94C2DBAA
:1093B00087FF0FC0A7019601C501B4010E94C2DB5F
:1093C00087FF7ACFED81FE81C082D182E282F38273
:1093D0007ACFA3019201C501B4010E9443E418169B
:1093E0000CF06ACFED81FE814082518262827382ED
:1093F0006ACF20E030E44CE156E4C701B6010E9498
:1094000027DC4B015C0120E030E0A901C701B60177
:109410000E94C2DB20E030E040EA50E487FF04C055
:1094200020E030E040EA50ECC501B4010E94E0E2E7
:109430002DEC3CEC4CEC5DE30E9427DC0E94BFE38A
:109440006B017C01F7FC64C020EA36E841E050E0A3
:109450000E946BE2CA01B9012AE030E040E050E02E
:109460000E946BE2605D60939502C701B60120E146
:1094700037E240E050E00E946BE28AE0882E912CB7
:10948000A12CB12CCA01B901A50194010E946BE283
:10949000605D60939602C701B60128EE33E040E0BC
:1094A00050E00E946BE2CA01B901A50194010E943B
:1094B0006BE2605D609397028EE280939802C70131
:1094C000B60124E630E040E050E00E946BE2CA01C1
:1094D000B901A50194010E946BE2605D609399025D
:1094E000C701B601A50194010E946BE26B017C01EA
:1094F000CA01B901A50194010E946BE2605D60930D
:109500009A0280E3C80EC0929B0285E992E010CFD8
:10951000F094E094D094C094C11CD11CE11CF11CC7
:109520006DE2A1CF62E087E49CE253CE61E08EE47D
:109530009CE24FCE60E085E59CE24BCEA4E0B0E03B
:10954000E4EAFAE40C94B8E280912407109224072C
:10955000882339F01092940278D92496E2E00C9492
:10956000D4E260913F07709140078091410790914C
:109570004207611571058105910561F10E94C8DB03
:10958000209108013091090140910A0150910B018D
:109590000E9427DC20917E0130917F014091800163
:1095A000509181010E94E0E260937E0170937F01FF
:1095B000809380019093810183E00E94E26781E0C3
:1095C0008093670110923F07109240071092410765
:1095D0001092420780916701882309F4BECF209141
:1095E0002507309126074091270750912807609161
:1095F0007E0170917F0180918001909181010E9494
:10960000DFE269837A838B839C83CE0101960E947B
:109610005819BC0189E39CE20E94D26E9ECFB0E053
:10962000A0E0E5E1FBE40C94B3E20E94F520082FF2
:109630000E9472BDC0913A07FC2E85E0E82EEC0E28
:1096400011E01C1BDC2ED194C11114C080913D0788
:109650008823F9F080916701882309F473C081E0C1
:1096600090913D07911180E024E04CE753E06D2D8F
:109670000E94BEBC011139C0D2E0C130B9F5809161
:109680003D078130B1F080916701811121C0D2E0A6
:1096900043C080912407109224078823D9F2D5D89B
:1096A00080913C078823B1F2CDB7DEB7E7E00C9498
:1096B000CFE28091240710922407882321F38EEBB8
:1096C0009BE40E94C8BD80913C078823E1F2ECCF67
:1096D00081E090913D07913009F080E023E043E77D
:1096E00053E0612F0E94BEBCD2CFD1E0DC1314C086
:1096F00080913D078D17B9F080916701882361F053
:109700006C2F6F1981E090913D079C1380E023E05E
:1097100047E653E00E94BEBCCF5FCE1195CFDF5F1E
:10972000D0933B07C1CF8091240710922407882350
:1097300019F380EE90E50E94C8BD80913C07882314
:10974000D9F2B2CFD1E0002309F4A1CFE5CF80E078
:1097500090E0A0E8B0E480937A0190937B01A0931D
:109760007C01B0937D0187E192E00E9445208091C9
:10977000E7030E9490731092940267C8B0E0A0E0E3
:10978000E4ECFBE40C94B1E20E9472BDC0913A0794
:1097900085E0C82ECC0ED4E0DC1B13E01C1B82E05D
:1097A000F82EFC1A81E0E82EEC1ABC2EB194C111FF
:1097B0002AC080913D078823B1F0809167018823FA
:1097C00059F081E090913D07911180E024E045E55A
:1097D00053E06B2D0E94BEBCCF5FCC12E8CF85E07A
:1097E00080933B070BC080912407109224078823A5
:1097F00021F32BD880913C078823F9F2CDB7DEB74F
:10980000E9E00C94CDE2C13089F580913D078130CB
:10981000C1F0809167018823F9F2DD24D39480910F
:109820003D07813009F0D12C83E59DE00E943E1C6C
:1098300000E09C014AE453E06E2D8D2D0E94396FAB
:10984000CBCF8091240710922407882311F30E9424
:1098500066BD42E259E263E57DE08AE493E00E945E
:10986000D7BD80913C078823A1F2C8CFC23009F050
:1098700073C080913D078230B1F0809167018823E9
:1098800009F4AACFDD24D39480913D07823009F0FA
:10989000D12C87E59DE00E943E1C00E09C014FE337
:1098A00053E06F2DCACF809124071092240788239C
:1098B00021F30E9466BD41E259E267E57DE08FE356
:1098C00093E00E94D7BD80913C078823B1F296CFE8
:1098D00080913D078330B1F080916701882309F4BE
:1098E0007BCFDD24D39480913D07833009F0D12CC8
:1098F0008BE59DE00E943E1C00E09C0144E353E0A8
:10990000612F9BCF8091240710922407882321F395
:109910000E9466BD40E259E26BE57DE084E393E09E
:109920000E94D7BD80913C078823B1F267CF809118
:109930002407109224078823C9F00E9466BD4FE1D6
:1099400059E26FE57DE089E293E00E94D7BD809106
:109950003C07882359F052CFC33009F4B9CFC43043
:1099600009F03ACF80913D07843009F38091670177
:10997000882309F431CFDD24D39480913D078430CE
:1099800009F0D12C8FE59DE00E943E1C00E09C0177
:1099900049E253E06D2F51CFA3E0B0E0E2EDFCE4EB
:1099A0000C94A8E24C013B015A011901280181E005
:1099B0008093940240913F07509140076091410786
:1099C00070914207411551056105710571F014163A
:1099D00015060CF080E08093E50310923F0710928B
:1099E000400710924107109242071091E5038091C1
:1099F00024078B8310922407811105C08091670191
:109A0000882309F46FC0C2010E948A68082F80E091
:109A1000C114D10419F0C6010E948A681A82198201
:109A2000E114F104B1F4402F50E0282F30E0CA01D6
:109A3000820F931F46976CF485E190E0841B950B91
:109A4000821B930B97FD0196959587958A8381E0FC
:109A5000898301E026E232E6A201BE016F5F7F4FFB
:109A6000CE0102960E94E269E114F10491F08A812C
:109A7000882321F01A8289818F5F898300E029E29F
:109A800032E6A701BE016F5F7F4FCE0102960E94B2
:109A9000E269C114D10459F000E026E232E6A601E1
:109AA000BE016F5F7F4FCE0102960E94E26941E0E6
:109AB0004127B30181E00E94CEC4C4010E948A689C
:109AC000412FB40194E1981B892F0E94CEC4EB81F1
:109AD000EE2341F0111101C05101A114B10431F084
:109AE000F50109952396E2E10C94C4E20E94254415
:109AF000F9CFCF92DF92EF92FF920F931F9384E6FC
:109B0000C82E85E0D82EF12CE12C06E615E030E0D9
:109B100020E042ED52E466E775E08BE795E03CDF3C
:109B20001F910F91FF90EF90DF90CF900895B0E0DC
:109B3000A0E0EDE9FDE40C94B0E2ADB6BEB68091D4
:109B4000F90F60E577E0882311F069EF7FE0FB0112
:109B500001900020E9F7CF01861B970B01962DB7E6
:109B60003EB7281B390B0FB6F8943EBF0FBE2DBF72
:109B70008DB79EB701967C0180E2EDB7FEB7818379
:109B8000C70101960E9404E580E2C82E85E0D82E28
:109B900002E215E030E020E045EC53E46EE275E0CF
:109BA00085E395E0F9DE0FB6F894BEBE0FBEADBEFC
:109BB000EAE00C94CCE2CF92DF92EF92FF920F9307
:109BC0001F938EE7C82E84E0D82EF12CE12C01EFF4
:109BD00014E030E020E04AEF57E560E874E085E803
:109BE00094E0DADE1F910F91FF90EF90DF90CF901D
:109BF0000895CF92DF92EF92FF920F931F938AE81E
:109C0000C82E83E0D82EF12CE12C0CE813E027EAD3
:109C10003BE44DE450E268E973E08DE993E0BCDE9B
:109C20001F910F91FF90EF90DF90CF900895B0E0DB
:109C3000A0E0EDE1FEE40C94B0E2ADB6BEB683E385
:109C400092E00E948A6890E001962DB73EB7281BEB
:109C5000390B0FB6F8943EBF0FBE2DBF8DB79EB720
:109C600001967C0163E372E00E940ADB8091200789
:109C700000E012E0813031F00BEE11E0823011F0A3
:109C800003E112E084E2C82E82E0D82E20E933E41A
:109C900041E755E566E272E08DE292E07DDE0FB6C7
:109CA000F894BEBE0FBEADBEEAE00C94CCE28F923B
:109CB0009F92AF92BF92CF92DF92EF92FF920F935B
:109CC0008091240710922407882371F01092940247
:109CD0000E9425440F91FF90EF90DF90CF90BF90AE
:109CE000AF909F908F90089581E08093940280912F
:109CF0003F0790914007A0914107B091420700971C
:109D0000A105B10509F44AC05C01AA0CBB1CAA0C50
:109D1000BB1C10923F07109240071092410710920F
:109D20004207B5010B2C000C880B990B0E94C8DB75
:109D300020918607309187074091880750918907C5
:109D40000E9427DC2091FB123091FC124091FD1201
:109D50005091FE120E94E0E26B017C0120E030E0B5
:109D600040EA51EC0E9443E487FD18C020E030E057
:109D700040EA51E4C701B6010E94C2DB181674F034
:109D8000C5010E94DCB8C092FB12D092FC12E09296
:109D9000FD12F092FE1282E08093670180916701CC
:109DA000882309F497CFC090FB12D090FC12E0906A
:109DB000FD12F090FE1220E030E44CE156E4C701C1
:109DC000B6010E9427DC4B015C0120E030E0A901D4
:109DD000C701B6010E94C2DB20E030E040EA50E457
:109DE00087FF04C020E030E040EA50ECC501B40138
:109DF0000E94E0E22DEC3CEC4CEC5DE30E9427DCA1
:109E00000E94BFE36B017C018BE2F7FE09C0F09476
:109E1000E094D094C094C11CD11CE11CF11C8DE2D3
:109E200080939502C701B60120E137E240E050E09F
:109E30000E946BE26AE0862E912CA12CB12CCA0103
:109E4000B901A50194010E946BE2605D60939602E6
:109E5000C701B60128EE33E040E050E00E946BE21B
:109E6000CA01B901A50194010E946BE2605D609393
:109E700097028EE280939802C701B60124E630E093
:109E800040E050E00E946BE2CA01B901A5019401D3
:109E90000E946BE2605D60939902C701B601A50163
:109EA00094010E946BE26B01CA01B901A501940102
:109EB0000E946BE2605D60939A0260E36C0D6093B8
:109EC0009B0265E972E084EF92E00E94D26EC0903E
:109ED000FB12D090FC12E090FD12F090FE128090E8
:109EE000E1039090E203A090E303B090E403A501A6
:109EF0009401C701B6010E94C2DB8823E9F020E08B
:109F000030E0A901C701B6010E94C2DB882309F431
:109F100079C0A5019401C701B6010E94C2DB87FD8B
:109F200073C081E08093E003C092E103D092E2032A
:109F3000E092E303F092E403D090E0038091641395
:109F4000813188F480916613833068F044E04D19C4
:109F50005CEDE52E52E0F52E0CE022E062E480E3B9
:109F600093E10E940AC680916413853180F4809148
:109F70006613843160F049EDE42E42E0F42E01E0F6
:109F800023E044E16CE380E393E10E940AC6809100
:109F900064138F3308F09ECE809166138F3208F4DD
:109FA00099CE40E34D198FEBE82E82E0F82E0DE0BC
:109FB00022E06AE580E393E10E940AC641E34D197D
:109FC00095EAE92E92E0F92E22E065E080E393E144
:109FD0000E940AC625E7E22E22E0F22E00E123E0ED
:109FE0004FE262E180E393E10E940AC635E4E32E8A
:109FF00032E0F32E23E04FE267E680E393E10E9434
:10A000000AC668CE80E08ECF8FEF8CCF0F931F9360
:10A01000CF93DF93FC01EB0180913F0790914007C4
:10A02000A0914107B0914207B7FF08C010923F07C7
:10A0300010924007109241071092420780912E071C
:10A0400090912F07A0913007B091310740913F07C1
:10A05000509140076091410770914207841795071E
:10A06000A607B70744F480933F0790934007A09357
:10A070004107B0934207809167018823E1F0609126
:10A080003F077091400780914107909142070091EE
:10A090003207109133072091340730913507600F54
:10A0A000711F821F931F0995BC0180913807909101
:10A0B00039070E94D26E80912407811108C08091D7
:10A0C0002B078823A9F180916701882389F180916A
:10A0D0003607909137070097B1F040913F075091B4
:10A0E000400760914107709142070091320710913B
:10A0F00033072091340730913507400F511F621FFD
:10A10000731FFE010995E0912C07F0912D07309700
:10A1100041F080912B07811103C0809124078111A8
:10A120000995809124071092240781110E942544EB
:10A13000DF91CF911F910F91089564E47BE18DE54C
:10A140009BE164CF61EC7BE189E891E45FCF6FEC48
:10A150007BE182EF9CE15ACF63EE7BE187EF9BE1ED
:10A1600055CF60E37CE185EA91E450CFE091D903DB
:10A17000E63028F581E08E0F8093D90340913F07A8
:10A1800050914007609141077091420720913A0732
:10A1900090913B078091940239E0E39FF0011124F4
:10A1A000ED55FC4FA0912A13B0912B13B183A083DE
:10A1B00042835383648375832683978380870895BE
:10A1C000A7E0B0E0E6EEF0E50C94A8E20E9472BDD4
:10A1D000F0903A072F2C85E08F0D8D833324339434
:10A1E00083E0E82E98EE892E93E0992EA12CB12CD5
:10A1F00084E08F198E839E2D9F199F8382E0D82E35
:10A20000DF18C32CCF18F1102CC080913D07882394
:10A21000C1F080916701882361F0622D619581E032
:10A2200090913D07911180E024E045E553E00E94C4
:10A23000BEBCF3949D81F912E6CF85E080933B0785
:10A240000CC08091240710922407882311F30E94E8
:10A25000254480913C078823E1F22796E2E10C94A3
:10A26000C4E281E0F8122DC090913D079130B9F021
:10A27000809167018823E9F281E0913009F080E064
:10A28000909198032DE133E0911102C029E133E070
:10A2900001E040E253E06C2D0E94396FCACF8091FB
:10A2A000240710922407882319F3809198038F259F
:10A2B00080939803E092670180913C078823C1F264
:10A2C000CCCF92E0F912D1C080913D07823021F1CC
:10A2D00080916701882309F4ACCF11E080913D079C
:10A2E000823009F010E06091060170910701072E9D
:10A2F000000C880B990B0E94C8DB69837A838B83DF
:10A300009C83CE0101960E949C4100E09C0142E1A9
:10A3100053E06D2D812FC0CF809124071092240728
:10A320008823B1F210E000E025EF30E050E040E09B
:10A3300066E071E082E193E00E9437BE80913C07C5
:10A34000882331F28ACF80913D07833019F18091C3
:10A350006701882309F46DCF11E080913D078330B8
:10A3600009F010E06091040170910501072E000CC6
:10A37000880B990B0E94C8DB69837A838B839C834B
:10A38000CE0101960E949C4100E09C014BE053E00D
:10A390006F81C0CF80912407109224078823B9F2DF
:10A3A00010E000E025EF30E050E040E064E071E0D4
:10A3B0008BE093E00E9437BE80913C07882339F2FE
:10A3C0004CCF8091240710922407882309F459C0A8
:10A3D00020E030E048EC52E460910001709101010E
:10A3E00080910201909103010E9427DC0E94C4E346
:10A3F0002B0130923C07BADEE092670183E093E0E4
:10A40000909339078093380780E091E09093370765
:10A410008093360710923207109233071092340758
:10A420001092350780922E0790922F07A092300746
:10A43000B0923107712C612C40923F075092400737
:10A4400060924107709242078CEA90E590932B133B
:10A4500080932A1310922D0710922C0710922B072D
:10A4600080913C07882369F0F8CE83E0F81609F460
:10A470006ACF94E0F912DDCE80913D07843009F473
:10A48000A0CF80916701882309F4D3CE11E0809199
:10A490003D07843009F010E0409000015090010128
:10A4A000609002017090030120E030E0A901C30137
:10A4B000B2010E94C2DB2DEB37E346E055EB87FD8E
:10A4C00004C02DEB37E346E055E3C301B2010E941F
:10A4D000E0E269837A838B839C83CE0101960E949C
:10A4E000CE1900E09C0143E053E06E8113CFB0E051
:10A4F000A0E0EDE7F2E50C94B8E28D8190916A104E
:10A50000891778F080936A109E01285F3F4F4E8133
:10A510005F8164E570E085E190E10E948ADB109242
:10A520001410E2E00C94D4E20F931F93CF93DF93C7
:10A530006F3F11F410926A1020916A1021111EC011
:10A540008C010E9411DB800F911FEC01C01BD10B0D
:10A55000C535D1053CF00197FC012491207C2038C1
:10A56000D1F3F3CFDD27AE01B80185E190E10E9480
:10A5700032DBCB5EDF4E188210921410DF91CF9148
:10A580001F910F9108958F929F92AF92BF92DF9289
:10A59000EF92FF920F931F93CF93DF93CDB7DEB768
:10A5A000C658D1090FB6F894DEBF0FBECDBFC35851
:10A5B000DF4F188219821A821B82CD57D0408091BA
:10A5C000870290918802A0918902B0918A02CF57A8
:10A5D000DF4F88839983AA83BB83C158D04084E628
:10A5E00090E09093741280937312109298121092CC
:10A5F00097121092160464E070E0CE018F579F4FBF
:10A600000E949AC180917312909174120296909355
:10A61000741280937312109298121092971281E024
:10A62000CA57DF4F8883C658D040CE018A579F4F04
:10A630000E942E2068E470E08FE39DE00E949AC1A2
:10A6400080E1EEE8F1E08E010F5F1F4FD80101902D
:10A650000D928A95E1F760E170E0C8010E949AC10D
:10A6600081E697E00E9436208CE0F80111928A95ED
:10A67000E9F7C8010E9432207E01FDE6EF0EF11CD1
:10A680008FEFF7018083C7010E942E2019821A8262
:10A690001B821C82C8010E9436208091B5029091D5
:10A6A000B602A091B702B091B80289839A83AB83B6
:10A6B000BC83C8010E943620C358DF4F188219821C
:10A6C0001A821B82CD57D04083E0F70180838983B3
:10A6D000CE0183589F4F0E943620C7010E942E2032
:10A6E000C8010E942E203AE0D32EDA94DD2031F00A
:10A6F000CE0183589F4F0E943620F7CF83EF92E11F
:10A700000E943220C358DF4F188219821A821B829E
:10A71000CD57D0402AE0D22EDA94DD2031F0CE01A0
:10A7200083589F4F0E943620F7CF87E08983F70137
:10A730008083C8010E942E20C7010E942E2068E05D
:10A7400070E08AEB92E00E949AC168E070E08DEAC6
:10A7500092E00E949AC164EC70E08AEC92E00E9460
:10A760009AC11982BB24BA94F701B082C8010E9431
:10A77000F0C1C7010E942E2080E1D82EF8018D2D56
:10A7800011928A95E9F760E170E0C8010E949AC1D0
:10A790001982C8010E94F0C168E070E082EC92E08A
:10A7A0000E949AC1198A1A8A1B8A1C8A80E090E04A
:10A7B000A0E8BFE38D879E87AF87B88B80918B120F
:10A7C00090918C12A0918D12B0918E1289839A83F0
:10A7D000AB83BC8320E030E543EC50E460918F1202
:10A7E0007091901280919112909192120E9427DCA8
:10A7F0006D837E838F8398872CEA35EC47E25EE396
:10A80000609193127091941280919512909196128A
:10A810000E9427DC69877A878B879C8764E170E0D8
:10A82000C8010E949AC184E190E09A83898362E022
:10A8300070E0C8010E949AC18CE0EEE9F1E0D80115
:10A8400001900D928A95E1F7C8010E942A208CE0C0
:10A85000EEE9F1E0D80101900D928A95E1F7C80187
:10A860000E942A201982C8010E942E208FE7898326
:10A87000C8010E942E20B982C8010E942E2085E0C6
:10A88000EAEAF1E0D80101900D928A95E1F765E0DE
:10A8900070E0C8010E949AC11982C8010E94F0C1EB
:10A8A00080E2EFEAF1E0D80101900D928A95E1F79C
:10A8B00060E270E0C8010E949AC1F7011082C701EE
:10A8C0000E94F0C11982C8010E94F0C180E090E0AE
:10A8D000A0EEBFE3C358DF4F88839983AA83BB836D
:10A8E000CD57D040CE0183589F4F0E943620C35889
:10A8F000DF4F188219821A821B82CD57D040CE01B9
:10A9000083589F4F0E94362082E1F80111928A9568
:10A91000E9F762E170E0C8010E949AC184E2EFECBD
:10A92000F1E0D80101900D928A95E1F764E270E0C0
:10A93000C8010E949AC1F8011192DA94E9F760E126
:10A9400070E0C8010E949AC189E0F80111928A95CD
:10A95000E9F769E070E0C8010E949AC1C358DF4F6F
:10A96000188219821A821B82CD57D040CE0183589B
:10A970009F4F0E9436209CE0D92EF8018D2D119218
:10A980008A95E9F76CE070E0C8010E949AC18CE6F4
:10A99000F80111928A95E9F76CE670E0C8010E940F
:10A9A0009AC18AE094E00E942A20F7011082118265
:10A9B00012821382148215821682178268E070E078
:10A9C000C7010E949AC1F7011192DA94E9F7CB57B7
:10A9D000DF4F1882C558D04080E090E0A0E4B0E49A
:10A9E000ED968CAF9DAFAEAFBFAFED97C7010E94A4
:10A9F0003220CE018B579F4F0E942E20CE018758C8
:10AA00009F4F0E943620D0901604D11048C000916C
:10AA1000731210917412045611098091971290913B
:10AA20009812F7019183808384E690E090937412EA
:10AA30008093731264E070E08FE192E00E949AC10B
:10AA400062E070E0C7010E949AC10E94108189EF04
:10AA500099E00E94B27BC8010E946B75F70180806B
:10AA60009180B12CA12C8CEE99E00E94B27BC501A3
:10AA7000B4010E9437A589EE99E00E94B27B0431AF
:10AA8000134041F00E940D818BE09AE00E94B27B5E
:10AA9000DD24D394809116048D298093160480912F
:10AAA0001604811104C060E089ED99E03DDD9091CC
:10AAB000160481E08927CA57DF4F0FB6F894DEBF2E
:10AAC0000FBECDBFDF91CF911F910F91FF90EF90FF
:10AAD000DF90BF90AF909F908F90089554DD0C94BD
:10AAE0004042CF930E94343D4EDDC82F882319F099
:10AAF00080E00E94D9278C2F0E9440420E94904300
:10AB0000CF910895CF9380919B03811109C08CED63
:10AB100091E09093DF038093DE0381E080939B03B9
:10AB200025DB20E040E070E060E080E091E20E9400
:10AB30005442C1E0C09394020E9423290E942544FC
:10AB4000C093940260E08FE99CE2EEDC88ED91E036
:10AB50009093DE068093DD06CF910895A6E0B0E0E5
:10AB6000E4EBF5E50C94A8E20E947075382E809114
:10AB7000821484FB662460F8412C84FF03C00E9489
:10AB80008375482E0E9472BD20913A072D83522E64
:10AB90002B5F298380E00FED14E091E0792E75188A
:10ABA000952D91959A8392E8E92E95E5F92E2CEF53
:10ABB000C22E24E0D22E92E095199B8393E0951942
:10ABC0009C833BE9832E34E0932E40EBA42E44E09B
:10ABD000B42E9D812981921709F409C2992349F164
:10ABE00031106AC00E947E7B882309F47AC19D815E
:10ABF000913009F444C122E02E832D818E812813E7
:10AC00005FC180913D07281709F46EC180916701EB
:10AC1000882309F455C16D81651981E090913D0744
:10AC20002D81921380E023E048ED54E00E94BEBCE9
:10AC300047C180913D07882379F18091670188237E
:10AC400079F281E090913D07911180E024E048E0A5
:10AC500055E06A810E94BEBC332021F224E02E839D
:10AC60009D812E8192134AC080913D07981709F467
:10AC70004CC180916701882309F440C06D8165193A
:10AC800081E090913D072D81921380E023E04CEC10
:10AC900054E00E94BEBC32C0809124071092240769
:10ACA000882359F20E94254480913C07882329F289
:10ACB0002696E2E10C94C4E28D81813009F47FC0D4
:10ACC000823009F4A6C09D81933041F680913D0702
:10ACD000833009F4C3C080916701882309F4BECF93
:10ACE00081E090913D07933009F080E023E04CEE45
:10ACF00054E06C810E94BEBC84E08E838E818F5FA5
:10AD00009D81981316C080913D07981709F40EC1D4
:10AD100080916701882369F06D81651981E09091C8
:10AD20003D072D81921380E023E04EEB54E00E941A
:10AD3000BEBC8E818E5F662009F430C141103BC0DD
:10AD40009D8198131BC020903D07921509F4FFC008
:10AD500080916701882391F01F92BF92AF928D81FD
:10AD600085198F9381E02D81221180E08F930E94BD
:10AD7000BF200F900F900F900F900F908E818D5FDE
:10AD80009D81981316C080913D07981709F4F5C06E
:10AD900080916701882369F06D81651981E0909148
:10ADA0003D072D81921380E023E04FE954E00E949B
:10ADB000BEBC8E818C5F9D819F5F9D830ACF8091F9
:10ADC0003D078130D1F080916701882309F446CF97
:10ADD000FF92EF92DF92CF927F9281E090913D07B8
:10ADE000913009F080E08F930E94BF200F900F9068
:10ADF0000F900F900F900F9031CF809124071092F9
:10AE00002407882301F37EDE80913C078823D9F252
:10AE10004FCF80913D07823091F080916701882368
:10AE200009F41CCF81E090913D07923009F080E059
:10AE300023E041EF54E06B810E94BEBC0FCF8091B4
:10AE4000240710922407882341F38BED9DE40E9490
:10AE5000C8BD80913C07882301F32ACF8091240745
:10AE600010922407882309F436CF83E494E40E94E7
:10AE7000C8BD80913C07882309F42DCF19CF80915C
:10AE80003D07813009F180916701882309F4B3CE31
:10AE90008DE590E49F938F931F930F937F9281E0B2
:10AEA00090913D07913009F080E08F930E94BF2080
:10AEB0000F900F900F900F900F900F9082E08E8365
:10AEC0008E818F5F8E83CCCE8091240710922407D1
:10AED0008823C9F20E945D4080913C07882399F243
:10AEE000E7CE91E09E8389CE8091240710922407BB
:10AEF000882309F48BCE83E397E40E94C8BD809138
:10AF00003C07882309F482CED3CE80912407109287
:10AF10002407882309F4ADCE83EC95E40E94C8BDD4
:10AF200080913C07882309F4A4CEC2CE80912407E7
:10AF300010922407882309F4EBCE81E29FE50E945A
:10AF4000C8BD80913C07882309F4E2CEB1CE809140
:10AF5000240710922407882309F4FACE4FE350E027
:10AF60006AE874E08FED96E00E9419E580913C0755
:10AF7000882309F4EDCE8D811ECF80912407109295
:10AF80002407882309F404CF87E590E60E94C8BD12
:10AF900080913C07882309F4FBCEEDCF9D81981367
:10AFA00014C090913D072D81291791F08091670180
:10AFB000882359F06D81651981E02D81291380E086
:10AFC00020E24EE854E00E94BEBC8E818D5FF3CE3D
:10AFD0008091240710922407882341F39092DE0683
:10AFE0008092DD0680913C07882301F3C4CF8093D3
:10AFF0003B075ECE10929202109266010E9483750A
:10B000009091821480FB97F99093821460E08AEC0F
:10B0100091E08ADA0C9490430F931F930E94F3C13E
:10B0200000918E0210918F02209190023091910236
:10B03000601B710B820B930B97FD0CC089B183FBD6
:10B04000882780F991E089274A9B8260309B846041
:10B0500080938D0280918D02817090918D0291FD7F
:10B06000826090919A03981749F0813009F148F075
:10B07000823079F0833091F080939A031F910F9181
:10B080000895913079F09230B9F790918C029150F7
:10B090000CC0992339F09330C1F3EECF9130A9F36E
:10B0A000923051F790918C029F5F90938C02E4CF85
:10B0B000992359F3933001F7F5CF1F93CF93DF9383
:10B0C000809134018F3708F468C08F5790918A12AD
:10B0D00090938504992309F465C05D9A8F5F8093EE
:10B0E00034018091840491E0892780938404811144
:10B0F00093DF8091330191E0980F83300CF090E062
:10B10000813009F485C00CF04FC0882309F462C077
:10B1100090933301C0914E07D0914F07209709F4C7
:10B120002DC0F89413B1147082E00E94C42700C0AF
:10B1300000C01C161D060CF08BC02A9A00C000C06F
:10B140002B9A00C0000082E090E00197F0F72B9866
:10B1500000C000C0112309F47DC02A9A00C000C0BD
:10B16000789480914E0790914F071C161D060CF0A5
:10B1700073C0019790934F0780934E078091870D7E
:10B180009091880D009729F001979093880D8093F6
:10B19000870DDF91CF911F910895909185048917B4
:10B1A00008F49CCF5D989ACF8230E9F1833009F0A2
:10B1B000AFCF80918304811103C087E08093830423
:10B1C00080918304815080938304882309F4A0CF65
:10B1D00093E09ECF809132018F5F80311CF4809389
:10B1E000320196CF109232018091990381110BC0E8
:10B1F0002091801230918112309383122093821219
:10B2000081E080939903109281121092801280CF76
:10B2100010927B0087E480937C0080917A008064A8
:10B2200080937A0075CF80917A0086FD0FC040919F
:10B230007800509179002091801230918112240F72
:10B24000351F309381122093801262CF92E060CF3D
:10B250002A9874CF2A9882CF01968CCFA4E8B0E0C8
:10B26000E4E3F9E50C94A8E22DB73EB7CD57DF4FE4
:10B2700039832883C358D04084E690E090937412B9
:10B2800080937312109298121092971241E064E02A
:10B2900070E0CE0187589F4F0E9493A743E050E093
:10B2A000BE0167587F4F8FE192E00E940BE5892B2A
:10B2B000F1F1ED968FADED97882339F08FE3EA96A3
:10B2C0008FAFEA97EB961FAEEB970E941081BE01FD
:10B2D00067587F4F83EA9AE00E94BF7B85E99AE036
:10B2E0000E94B27B82E00E941C4481E0809316049D
:10B2F00080918E03811107C080911F07833018F061
:10B3000080E00E94D9279091160481E08927CD57CB
:10B31000DF4F28813981C358D0400FB6F8943EBF23
:10B320000FBE2DBFCC57DF4FE2E10C94C4E241E0E9
:10B3300062E070E0CE0183589F4F0E9493A7E99688
:10B340001CAE1DAE1EAE1FAEE99710929812109261
:10B350009712CE018F579F4F0E941F20EDB6FEB669
:10B36000CF57DF4FC880C158D040D12C33E0C30E37
:10B37000D11CCC0CDD1CCC0CDD1C8DB79EB78C1900
:10B380009D090FB6F8949EBF0FBE8DBFEDB7FEB7F7
:10B3900031963F012DB73EB72C193D090FB6F894F1
:10B3A0003EBF0FBE2DBF8DB79EB701964C01EDB7C6
:10B3B000FEB7EC19FD090FB6F894FEBF0FBEEDBF46
:10B3C0000DB71EB70F5F1F4FB601C3010E942420A7
:10B3D00040918E0381E0482764E070E08FE49DE0B7
:10B3E0000E9493A7B601C4010E942420B601C8019F
:10B3F0000E942420F0918E03CE57DF4FF883C2586D
:10B40000D040F1114FC0CF57DF4F8881C158D04095
:10B4100090E00296AFE3BDE050E040E030E020E095
:10B4200063E17BE0E3E0CE2EEBE0DE2EF3EFAF2E28
:10B43000FAE0BF2E821793070CF495C0F301E40FD6
:10B44000F51F20803180428053802D923D924D9295
:10B450005D92821793070CF48CC0F401E40FF51F82
:10B46000208031804280538050962D923D924D92A3
:10B470005C925397821793070CF481C0F801E40F94
:10B48000F51F208031804280538090962D923D920E
:10B490004D925C9293972F5F3F4F4C5F5F4F2430EC
:10B4A000310541F683E79DE00E94F71F87E79DE0A5
:10B4B0000E94F71F8BE79DE00E94F71F8FE79DE03A
:10B4C0000E94F71F83E89DE00E94F71FCE018B5872
:10B4D0009F4F0E94F71FCE018B589F4F0E94F71F6E
:10B4E000CE018B589F4F0E94F71FCE018B589F4F64
:10B4F0000E94F71F81E697E00E94F71F0FB6F894AD
:10B50000FEBE0FBEEDBE8E010F5F1F4FC8010E9431
:10B510001720CE0183599F4F0E94FF1FC8010E9430
:10B52000F71F87E194E00E94F71FCE018B589F4FD1
:10B530000E94F71FCE0183599F4F0E941F20C80110
:10B540000E941F20AE96CFACAE978981C89E600145
:10B55000112421E0C21AD108C0F0CE018B589F4FB0
:10B560000E94F71FF6CFFB0125903590459054902F
:10B570006CCFF601259035904590549075CFF5012C
:10B58000259035904590549080CF83EF92E10E94B2
:10B5900017208AE0D82EDA94CE01DD2029F08B58CE
:10B5A0009F4F0E94F71FF7CF80589F4F0E941F2088
:10B5B000CE0181589F4F0E941F20C058DF4F8881C5
:10B5C000C058D040873009F046C1C158DF4F88814C
:10B5D000CF57D040873009F03EC1CE57DF4F88812A
:10B5E000C258D040811102C00E9490738AEB92E051
:10B5F0000E940F208DEA92E00E940F2040918E035E
:10B6000081E0482764EC70E08AEC92E00E9493A706
:10B61000CE0183599F4F0E940720C8010E94FF1F3F
:10B6200040918E03FF24F3944F2560E170E0C80140
:10B630000E9493A7C8010E94072040918E034F25C6
:10B6400068E070E082EC92E00E9493A740918E0344
:10B650004F2564E170E0C8010E9493A7D0908E034B
:10B66000D11030C089819A81AB81BC8180938B12CB
:10B6700090938C12A0938D12B0938E122CEA35EC1D
:10B6800047E25EE36D817E818F8198850E9427DC91
:10B6900060938F12709390128093911290939212F4
:10B6A00020E030E543EC50E469857A858B859C8504
:10B6B0000E9427DC609393127093941280939512EA
:10B6C00090939612FF24F3944D2D4F2562E070E085
:10B6D000C8010E9493A7C8010E94EF1FC8010E94E1
:10B6E000EF1FC8010E94FF1FC8010E94FF1FC80171
:10B6F0000E94FF1F85E0F80111928A95E9F74091B9
:10B700008E034F2565E070E0C8010E9493A7C80131
:10B710000E94072040918E034F2560E270E0C8012F
:10B720000E9493A7CE0183599F4F0E94072040910A
:10B730008E034F2569E070E0C8010E9493A74091F5
:10B740008E034F2562E170E0C8010E9493A74091EB
:10B750008E034F2564E270E0C8010E9493A74091D8
:10B760008E034F2560E170E0C8010E9493A74091CD
:10B770008E034F2569E070E0C8010E9493A7C801BD
:10B780000E94F71F40918E034F256CE070E0C801C6
:10B790000E9493A740918E034F256CE670E0C8018C
:10B7A0000E9493A719821A821B821C821D821E820C
:10B7B0001F82188619861A861B861C86C8010E945D
:10B7C000EF1F40918E034F2568E070E0C8010E9492
:10B7D00093A7C8010E941720CE0181589F4F0E9455
:10B7E000FF1FCE0183599F4F0E94F71F8091731254
:10B7F000909174128837934009F44DC00E940D81D6
:10B800008BE09AE00E94B27BF09216040E941081B5
:10B810006091731270917412645671098DE89AE008
:10B820000E94768185E89AE00E94B27B84E193E0F1
:10B830000E946B758AE00E94917B81E00E941C440B
:10B8400080918E03811154CD80911604811150CDC9
:10B850000E947A3C4DCDCE0183599F4F0E940F200C
:10B86000C8010E940F20C058DF4FC880C058D04088
:10B87000C158DF4F8881CF57D040C89E6001112446
:10B8800091E0C91AD10808F4C3CECE018B589F4F5E
:10B890000E94F71FF5CF1092160420919712309155
:10B8A0009812EF968EAD9FADEF972817390701F1EB
:10B8B000F09216040E940D81EF960EAD1FADEF972A
:10B8C00085E69AE00E94B27BC8010E946B750091E8
:10B8D00097121091981280E69AE00E94B27BC801FC
:10B8E0000E946B7580E59AE00E94B27B80E0A6CF53
:10B8F00080918E038111A4CF0E9410818FE192E08C
:10B900000E94987B60917312709174126456710951
:10B9100083E39AE00E94768180909712909098122B
:10B92000B12CA12C86E29AE00E94B27BC501B40141
:10B930000E9437A583E29AE00E94B27B81CF81E02A
:10B9400080938E038BDC10928E03882309F086CCC3
:10B950000E94343D80E00895F2DF0C944042A7E05D
:10B96000B0E0E5EBFCE50C94A8E280914D07877010
:10B9700089838090BA029090BB02A090BC02B090E4
:10B98000BD020E9472BD20913A072E833981373063
:10B9900009F075C085E194E09B838A831E81312F75
:10B9A0003B5F3C8333243394812F81958D83232CFB
:10B9B000211A84E6482E512C612C712C2E812223D1
:10B9C00009F462C03981373009F434C22E81213044
:10B9D00009F029C290913D07913009F445C1809149
:10B9E0006701811154C182E0F82E81E08F0D8F83B1
:10B9F0009981973009F063C020E030E0A901C501CA
:10BA0000B4010E94C2DB882309F459C03F818E81B2
:10BA1000381331C09091B9029F8380913D072E81E8
:10BA2000821311C08091240710922407882359F0B3
:10BA300093259F8383E0809367010E943A20809141
:10BA40003C0781110DC1809167018823A1F06E81AF
:10BA5000611B81E090913D073E81931380E09F81BF
:10BA600026EF33E0911102C022EF33E001E049EF0D
:10BA700053E00E94396FF394F394FF8220C020E1D9
:10BA800034E03B832A838ACF80913D07882309F4E1
:10BA9000D9C080916701882309F494CF81E0909107
:10BAA0003D07911180E024E043E254E06D810E9463
:10BAB000BEBC8981873009F41DC193E09F838091CA
:10BAC000B5029091B602A091B702B091B8028093EE
:10BAD000200790932107A0932207B09323072F817B
:10BAE0003E8123131EC080913D07821709F407C1D0
:10BAF000809167018823A9F0EE80E11AFF24F39476
:10BB000080913D073E818313F12C80E297E00E94F3
:10BB10004C4100E09C0146EE53E06E2D8F2D0E94BB
:10BB2000396F8F818F5F9E81891316C080913D0789
:10BB3000891709F439C180916701882369F06E8102
:10BB4000611B81E090913D072E81921380E023E0FC
:10BB500047ED53E00E94BEBC8F818E5F3E81831310
:10BB600016C080913D07831709F42FC180916701AA
:10BB7000882369F06E81611B81E090913D072E81E1
:10BB8000921380E023E04AEC53E00E94BEBC8F8118
:10BB90008D5F3E81831323C080913D07831709F495
:10BBA00025C1809167018823D1F08CEA9CE59F93A1
:10BBB0008F938CEB93E09F938F938E81811B8F9358
:10BBC00081E090913D073E81931380E08F930E9426
:10BBD000BF200F900F900F900F900F900F908F81BC
:10BBE0008C5F9E81891323C080913D07891709F4DA
:10BBF0000BC1809167018823D1F08EE695E59F9374
:10BC00008F938DEA93E09F938F938E81811B8F9307
:10BC100081E090913D072E81921380E08F930E94E6
:10BC2000BF200F900F900F900F900F900F903E81BC
:10BC30003F5F3E838C818313C1CE9F819B5F909336
:10BC40003B070EC08091240710922407882309F433
:10BC500020CF0E94254480913C07882309F419CF06
:10BC60002796E2E10C94C4E2809124071092240705
:10BC7000882309F4B4CE26EB35E03093DE0620931A
:10BC8000DD0680913C07882309F4A9CEE9CF81E045
:10BC9000913009F080E020E249E154E0622D0E94F9
:10BCA000BEBCA1CE90913D073E81931731F08091AB
:10BCB0006701811113C08E8197CE80912407109265
:10BCC00024078823A1F32A813B813093DE06209349
:10BCD000DD0680913C07882351F3C2CF6E81611B42
:10BCE00081E03E81931380E020E246E054E00E9430
:10BCF000BEBCE1CF22E02F83FF24F3947DCE809160
:10BD0000240710922407882309F4F2CE0E9466BD0E
:10BD1000609120077091210780912207909123075D
:10BD20000E94C4E36B0130923C070E94B65083E04E
:10BD30008093670186EE93E09093390780933807EC
:10BD400020E237E03093370720933607109232070E
:10BD500010923307109234071092350740922E0745
:10BD600050922F076092300770923107F12CE12C2E
:10BD7000C0923F07D0924007E0924107F0924207FD
:10BD800082EA90E590932B1380932A1320E430E20B
:10BD900030932D0720932C0710922B0780913C079E
:10BDA000882309F4A5CE5CCF809124071092240744
:10BDB000882309F4C0CE87E59EE40E94C8BD809127
:10BDC0003C07882309F4B7CE4BCF8091240710920B
:10BDD0002407882309F4CACE82E593E40E94C8BDF3
:10BDE00080913C07882309F4C1CE3ACF8091240783
:10BDF00010922407882309F4D4CEAEDD80913C074D
:10BE0000882309F4CECE2CCF8091240710922407EA
:10BE1000882309F4EECE0E946E5580913C0788235A
:10BE200009F4E7CE1DCF2E81223009F43BCF33E059
:10BE30003F8345CE8E81813009F434CF92E09F83D9
:10BE40005BCFB0E0A0E0E7E2FFE50C94ABE20E943C
:10BE5000F520D82F0E9472BDC0913A075C2E85E074
:10BE6000682E6C0E9CEAE92E9CE5F92E2BE3C22E7F
:10BE700024E0D22E14E01C1B31E5A32E32E4B32EB5
:10BE800005E00C1B83E0982E9C1A82E0882E8C1A09
:10BE900081E0782E7C1AC11141C080913D07882332
:10BEA00061F180916701882361F0652D619581E0E2
:10BEB00090913D07911180E024E049E754E00E9411
:10BEC000BEBCD111EDC0C43009F0A0C080913D07C7
:10BED000843009F480C080916701882309F4B6C0DA
:10BEE000FF92EF92DF92CF921F9381E090913D07F6
:10BEF000943009F4A2C080E0A0C080912407109281
:10BF00002407882371F20E94254480913C078823EE
:10BF100041F2CDB7DEB7EFE00C94C7E2C13031F5A6
:10BF200080913D07813099F080916701882361F00D
:10BF300081E090913D07913009F080E023E047E6F1
:10BF400054E0672D0E94BEBCD111AAC07FC0809171
:10BF5000240710922407882339F38FE09BE40E9482
:10BF6000C8BD80913C078823F9F2D3CFC23009F0D5
:10BF70006FC080913D07823081F0809167018823F6
:10BF800009F48BC081E090913D07923009F080E088
:10BF900023E048E554E0682DD5CF80912407109226
:10BFA0002407882351F387E59EE40E94C8BD809151
:10BFB0003C07882311F3ADCF80912407109224070A
:10BFC000882309F44DC00E946E5580913C07882358
:10BFD00009F446C09ECF809124071092240788233D
:10BFE00009F479CFB9DC80913C07882309F473CF39
:10BFF00090CF8091240710922407882369F00E9433
:10C00000514280913C07882339F083CFC530F1F449
:10C0100080913D07853069F3809167018823B1F0F5
:10C02000BF92AF928AE294E09F938F930F9381E047
:10C0300090913D07953009F05ECF8F930E94BF200D
:10C040000F900F900F900F900F900F9086E029C0E7
:10C05000C33009F036CF80913D07833009F4ACCF6F
:10C06000809167018823C9F08EE695E59F938F93B1
:10C0700089E494E09F938F939F9281E090913D0794
:10C08000933009F080E08F930E94BF200F900F90B3
:10C090000F900F900F900F9057CFDD2309F4B6CF7C
:10C0A00084E0CF5F6C12F7CE80933B0732CFACE3D6
:10C0B000B0E0EDE5F0E60C94A8E280913E0788231D
:10C0C00069F18091821410E000E084FF23C084EBCA
:10C0D00092E10E943C228BE1E4EBF2E1DE019196D9
:10C0E00001900D928A95E1F710E000E0BE016F5FCC
:10C0F0007F4FCE0181960E94E7CB18163CF4CE010B
:10C1000001960E945AC6080F111DF0CFCE018196EC
:10C110000E940C241093E9030093E8030E9472BD6F
:10C1200010913A07312E85E0810F8CAF212E21949A
:10C1300082E8A82E8BE1B82E91E5892E95E0992E04
:10C1400001E0011B26E5622E25E0722E111113C0BD
:10C1500080913D07882391F180916701882359F0F0
:10C1600081E090913D07911180E024E04FE555E09A
:10C17000622D0E94BEBC8091821486FF3EC01130A9
:10C18000D9F480913D07813049F18091670188237E
:10C1900009F43EC11F927F926F920F9381E09091BC
:10C1A0003D07913009F080E08F930E94BF200F90EF
:10C1B0000F900F900F900F9082E04FC08091240756
:10C1C00010922407882341F20E94254480913C0765
:10C1D000882311F2EC96E2E10C94C4E280912407EA
:10C1E00010922407882389F210923A070E9413CDF7
:10C1F00080913C07882349F2EDCF84FF2DC0113098
:10C20000D9F680913D078130D1F080916701882374
:10C2100009F4FEC0BF92AF929F928F920F9381E07C
:10C2200090913D07913009F080E08F930E94BF20EC
:10C230000F900F900F900F900F900F90BDCF8091A7
:10C24000240710922407882301F30E94821B809107
:10C250003C078823D1F2BECF81E0909167019923FA
:10C2600009F4D7C0582ED12CC12C412E4318852D4E
:10C27000E090E803F090E903CE14DF0408F0C9C0B1
:10C280005112A5C091E0E91AF108EC18FD0884EB01
:10C2900092E10E943C228BE1E4EBF2E1DE01919617
:10C2A00001900D928A95E1F7F12CBE016F5F7F4FEF
:10C2B000CE0181960E94E7CB18167CF4CE01019640
:10C2C0000E945AC6882389F3EF106BC0BE016F5FCE
:10C2D0007F4F80E597E00E9475C6CE0181960E944F
:10C2E0000C248091821490913D0785FF75C09113B5
:10C2F00063C08091240710922407882309F45CC04E
:10C3000019821C828091B7126FEC72E1882311F0C0
:10C3100064EB72E121E040E557E0CE0101960E9416
:10C320001124882309F43FC08BE1FE013196A4EB70
:10C33000B2E101900D928A95E1F7809182148F7B92
:10C3400080938214A0917814AA3080F481E08A0F3F
:10C35000809378148BE18A9FD0011124A659BC4E9A
:10C36000E4EBF2E101900D928A95E1F7CE0101969E
:10C370000E940C2410923A0782E090E0A0E0B0E026
:10C3800080933F0790934007A0934107B0934207E3
:10C3900081E080933C071092930283E080936701D1
:10C3A00019CFF39482CF0E94108160E577E08BE390
:10C3B00095E00E9470CEDACF80916701882339F032
:10C3C00081E0911380E041E0642D0E94FCBC8FEF7E
:10C3D000C81AD80A53944BCF911759F0809167012E
:10C3E0008823A9F381E090913D07911380E040E01C
:10C3F000EBCF8091240710922407882379F387E9F3
:10C400009DE40E94C8BD80913C07882339F3E2CEA9
:10C4100082E01F5F9CAD911399CE80933B07DACEEB
:10C42000FC01A081B1811C92A281B3818C918F5FAC
:10C430008C930280F381E02D90818CE0989F800D99
:10C440001124ECE2F3E113AE84AF0895FC01849172
:10C450000895FC0180810895009751F0FC0180E06F
:10C460009191992331F0907C9038D1F38F5FF8CF80
:10C4700080E00895119800C087FD43C0419800C036
:10C48000119A00C000C0119800C086FD46C04198B6
:10C4900000C0119A00C000C0119800C085FD3BC0CB
:10C4A000419800C0119A00C000C0119800C084FDDE
:10C4B00030C0419800C0119A00C000C0119800C05F
:10C4C00083FD25C0419800C0119A00C000C011989A
:10C4D00000C082FD1AC0419800C0119A00C000C07F
:10C4E000119800C081FD0FC0419800C0119A00C092
:10C4F00000C0119800C0419800C0119A00C000C04F
:10C500000895419ABCCF419AF0CF419AE5CF419A24
:10C51000DACF419ACFCF419AC4CF419AB9CF90E0B8
:10C5200080E00895CF93DF93DB01F9019C91913076
:10C53000C1F0943080F094509C938830D1F4808185
:10C540009181009771F0019791838083480F591F63
:10C55000EA01188206C08C3539F49C5F9C939430B4
:10C5600041F4DF91CF9108958B3339F781E08C93BB
:10C57000F8CF20813181B9016F5F7F4F7183608374
:10C58000420F531FEA018883808191818F35910585
:10C590006CF7E7CF0F931F9381E000917E14109109
:10C5A0007F14209180143091811440917A1450911D
:10C5B0007B1460917C1470917D1404171507260775
:10C5C000370708F480E01F910F91089590E080E014
:10C5D00008952091E805833021F425FD0CC024FD49
:10C5E0000CC030E0A90102C0559547958A95E2F745
:10C5F000CA018170089581E0089580E008958091D6
:10C60000040684FD0BC08091060687FD07C090914B
:10C610000706937081E019F480E0089581E00895A1
:10C620002FEB280F2A3108F047C0E22FF0E080916D
:10C63000040690910506A0910606B091070604C075
:10C64000B695A795979587952A95D2F780FD02C054
:10C6500081700895E651FA4FE081EE2341F1809117
:10C660005F0790916007E80FF92FF11D808190ED31
:10C67000980F9A3030F08E3251F4818180538A3095
:10C6800098F4F093D905E093D80581E008958D32B0
:10C6900011F08B3249F4818190ED980F9A3088F334
:10C6A0008E3211F48281EACFF0E0E0E0EACF10921E
:10C6B000D9051092D805E9CF80E00895CF93DF9394
:10C6C00085E4AEDF882309F188E0409104065091AB
:10C6D00005066091060670910706972F9170C92F85
:10C6E00090E0D92FCC0FDD1F71FB222720F930E01D
:10C6F000220F331F220F331FC22B67FB442740F941
:10C70000C42B8C2BDF91CF91089580E0DECF88DFA2
:10C71000882341F081E02091D8053091D905232B61
:10C7200009F480E00895B0E0A0E0E9E9F3E60C94B4
:10C73000B1E26B01E9014A3009F4D5C0453109F095
:10C7400081C0DB011296ED91FC91F2809681878188
:10C75000139A00C00000E6E2F0E03197F0F7092FED
:10C76000182FEF2CE29420EFE22230E1B32EBF0C21
:10C77000E80188EF7FDE00C0000086E290E00197CC
:10C78000F0F7BFE1BF1508F49BC08F2D807780685C
:10C7900071DE8E2D6FDE00C0000086E290E0019712
:10C7A000F0F780E867DE80E065DE00C0000086E22A
:10C7B00090E00197F0F78AEF5DDE00C0000086E2AE
:10C7C00090E00197F0F7005F1F4F8881807F52DE75
:10C7D00089918295807F4EDEC017D107B1F700C0E6
:10C7E000000086E290E00197F0F7F394E0E1EE0EAE
:10C7F000FB10BECF1398D6011296ED91FC9180816B
:10C800009281980F92832181921708F09FC19481A1
:10C810009F5F94839381890F821710F08FEF820FAF
:10C820008383458150E0440F551F70E060E08681AE
:10C8300097810E94DFE481E0CDB7DEB7E9E00C9498
:10C84000CDE2DEC1FB0102811381423309F485C1CF
:10C8500008F48DC1463409F475C1473409F482C126
:10C860004B3349F789812B81D80112967C9112971D
:10C8700013963C91213009F4BFC1233009F0A0C1C7
:10C8800048EF480F582F91E0341708F490E031E05A
:10C89000541708F030E0492F432B61E0571708F494
:10C8A00060E0462311F4932331F2FA8030E0F9017D
:10C8B000E95CFD4FD0802D5C3D4FF901E08099C1CE
:10C8C00080EE8F0D8068807FD5DD8F2D8295807FF3
:10C8D000D1DD00C0000086E290E00197F0F780E82B
:10C8E000C9DD80E861CF0B9A1398399A4198099A6B
:10C8F000119A139A00C0000086E290E00197F0F7C9
:10C9000088E790E0CEE9DFE0FE013197F1F701978B
:10C91000D9F788EFAFDD00C0000086E290E0019714
:10C92000F0F780E2A7DD80E0A5DD00C0000086E230
:10C9300090E00197F0F780E09DDD80E89BDD00C08E
:10C94000000086E290E00197F0F780E093DD80E15F
:10C9500091DD00C0000086E290E00197F0F7CE0183
:10C960000197F1F7CE010197F1F7CE010197F1F7A9
:10C97000CE010197F1F7CE010197F1F7CE010197B2
:10C98000F1F7CE010197F1F7CE010197F1F7CE0152
:10C990000197F1F7CE010197F1F7CE010197F1F779
:10C9A000CE010197F1F7CE010197F1F7CE01019782
:10C9B000F1F72197F1F780E25DDD80E45BDD00C0F7
:10C9C000000086E290E00197F0F780E253DD80E618
:10C9D00051DD00C0000086E290E00197F0F7D0E062
:10C9E000C0E08C2F8077806845DD8D2F43DD00C04F
:10C9F000000086E290E00197F0F780E83BDD80E000
:10CA000039DD00C0000086E290E00197F0F78AEF80
:10CA100031DD00C0000086E290E00197F0F780E28F
:10CA2000119800C0419800C0119A00C000C0119830
:10CA300000C0419800C0119A00C000C0119800C009
:10CA4000419800C0119A00C000C0119800C04198E0
:10CA500000C0119A00C000C0119800C0419800C0E9
:10CA6000119A00C000C0119800C0419800C0119AEE
:10CA700000C000C0119800C0419800C0119A00C0C9
:10CA800000C0119800C0419800C0119A00C000C0B9
:10CA9000119800C0419800C0119A00C000C01198C0
:10CAA00000C0419800C0119A00C000C0119800C099
:10CAB000419800C0119A00C000C0119800C0419870
:10CAC00000C0119A00C000C0119800C0419800C079
:10CAD000119A00C000C0119800C0419800C0119A7E
:10CAE00000C000C0119800C0419800C0119A00C059
:10CAF00000C0119800C0419800C0119A00C000C049
:10CB000000C00000E6E2F0E03197F0F7815009F054
:10CB100087CF88EFAFDC00C0000086E290E001978D
:10CB2000F0F7CF5FD05FC03209F05BCF80E0A2DCCE
:10CB300080ECA0DC00C0000086E290E00197F0F7F6
:10CB4000139879CEF8018581888375CE80E0CDB7C2
:10CB5000DEB7E9E00C94CDE253C0B901C8010E94F0
:10CB600047C369CED80111968C91888364CE443135
:10CB700091F0473109F05FCE1882D80112968C915E
:10CB80001297898315968C91159781508A831396F5
:10CB90008C918B8350CED80115964C91159750E00F
:10CBA000440F551F70E060E016968D919C910E9495
:10CBB000DFE4F801128280818150838314823BCEAE
:10CBC000381708F438CE871708F435CEFA80E12CF0
:10CBD000D12C243070F46ACEBE01C8010E9447C334
:10CBE000898198819D0D98838E0D8983FF0C09F4AE
:10CBF00022CEF7FEF6CFF0CF58E0580F482F43CEA5
:10CC0000EF92FF920F931F93CF93DF93EC018B0171
:10CC10007A018A859B858617970731F088819981EB
:10CC20000E9434C51B870A87B701888199810E94B9
:10CC300034BD2E813F81820F932F911D9F838E8360
:10CC400090E080E0CDB7DEB7E6E00C94D0E2B0E053
:10CC5000A0E0EDE2F6E60C94B0E2EC017B018A0183
:10CC60008A859B858617970731F0888199810E9474
:10CC700034C5FB86EA8688859985019609F5CC80BE
:10CC8000DA808E81D80EA880B980D5015596ED91B5
:10CC9000FC91C5010995C80E780110E0F7012191BA
:10CCA0007F0121111FC08E819F81810F911D9F8364
:10CCB0008E8390E080E0CDB7DEB7EAE00C94CCE262
:10CCC000EE80FF80B801888199810E9434BD8E0D6D
:10CCD0009F2D911D288539852817390780F681E019
:10CCE00090E0E9CF4C2D6D2DC5010E948CC5D80E6A
:10CCF000180FD4CFB0E0A0E0E0E8F6E60C94B3E281
:10CD0000EC01D62E1CAD0BAD7C0184E0E80EF11CCD
:10CD1000E98DFA8DC7010995412F480F2D2D602F00
:10CD2000C7010E948CC59BAD890F8BAF81E090E05D
:10CD3000CDB7DEB7E7E00C94CFE2A6E0B0E0E3EADF
:10CD4000F6E60C94A9E27E836D83342EFC014080CC
:10CD5000518062807380C301B20120E13EE040E077
:10CD600050E00E94F0E149015A0189018CE3C82E8C
:10CD7000D12CE12CF12CC301B201A70196010E9434
:10CD8000F0E169837A838B839C83CA01B901A7018F
:10CD900096010E94F0E16B017C01332061F1C30137
:10CDA000B20120E831E541E050E00E94F0E12901C4
:10CDB0003A015901DF92CF92C40168E170E00E940C
:10CDC00044E29F938F935F924F9285E591E29F9308
:10CDD0008F93FE81FF938D818F930E945BDB0FB653
:10CDE000F894DEBF0FBECDBF88E0FAE04F165104C5
:10CDF000D8F089E019C081149104D1F48A818F930D
:10CE000099819F93DF92CF9289E491E29F938F93D0
:10CE1000EE81EF93FD81FF930E945BDB0FB6F894E8
:10CE2000DEBF0FBECDBF85E02696E1E10C94C5E2E2
:10CE30000436110568F4DF926F939F928F928DE311
:10CE400091E29F938F939E819F93ED81EF93E4CF27
:10CE5000DF926F939F928F9283E391E29F938F93E0
:10CE60009E819F93ED81EF930E945BDB0FB6F89458
:10CE7000DEBF0FBECDBF86E0D7CF8091D8059091A1
:10CE8000D905009731F04AE050E070E060E00C9482
:10CE9000E3D960E070E0CB0108958091D8059091CE
:10CEA000D905009731F04AE050E070E060E00C9462
:10CEB000B6D860E070E0CB010895EFDF97FD0AC0BF
:10CEC000ECDF6F3F71058105910509F02CF4E5DF7A
:10CED000862F089580E008958FEF0895CF93C62F91
:10CEE00016DC882311F0E9DFC82F8C2FCF9108952D
:10CEF0008091D8059091D905892B39F0DEDF91E03A
:10CF0000811101C090E0892F089591E0FCCFCF936B
:10CF1000DF93C82FD62FFBDB882321F0E9DFDF91D9
:10CF2000CF9108958C2F7CDB8111F9CF8D2FF7CF16
:10CF3000B4DFCB010895CF93DF93EB01E8DB8823C7
:10CF400011F0F6DFEC01CE01DF91CF9108950F9340
:10CF50001F93CF938091D8059091D9050097D9F070
:10CF6000FC018F01C1912C2F2F7D81F0C53411F070
:10CF7000C536B9F7F801108270E060E00E9460D712
:10CF8000F801C083CF911F910F91089570E060E088
:10CF90000E9460D7F7CF60E070E0CB01F3CFCF9273
:10CFA000DF92EF92FF926A017B01B1DB882319F0D7
:10CFB000CEDF6B017C01C701B601FF90EF90DF90DF
:10CFC000CF900895CF92DF92EF92FF92CF93C82F28
:10CFD0000E94F3C16B017C0124EA30E74DE75FE377
:10CFE000609108017091090180910A0190910B01F3
:10CFF0000E94C2DB87FD18C08AEF90E0A0E0B0E09D
:10D000008C0D9D1DAE1DBF1D80935306909354063D
:10D01000A0935506B0935606C0935C01CF91FF9044
:10D02000EF90DF90CF90089580E090E0DC01E8CFB2
:10D03000CF9380911406811154C0109267131092FF
:10D0400068131092691310923513109234131092D2
:10D050003713109236131092391381E080933813EE
:10D0600082E280933A1310923F1310923E13E3E54D
:10D07000F3E121E633E18FEF81932E173F07E1F7CC
:10D08000C1E0C09350132CE733EA3093461320934A
:10D090004513C0934713109248131092491390E41C
:10D0A00090934A1310924B132BE733EA3093621399
:10D0B0002093611324E531E030933313209332132E
:10D0C0009EE19093571391E1909358139CE19093B4
:10D0D000551380935413809353130E9486C3C093B7
:10D0E000140681E08093130684E791E2909377120F
:10D0F00080937612109279121092781253985B9A5C
:10D1000052985A9A3898409A0E940C5810928C0261
:10D11000CF910895FC0180E0309749F094919923D4
:10D1200031F0907C903809F08F5F3196F7CF0895F9
:10D13000B0E0A0E0EEE9F8E60C94B0E2EC015B01AF
:10D140008A01FB01099587FD10C0C82ED12CF12C56
:10D15000E12C2196F801C082D182E282F382CE01D5
:10D16000CDB7DEB7EAE00C94CCE2982F907E903CED
:10D17000A9F48F7190E0B0E0A0E06C017D0156E071
:10D18000CC0CDD1CEE1CFF1C5A95D1F7CE0101968C
:10D19000F50109958F73C82A2296DCCF982F907FCE
:10D1A000903E11F58F7090E0B0E0A0E06C017D0141
:10D1B00036E0CC0CDD1CEE1CFF1C3A95D1F7CE01FD
:10D1C0000196F50109958F73C82A46E0CC0CDD1C49
:10D1D000EE1CFF1C4A95D1F7CE010296F501099588
:10D1E0008F73C82A2396B6CF982F987F903F79F5F2
:10D1F000877090E0B0E0A0E06C017D0186E0CC0C8F
:10D20000DD1CEE1CFF1C8A95D1F7CE010196F501BD
:10D2100009958F73C82A96E0CC0CDD1CEE1CFF1C10
:10D220009A95D1F7CE010296F50109958F73C82A18
:10D2300026E0CC0CDD1CEE1CFF1C2A95D1F7CE019C
:10D240000396F50109958F73C82A249683CF982FEA
:10D25000907C903841F4807C803869F42196CE012E
:10D26000F5010995F8CF8E7F8D3F28F02196CE01EC
:10D27000F5010995F8CFC12CD12C76016BCF9CE03C
:10D28000899F802D112491E0980F909312062CE035
:10D29000280F2093480730E02E5F3F4F40916413E2
:10D2A0004217130619F014F080E0089520916613D8
:10D2B0009217D0F7662341F08E5F0E946BC4809175
:10D2C00048078E5F0E946BC4809148079091641359
:10D2D000891750F32091661390911206291720F3B5
:10D2E000109267138093681381E0089520911106CE
:10D2F000022E000C330B8217130641F080931106A7
:10D3000069E972E280E393E10C9434C50895ACE0DE
:10D31000B0E0EDE8F9E60C94B2E26F3F71058105EB
:10D32000910509F070F48CE293E1E4DCE0913413B0
:10D33000F09135133196849190E02C96E8E00C94AE
:10D34000CEE2F0906713E09068132091130621114C
:10D350000FC043E151E26E2D8F2D0E94E5C590E094
:10D3600080E0F80EF0926713E09268139927E5CFFA
:10D37000C0903413D090351320E333E13A832983EE
:10D380002F2D30E03C832B832E2D30E03E832D83E8
:10D3900018861F822FEF3FEF3A8729871C861B864E
:10D3A00007E216E69E012F5F3F4FAB01BC01C601AD
:10D3B0000E9479A4B60180E393E10E9434C58F8175
:10D3C0009885CFCF4F925F926F927F928F929F926C
:10D3D000BF92CF92DF92EF92FF920F931F93CF9362
:10D3E000DF93CDB7DEB728970FB6F894DEBF0FBE38
:10D3F000CDBF7C016A014901FB0190818CE0989FBF
:10D40000800D1124982FF7012081822F880F820F21
:10D41000880F80936713909368134115510561F14C
:10D42000FA82E9827C836B8301111FC0AE014B5FDE
:10D430005F4FB401C6017CDE6C016D817E818F81FE
:10D4400098856115710581059105B1F060DFF701DF
:10D4500080818F5F8083853148F3CE0101960E94E1
:10D460001062E4CFB12C860129C08A01B12C26C0FC
:10D47000452846284728B1F728960FB6F894DEBF0E
:10D480000FBECDBFDF91CF911F910F91FF90EF9015
:10D49000DF90CF90BF909F908F907F906F905F9024
:10D4A0004F900895B39407C0B1102DC00115110518
:10D4B000C9F20F5F1F4F01151105A9F2AE014B5FB5
:10D4C0005F4FB401C60134DE6C014D805E806F8019
:10D4D00078844114510461047104A9F0F0E24F16FC
:10D4E00051046104710401F3D301C2018D97A109B4
:10D4F000B1090297A105B10530F04BE24416510481
:10D500006104710479F6F7018081482F4B0D55278E
:10D51000551F4631510534F0853020F0CE0101967B
:10D520000E94106281E0411451046104710409F405
:10D5300080E0B80EF70180818B0D8083BB2009F459
:10D5400097CFBA94AE014B5F5F4FB401C801F0DDD5
:10D550008C016D817E818F819885D9DEEFCFCF934D
:10D56000DF93FC0125AD211104C021E025AF0E940D
:10D5700086C3C0913213D0913313E0916113F091BF
:10D58000621382E00995E0916113F091621381E0EA
:10D59000099530E020E044E1BE0180E393E10E9480
:10D5A00081C323E633E147E1BE0180E393E10E94BA
:10D5B00081C3E0916113F091621380E00995DF91DE
:10D5C000CF9108954F925F926F927F928F929F9228
:10D5D000AF92BF92CF92DF92EF92FF921F93CF93C1
:10D5E000DF9300D000D0CDB7DEB70E94F3C16B014E
:10D5F0007C0180915C018F3FC1F10E94F3C180905A
:10D60000530690905406A0905506B090560668199F
:10D6100079098A099B0997FD28C08091041390918C
:10D6200005138F5F8F70891701F1E0915C01E53080
:10D6300008F054C024E0E29FF0011124E55CFD4FA6
:10D6400080819181A281B38189839A83AB83BC83DA
:10D6500020E030E0A901BE016F5F7F4F82E791E0DB
:10D660000E94CDB78FEF80935C010E940C5880918F
:10D670008D0282FF3CC08091620681113AC091E028
:10D6800090936206809192028927809324071092DA
:10D69000920283E08093670110928D020E94F3C191
:10D6A0006C507E4F8F4F9F4F60938E0270938F020E
:10D6B000809390029093910268E873E182E090E099
:10D6C0000E94144216E01150A1F00E94B84162E09D
:10D6D00070E080E090E00E9467C1F5CF8091680122
:10D6E00090916901A0916A01B0916B01ADCF109248
:10D6F000620680915E0690915F06A0916006B091EF
:10D700006106A7019601281B390B4A0B5B0BDA0156
:10D71000C901B7FF05C080919302882309F4B9C1FC
:10D72000D701C6018C599F4FAF4FBF4F80935E0604
:10D7300090935F06A0936006B093610660918C029F
:10D74000062E000C770B77FF03C071956195710968
:10D7500090918C0280915D06981365C0633008F04B
:10D7600062C010928C0280918C0280935D066430BE
:10D7700008F069C0809124078111E7C080912A13C5
:10D7800090912B138159954741F480915D01882335
:10D7900009F4EDC0815080935D010E94F72B8090C9
:10D7A000790790907A07A0907B07B0907C07811151
:10D7B0000E94042CD501C4013AE0B695A79597952F
:10D7C00087953A95D1F7009741E0A407B10520F07D
:10D7D0008FEF9FEFA0E0B0E09695879520916701CD
:10D7E0002111D7C030919302311180C180912A1349
:10D7F00090912B138159954709F45FC18091940250
:10D8000081115BC18091590690915A06A0915B06E7
:10D81000B0915C06C81AD90AEA0AFB0AF7FC5BC198
:10D820000E94904358C1633009F09DCF80918C02D3
:10D8300087FD07C081E0880F880F80938C0264E029
:10D8400092CF8FEFF8CF8091470721E030E040E0A2
:10D8500050E0882309F456C0809043079090440715
:10D86000A0904507B090460781149104A104B1042B
:10D87000E9F170E090E080E00E94C6DB20E030E05B
:10D8800040E85EE30E9427DC2B013C01C701B601A2
:10D89000681979098A099B090E94C6DB9B01AC01C2
:10D8A000C301B2010E9457E320E030E04AE754E4AC
:10D8B0000E9427DC4B015C0120E030E040EA52E4AA
:10D8C0000E9443E424E630E040E050E087FF12C0CD
:10D8D00020E030E040EF51E4C501B4010E9443E490
:10D8E0002AE030E040E050E087FF04C021E030E073
:10D8F00040E050E0C0924307D0924407E0924507D1
:10D90000F0924607A0918C020A2E000CBB0B0E94DD
:10D91000A2E224E030E040E050E00E946BE280911F
:10D920003F0790914007A0914107B0914207820FB5
:10D93000931FA41FB51F80933F0790934007A093A8
:10D940004107B093420710928C02D701C601885656
:10D95000954CAF4FBF4F8093590690935A06A093B2
:10D960005B06B0935C0681E08093670107CF8CE093
:10D9700080935D018091570690915806009729F099
:10D980000197909358068093570681E08093670132
:10D9900004CF009741F04091570650915806481720
:10D9A000590708F023CF80919302811111C02230D2
:10D9B00038F0243008F43FC0243011F4109267018D
:10D9C0008CE293E1CCDD81E080933E07809393026B
:10D9D00083E08CDC81E080935013E0912A13F09176
:10D9E0002B13099510923E0780919302811127C055
:10D9F0001092240780912A1390912B1381599547F7
:10DA000009F0FCCE0E94F3C1DC01CB018C199D0909
:10DA1000AE09BF098090570690905806B12CA12CF2
:10DA200088169906AA06BB0608F0E0CE9093580621
:10DA300080935706DBCE81E080936701C1CF80E3FE
:10DA400093E10E9404C591E0811101C090E09093A0
:10DA50009302882369F280912A1390912B138159A4
:10DA60009547B9F40E94F3C1DC01CB018C199D09E3
:10DA7000AE09BF09C0905706D0905806F12CE12C92
:10DA8000C816D906EA06FB0620F490935806809340
:10DA900057060F900F900F900F90DF91CF911F912D
:10DAA000FF90EF90DF90CF90BF90AF909F908F90BE
:10DAB0007F906F905F904F90089548E9C40E4AE3BD
:10DAC000D41EE11CF11CC0925906D0925A06E09275
:10DAD0005B06F0925C06809193028111DACF80910F
:10DAE00067018130B1F610926701D3CF009709F436
:10DAF0006FCF51CFACE0B0E0E0E8FDE60C94B2E2CD
:10DB0000F0906713E090681320911306211112C062
:10DB100043EF50E26E2D8F2D0E94E5C590E080E02E
:10DB2000F80EF0926713E092681399272C96E8E0BC
:10DB30000C94CEE2C0903413D090351320E333E13F
:10DB40003A8329832F2D30E03C832B832E2D30E028
:10DB50003E832D8318861F827A8769871C861B86E1
:10DB600007E216E69E012F5F3F4F46E252E6BC01F8
:10DB7000C6010E940EA5B60180E393E10E9434C560
:10DB80008F819885CDCFA4E0B0E0E9ECFDE60C9460
:10DB9000AEE27C01062F5A01122F862F660F990BD9
:10DBA0009C01215D3D4F690186E0882E912C111664
:10DBB0000CF03DC0AE014F5F5F4F66E272E6C701F9
:10DBC000B7DA7C0169817A818B819C81611571054D
:10DBD0008105910561F16D3371058105910509F4A8
:10DBE00050C06E3771058105910509F44AC06A324B
:10DBF00071058105910501F507FF11C08AE691E2E3
:10DC00000E3F11F086E691E236E01302B0011124D6
:10DC100071DF66E070E00E9458E2161B60C065E4A8
:10DC200070E080E090E073DB115069F510E0812F27
:10DC30002496ECE00C94CAE26432710581059105EA
:10DC400071F4A114B104D1F0E6E01E02B001112478
:10DC5000C50150DFB4010E9458E2161BA8CF603402
:10DC600071058105910551F41150F6016081062E70
:10DC7000000C770B880B990B4ADB99CF48DB1150CE
:10DC800096CF07FDBBCF61E089819A81AB81BC81D2
:10DC9000CD97A105B10509F460E0600F6A30A4F0EA
:10DCA0001150862F6AE00E9437E2092F682F880FF3
:10DCB000770B605D7F4F072E000C880B990B27DBDD
:10DCC000112309F4B3CF602F062E000C770B605D93
:10DCD0007F4F072E000C880B990B19DB1150112375
:10DCE00009F4A4CF86E01802B0011124C70102DFB5
:10DCF00066E070E00E9458E2161B99CFECE2F3E177
:10DD000083AF64AF6FEF7FEFCA01F4CEACE0B0E059
:10DD1000ECE8FEE60C94B2E2F0906713E090681332
:10DD200020911306211112C043ED50E26E2D8F2D6C
:10DD30000E94E5C590E080E0F80EF0926713E09253
:10DD4000681399272C96E8E00C94CEE2C090341327
:10DD5000D090351320E333E13A8329832F2D30E02F
:10DD60003C832B832E2D30E03E832D8318861F822B
:10DD70007A8769871C861B8607E216E69E012F5F5D
:10DD80003F4F49E252E6BC01C6010E940EA5B60112
:10DD900080E393E10E9434C58F819885CDCF6FEFEA
:10DDA0007FEFB4CFB0E0A0E0E8EDFEE60C94B0E287
:10DDB0005C016B01AFD9E82EC6010E942C62F12CE8
:10DDC00003E110E0081B1109C5E20E151F050CF454
:10DDD000CFE18C2F90E09C012E5F3F4F4091641368
:10DDE0004217130609F08CF509972091661328173E
:10DDF00019065CF140914A0750914B076091490721
:10DE000010926713C093681325E1C501BCDED1E011
:10DE1000C114D104A9F06AE370E080E090E077DA01
:10DE20000E151F05A4F4C45F80916413C81740F059
:10DE3000209166134C2F4950550B241715064CF4AE
:10DE4000CDB7DEB7EAE00C94CCE2D0E0E1CFDD2341
:10DE5000B9F3802F880F080F000F00936713C0934A
:10DE6000681360E270E080E090E051DAC60197DF6D
:10DE7000E7CFACE0B0E0EFE3FFE60C94AEE2982F22
:10DE8000862F6A017901B02E692FF9D9882309F408
:10DE900087C010911306C701002371F13BD9A82E4A
:10DEA0008090341390903513111142C02FEF3FEF43
:10DEB000122F23E12A1940914A0750914B07609194
:10DEC0004907C60160DEAA2009F46AC0B6E08B9F4C
:10DED000600111246AE370E080E090E018DA57E016
:10DEE000C516D10408F442C060E270E080E090E022
:10DEF0000EDAC81AD90AF3CF0E942C62A82E80909D
:10DF0000341390903513112389F2FE0133968AE081
:10DF1000DF011D928A95E9F780E393E19A83898373
:10DF200000E016E69E012F5F3F4F49E252E612C025
:10DF3000FE0133968AE0DF011D928A95E9F780E3BE
:10DF400093E19A83898300E016E69E012F5F3F4F9D
:10DF500046E252E6B701C4010E940EA5B40180E377
:10DF600093E10E9434C52F813885A2CF40914807A4
:10DF7000212F30E0A6E0AA9EC00111242E5F3F4F62
:10DF8000281739070CF49C0180E8821B80936713E3
:10DF900040936813BB2041F06FEF7FEFC701AADD0C
:10DFA0002C96ECE00C94CAE2C701F9DEF9CF0C9490
:10DFB00094A54F925F926F927F928F929F92BF92A1
:10DFC000CF92DF92EF92FF920F931F93CF93DF9345
:10DFD00010920906109208062FE320930C06109267
:10DFE0000B0610920A061092040610920506109273
:10DFF0000606109207069C01F90190812F5F3F4FA2
:10E000009032D1F39E34C9F4818190ED980F9A300B
:10E0100020F08D3211F08B3281F432969F012F5F08
:10E020003F4F808180538A3008F46DC09F012F5F7D
:10E030003F4F8081803209F468C0F0936007E0931D
:10E040005F078F010F5F1F4FC0816AE270E0C80158
:10E050000E94F9E4009731F0FC0131978081803211
:10E06000E1F31182CD3421F0C43511F0C734D9F574
:10E07000F80180810F5F1F4F8032D1F380538A30C7
:10E0800090F5C0930C0690E080E06AE0AF014F5F2E
:10E090005F4F689F9001699F300D1124C901C0979F
:10E0A0002081820F911D27FD9A95FA01208120532E
:10E0B0002A3060F390930B0680930A06DF013196B5
:10E0C0002C912032D9F3CD3461F58E31910539F0A0
:10E0D000F0F48731910519F08C31910511F5B09369
:10E0E0000906A0930806DF91CF911F910F91FF9031
:10E0F000EF90DF90CF90BF909F908F907F906F9028
:10E100005F904F900895F90189CFF9018FCF85373E
:10E11000910538F08737910510F3803A13E09107A5
:10E12000F1F280905F079090600740E050E0BA0104
:10E1300030E020E0C12CD12C7601C394FD01319652
:10E14000DC91DD2309F484C0D132F1F4CD34E1F463
:10E1500080329105C9F440930406509305066093FC
:10E16000060670930706F0930906E093080663E23B
:10E1700070E0CF010E94F9E4009709F4B4CFFC01EC
:10E180001082B1CFDF01DACFD154DA3108F05BC0B1
:10E19000DF011D91103291F0A0EDA10FAA30E8F03F
:10E1A0001E3271F4A181A053AA30B8F021153105B7
:10E1B00019F49F0121503109B12C13C0FD01E8CFA2
:10E1C0001D3211F01B3291F7A181B0EDBA0FBA30B8
:10E1D00020F0AE3259F7A281E6CFBE2EB8183097A4
:10E1E00059F3AD2FB0E02601370104C0440C551C93
:10E1F000661C771CDA95D2F74429552966297729B8
:10E20000A651BA4FBC92A081A154AA3108F4BACF4A
:10E21000DF01D191DD2309F491CF00EDB02EBD0EC9
:10E2200019E01B15A8F713EDB12EBD0E11E01B155B
:10E2300078F7DB3269F3FD013196DC91D03209F0D9
:10E240007DCFDF01F8CF21153105E9F69D01DBCF48
:10E250003093090620930806409304065093050660
:10E2600060930606709307063ECFFC016591759199
:10E270008591949108958F929F92AF92BF92CF9281
:10E28000DF92EF92FF92CF93DF93EC018090B50283
:10E290009090B602A090B702B090B80220E030E0B3
:10E2A000A901C501B4010E94C2DB882309F452C050
:10E2B000C880D980EA80FB80A7019601C501B4011E
:10E2C0000E94C2DB18160CF04AC02091D405309190
:10E2D000D5054091D6055091D705C701B6010E94DA
:10E2E000C2DB882321F1C092D405D092D505E092FB
:10E2F000D605F092D7052091D0053091D1054091F7
:10E30000D2055091D305C701B6010E9427DC9B01BD
:10E31000AC0160E070E080E89FE30E94DFE2609380
:10E32000490170934A0180934B0190934C01609195
:10E33000490170914A0180914B0190914C01DF910C
:10E34000CF91FF90EF90DF90CF90BF90AF909F90D4
:10E350008F90089560E070E080E89FE3F0CF60E088
:10E3600070E0CB01ECCF682F70E090E080E00C947F
:10E3700037A5B0E0A0E0EFEBF1E70C94AAE2EC01E6
:10E380002091AD023091AE024091AF025091B002A7
:10E39000688179818A819B810E94DFE24B015C0167
:10E3A0002091B1023091B2024091B3025091B40277
:10E3B0006C817D818E819F810E94DFE26B017C01F7
:10E3C000A501940160914101709142018091430146
:10E3D000909144010E94C2DB882309F454C08092CA
:10E3E000410190924201A0924301B09244012091D8
:10E3F000C8053091C9054091CA055091CB05C501AA
:10E40000B4010E9427DC2B013C010E94F0E34B0188
:10E410005C0120E030E040EA50E40E94C2DB1816C4
:10E4200034F4812C912CC0EAAC2EC0E4BC2E20E048
:10E4300030E0A901C501B4010E9443E487FF03C095
:10E44000812C912C5401A5019401C301B2010E94B9
:10E45000DFE26093C0057093C1058093C20590937D
:10E46000C305C501B4010E94BFE36093BE05062E3B
:10E47000000C770B6F5F7F4F6630710514F066E01C
:10E4800070E06093BC05D0913F011091BE05A701DB
:10E4900096016091450170914601809147019091EC
:10E4A00048010E94C2DB811123C0D11375C02091A5
:10E4B000A4053091A5054091A6055091A70560914E
:10E4C000C0057091C1058091C2059091C3050E945D
:10E4D00027DC2091A8053091A9054091AA0550910B
:10E4E000AB050E94E0E2CDB7DEB7E0E10C94C6E2F6
:10E4F000C0924501D0924601E0924701F092480156
:10E500002091CC053091CD054091CE055091CF059D
:10E51000C701B6010E9427DC4B015C010E94F0E3B9
:10E520006B017C0120E030E040EA50E40E94C2DB55
:10E53000181634F4C12CD12CB0EAEB2EB0E4FB2E2B
:10E5400020E030E0A901C701B6010E9443E487FF43
:10E5500003C0C12CD12C7601A7019601C501B401DD
:10E560000E94DFE26093C4057093C5058093C605E1
:10E570009093C705C701B6010E94BFE36093BF0532
:10E58000062E000C770B6F5F7F4F6630710514F01D
:10E5900066E070E06093BD05C091BF05D11305C072
:10E5A000809140018C1709F470C08091BE05909154
:10E5B000BF059093400180933F010C2E000CDD0BB2
:10E5C00027E01203C0011124FC01EC0FFD1FEE0F28
:10E5D000FF1FEE0FFF1FE653FD4F20813181428167
:10E5E00053812093B8053093B9054093BA055093F1
:10E5F000BB050091BD05002E000C110BFC01E00FC6
:10E60000F11FEE0FFF1FEE0FFF1FE653FD4F60815E
:10E610007181828193810E94DFE26093B4057093DF
:10E62000B5058093B6059093B7052091BC0537E0FA
:10E630002303F0011124CE0FDF1FCC0FDD1FCC0F01
:10E64000DD1FC653DD4F288139814A815B812093CC
:10E65000B0053093B1054093B2055093B305E00F78
:10E66000F11FEE0FFF1FEE0FFF1FE653FD4F6081FE
:10E670007181828193810E94DFE26093AC05709387
:10E68000AD058093AE059093AF058090C405909042
:10E69000C505A090C605B090C7052091B40530917E
:10E6A000B5054091B6055091B705C501B4010E946A
:10E6B00027DC2091B8053091B9054091BA055091F9
:10E6C000BB050E94E0E26B017C01C092A805D092DC
:10E6D000A905E092AA05F092AB052091AC05309116
:10E6E000AD054091AE055091AF05C501B4010E9442
:10E6F00027DC2091B0053091B1054091B2055091D1
:10E70000B3050E94E0E2A70196010E94DFE2609358
:10E71000A4057093A5058093A6059093A705C7CE81
:10E72000ACE0B0E0E6E9F3E70C94B7E2182F8823F9
:10E7300079F020E030E0A9016091BA027091BB024B
:10E740008091BC029091BD020E94C2DB8823F1F04F
:10E750008091B9028117D1F00E9423298CE0E3E275
:10E76000F2E0DE01119601900D928A95E1F7CE015B
:10E770000196FFDD8091B902882361F082E791E084
:10E780000E9479291092B9020E94363C2C96E3E04F
:10E790000C94D3E281E08093B90282E791E00E9479
:10E7A0004529F2CFCF92DF92EF92FF9280E0B8DF5F
:10E7B0001092B1021092B2021092B3021092B402FF
:10E7C0001092AD021092AE021092AF021092B002FF
:10E7D0001092BE021092BF021092C0021092C102AB
:10E7E0001092BA021092BB021092BC021092BD02AB
:10E7F0004AEC52E027E0C12CD12C60ECE62E6FE70A
:10E80000F62E90E080E0FC01EE0FFF1FEE0FFF1FE1
:10E81000E40FF51FC082D182E282F3820196873035
:10E82000910589F72150445E5F4F2111EACFFF9097
:10E83000EF90DF90CF9008954F925F926F927F920A
:10E840008F929F92AF92BF92CF92DF92EF92FF9200
:10E850001F93CF93DF93EC01162F2091B5023091D7
:10E86000B6024091B7025091B802688179818A81DD
:10E870009B810E94C2DB882309F497C0B090B90243
:10E8800080E04EDFC880D980EA80FB8020E030E065
:10E89000A901C701B6010E9443E487FF03C0C12C50
:10E8A000D12C7601C092B502D092B602E092B702A6
:10E8B000F092B8022DEB37E346E855EBC701B601FD
:10E8C0000E94C2DB87FD0BC02DEB37E346E855E322
:10E8D000C701B6010E9443E418160CF076C0A701E8
:10E8E000960160E070E080E89FE30E9457E3609348
:10E8F000D0057093D1058093D2059093D30580EF16
:10E900009FEFA9E7B4EC8093D4059093D505A0932D
:10E91000D605B093D705BB2009F447C040907201DB
:10E920005090730160907401709075018090760131
:10E9300090907701A0907801B0907901C0907A0111
:10E94000D0907B01E0907C01F0907D0181E0E8DED9
:10E95000112359F1A3019201609172017091730129
:10E9600080917401909175010E94C2DB81111BC0DE
:10E97000A5019401609176017091770180917801F1
:10E98000909179010E94C2DB81110DC020917A0122
:10E9900030917B0140917C0150917D01C701B6010E
:10E9A0000E94C2DB81110E945C3CDF91CF911F91DC
:10E9B000FF90EF90DF90CF90BF90AF909F908F909F
:10E9C0007F906F905F904F90089560E070E0CB0172
:10E9D0008ECF8F929F92AF92BF92CF92DF92EF92A3
:10E9E000FF92C090BA02D090BB02E090BC02F090BF
:10E9F000BD0220E030E0A901C701B6010E94C2DBE0
:10EA00008823E1F1A701960160E070E080E89FE3D0
:10EA10000E9457E36B017C018090BE029090BF0280
:10EA2000A090C002B090C10220E030E0A901C50171
:10EA3000B4010E94C2DB882329F1A501940160E0A2
:10EA400070E080E89FE30E9457E3C092C805D0922F
:10EA5000C905E092CA05F092CB056093CC0570938E
:10EA6000CD058093CE059093CF05FF90EF90DF907A
:10EA7000CF90BF90AF909F908F900895C12CD12CD4
:10EA80007601CACF60E070E0CB01DFCFCF92DF929A
:10EA9000EF92FF926B017C0183E3C816D104E1047D
:10EAA000F10470F082E3C81AD108E108F10862E3CA
:10EAB00070E080E090E00E9467C10E94FA25ECCFF0
:10EAC000C701B6010E9467C10E94FA25FF90EF902E
:10EAD000DF90CF900895BC0190E080E00C9437A5C2
:10EAE00080915D07813069F09091821492FB8827B4
:10EAF00080F992FF07C097FB882780F991E089276A
:10EB0000089581E008959091821494FB882780F9FC
:10EB100094FF06C081E090919C12911101C080E0A9
:10EB20000895ACE0B0E0E7E9F5E70C94AAE21092B2
:10EB300047078091240710922407882361F020E082
:10EB400040E070E060E08EEA95E50E9454422C9629
:10EB5000E0E10C94C6E22091100130911101409146
:10EB60003F0750914007CA01820F931F2436310599
:10EB700009F0E9C34730510544F006978A30910502
:10EB80000CF0F0C38AE090E0F7C306964A3F5F4F6F
:10EB9000ACF380913E07882309F4D0C160918812BC
:10EBA00070918912072E000C880B990B0E94C8DB0C
:10EBB00011E020918412309185124091861250917B
:10EBC00087120E9443E418160CF010E010935206CE
:10EBD00080907A0190907B01A0907C01B0907D01A3
:10EBE00020E030E0A901C501B4010E94C2DBC12CC4
:10EBF000D12CE0EAEE2EE0ECFE2E87FD06C0C12C03
:10EC0000D12C70EAE72E70E4F72E20E030E04AE7DE
:10EC100054E4C501B4010E9427DCA70196010E94BB
:10EC2000E0E22DEC3CEC4CEC5DE30E9427DC0E9422
:10EC3000BFE36B017C0180E2F7FE09C0F094E09431
:10EC4000D094C094C11CD11CE11CF11C8DE24090F9
:10EC50007201509073016090740170907501209161
:10EC6000760130917701409178015091790129879F
:10EC70003A874B875C878093950260E230E1C31648
:10EC800037E2D306E104F1048CF0C701B60120E1BC
:10EC900037E240E050E00E946BE2CA01B9012AE08D
:10ECA00030E040E050E00E946BE2605D60939602CD
:10ECB00060E248EEC41643E0D406E104F1048CF0AF
:10ECC000C701B60128EE33E040E050E00E946BE25D
:10ECD000CA01B9012AE030E040E050E00E946BE256
:10ECE000605D60939702C701B60124E630E040E022
:10ECF00050E00E946BE26AE0862E912CA12CB12C90
:10ED0000CA01B901A50194010E946BE2605D6093A4
:10ED10009802C701B601A50194010E946BE26B0144
:10ED2000CA01B901A50194010E946BE2CC2009F44B
:10ED300033C32EE220939902605D60939A0250E300
:10ED4000C50EC0929B0265E972E08AE496E00E94DB
:10ED500004E520E030E0A901C301B2010E94C2DB5A
:10ED600020E030E040E05FEB87FD04C020E030E0D1
:10ED700040E05FE3C301B2010E94E0E20E94BFE312
:10ED8000CB010E949840BC0185E496E00E9404E516
:10ED900020E030E0A90169857A858B859C850E94F9
:10EDA000C2DB20E030E040E05FEB87FD04C020E004
:10EDB00030E040E05FE369857A858B859C850E9421
:10EDC000E0E20E94BFE3CB010E949840BC0180E4D6
:10EDD00096E00E9404E58091821400E117E283FD31
:10EDE00028C091DE882309F4E9C280917A149091B9
:10EDF0007B14A0917C14B0917D140097A105B105FE
:10EE000009F4DCC2BC01CD01615F784D8F4F9F4F8B
:10EE100020E137E240E050E00E94F0E160917E1492
:10EE200070917F1480918014909181140E94F0E180
:10EE300089010E94EE3F4B015C018D829E82AF8270
:10EE4000B886D62E80915B018017C1F100935B01DB
:10EE5000C80164E670E00E9444E27B0188E48E9D74
:10EE6000B0018F9D700D112490E080E00E94C6DB00
:10EE70002AE037ED43E25CE30E9427DC0E94C4E312
:10EE800060933F060115110509F09BC210923A06E6
:10EE90001092300680E880932F068AE396E0FC010A
:10EEA00001900020E9F7CF018A539640982F990FDF
:10EEB000890F880F90E8981B90932E0680915A0135
:10EEC000D816E1F180925A0141E08D819E81AF8197
:10EED000B88580389145A140B10508F440E06EE165
:10EEE00076E0CE0105960E949D66982F990F990FA6
:10EEF000891B880F805880931D06282D2370822E31
:10EF0000E9F401151105A9F0A0E1B7E2A01BB10BCE
:10EF10002D813E814F8158850E9412E2980150E078
:10EF200040E00E94F0E1211531054105510509F04D
:10EF30006EC21092300680E880932F060E94F3C1C3
:10EF400000911606109117062091180630911906A7
:10EF50006B017C01C01AD10AE20AF30A970186010B
:10EF600037FD11C0209115062095209315066A548F
:10EF70007C4F8F4F9F4F60931606709317068093B8
:10EF8000180690931906D090150611E0D11001C013
:10EF900010E081E00E94766980916413873180F4EB
:10EFA00080916613843060F037E2E32E32E2F32E74
:10EFB00003E126E044E069E080E393E10E940AC6B1
:10EFC000809164138431B8F480916613823098F094
:10EFD000DD2009F435C280917D07882309F430C211
:10EFE00081EF91E27C0102E123E042E068E680E308
:10EFF00093E10E940AC6809164138C3108F06EC0C0
:10F000004090841250908512609086127090871202
:10F01000A0908812B0908912843198F48091661380
:10F02000883078F08091520680FF0DC283EA91E229
:10F030007C010CE022E048E064E480E393E10E947C
:10F040000AC680916413883040F4B7FEFFC147E8D8
:10F0500051E267E082E40E947E6E809164138C31FD
:10F06000B0F480916613843190F020E030E040E00D
:10F070005FE3C301B2010E94E0E20E94BFE377FFB9
:10F080000EC247E851E26CE182E40E947E6E8091FC
:10F0900064138C3118F5809166138431F8F08091F7
:10F0A0007D078823D9F024E6829FC001112481586E
:10F0B0009F4F6FEF70E00E9458E2CB010E94174112
:10F0C00027E6209367132CE1209368130E94CF6EEC
:10F0D00065E270E080E090E00E94876914DD88239B
:10F0E00079F180916413843358F5809166138A32E4
:10F0F00038F107E028E04AE26AE280E393E10E9407
:10F10000B1C405E022E04CE262E380E393E10E94B7
:10F11000B1C424E04AE061E38AE20E9481C46091C4
:10F1200032137091331382E380934C138BE28093FC
:10F130004D132CE433E142E380E393E10E9481C369
:10F1400080916413853350F480916613813330F0DD
:10F1500024E04AE461E386E30E9481C48091641361
:10F16000843368F480916613823348F002E0209182
:10F170003F0642E367E380E393E10E94B1C48091DC
:10F180006413803358F580916613883238F180918A
:10F190001C06811751F080911B0610931C068F5F8F
:10F1A000833008F0A5C180931B0680911B06811156
:10F1B000A2C180913A06882389F080912E0680931F
:10F1C000671380E3809368138AE396E00E94CF6E12
:10F1D00065E270E080E090E00E94876980916413AE
:10F1E000883208F05DC0809166138D3108F458C0F4
:10F1F0002BE040E86DE180E00E9481C480916413BF
:10F20000873208F04DC0809166138F3108F448C0F2
:10F2100083E08093671306E20093681368E570E06B
:10F2200080E090E00E9487698BE0809367130093F1
:10F230006813DD2009F491C185E496E00E94CF6E49
:10F2400088E28093671306E20093681369E570E033
:10F2500080E090E00E94876980E3809367130093C9
:10F260006813DD2009F49EC180E496E00E94CF6E11
:10F270008DE48093671306E2009368136AE570E0FB
:10F2800080E090E00E94876985E580936713009392
:10F290006813DD2009F4ABC18AE496E00E94CF6ECA
:10F2A00080916413833348F5809166138B3228F183
:10F2B00083E00E94766983E08093671303E3009301
:10F2C000681366E070E080E090E00E94876981E06A
:10F2D0000E94766980911001909111010E9417415E
:10F2E0002CE020936713009368130E94CF6E65E2B1
:10F2F00070E080E090E00E9487698091641381341F
:10F3000008F025CC80916613863308F420CC109247
:10F3100067138EE38093681385E190E10E942C626D
:10F32000082F863108F088C185E190E10E94CF6EF8
:10F33000053109F40CCC60E270E080E090E00E94BE
:10F3400087690F5FF5CF243631054CF4853691057A
:10F3500004F58A30910534F48AE090E009C08436DF
:10F360009105BCF0883EE3E09E0714F087EE93E041
:10F370002817390709F40DCC9093110180931001DF
:10F3800010923F07109240071092410710924207D7
:10F3900000CC84E690E0F0CF662351F02EE220937B
:10F3A0009902605D60939A0280E280939B02CBCCCD
:10F3B00080E280939A0280939902F6CF10E000E0F9
:10F3C00038CD2E2D80E2243628F08E2D64E60E9462
:10F3D0002BE2805D8093990290E22A3040F03AE07F
:10F3E000822F632F0E942BE20E942BE2905D90936C
:10F3F0009A02822F6AE00E942BE2905D90939B021A
:10F4000069E972E08AE396E00E9404E546CD29832B
:10F410003A834B835C8381E020383145414051057C
:10F4200008F480E0482F60E376E0CE0101960E9468
:10F430009D66982F990F990F891B880F80587CCD56
:10F440008BEB91E2CFCD8BE891E2F2CDC5010E942A
:10F450001741FC01808193E0803229F4818192E0A0
:10F46000803209F491E0892F880F880FE92EE81A7D
:10F470008E2D855B8093671387E08093681323E06C
:10F4800030E0291B3109CF01820F931F0E94CF6EFC
:10F4900069E070E080E090E00E948769DECDCB01FA
:10F4A0000E941741FC01808193E0803229F4818120
:10F4B00092E0803209F491E0892F880F880FF92EAD
:10F4C000F81A8F2D855B809367138CE18093681306
:10F4D00023E030E0291B3109CF01820F931F0E94E6
:10F4E000CF6E69E070E080E090E00E948769CFCD48
:10F4F00010921B065ACE8230B1F4809130068823D8
:10F5000091F044E851E260E386E30E947E6E8091D0
:10F510002F068093671380E38093681380E396E05F
:10F520000E94CF6E5BCE80911E06882309F456CED2
:10F5300086E38093671300E3009368136FEF7FEF18
:10F5400081E891E20E947A6D80911D068093671395
:10F55000009368138EE196E0E3CF87E00E945F3767
:10F5600080FF15C025E4E22E26E0F22EF70161911E
:10F570007F01662309F464CE6F320CF06FE3062E30
:10F58000000C770B880B990B0E948769EFCF809155
:10F590004D0780FD51CE6FEF7FEF8CE791E20E9427
:10F5A0007A6D4ECE87E00E945F3781FF15C090E4F0
:10F5B000E92E96E0F92EF70161917F01662309F4A7
:10F5C00057CE6F320CF06FE3062E000C770B880BD2
:10F5D000990B0E948769EFCF80914D0781FD44CE42
:10F5E0006FEF7FEF8CE791E20E947A6D41CE87E06A
:10F5F0000E945F3782FF15C08AE4E82E86E0F82E6D
:10F60000F70161917F01662309F44ACE6F320CF055
:10F610006FE3062E000C770B880B990B0E9487690D
:10F62000EFCF80914D0782FD37CE6FEF7FEF84E7FC
:10F6300091E20E947A6D34CE80911A061817B1F0CB
:10F640000091141010931A0685E190E10E942C623B
:10F65000081708F050C00F5FE02FF0E0EB5EFF4EA0
:10F660008081807C8038B9F300931410E0901410EE
:10F67000F12C97012B5E3F4E7901C9010E942C624B
:10F68000182F60E870E0C7010E94866E153108F0FF
:10F690005ECA60E270E080E090E00E948769143109
:10F6A00009F455CA60E270E080E090E00E9487694A
:10F6B000133109F44CCA60E270E080E090E00E94EF
:10F6C0008769123109F443CA212F30E02E5F3F4F82
:10F6D0004AEF4203B001439F700D112460587F4FE1
:10F6E00085E190E10E94866E60E270E080E090E04B
:10F6F0000E9487692CCA10921410B8CF80915D07C0
:10F70000823059F000DA882349F08091821482FB1C
:10F71000882780F991E08927089581E0089581E0A4
:10F7200008959091C00095FFFCCF8093C600089586
:10F73000CF93DF93EC018991882311F0F2DFFBCFA7
:10F74000DF91CF910895CF93DF93EC0189918823C6
:10F7500011F0E7DFFBCF8DE0E4DF8AE0E2DFDF914D
:10F76000CF910895CF93DF93EC01FE018491219610
:10F77000882311F0D6DFF9CFDF91CF910895CF9391
:10F78000DF93EB01EFDFCE01D3DFDF91CF9108955F
:10F790000F931F93CF938C01C62F80EF9EE1E2DF82
:10F7A000C801E0DF8AE3BDDF80E38C0FBADF8AE0C7
:10F7B000B8DFCF911F910F910895CF92DF92EF9212
:10F7C000FF926A017B01CEDF42E0C701B6010E94D1
:10F7D000DEA7FF90EF90DF90CF900895CF93DF9357
:10F7E00061E07FE10E9422B8C091FF12D091001326
:10F7F000488159816A817B8188EF9EE1DEDF4C81FF
:10F800005D816E817F818BEC9CE2D7DF4091FB12A2
:10F810005091FC126091FD127091FE1288EC9CE2F6
:10F82000CCDF85EF9EE19EDF87E19BE09BDF8AE0F6
:10F8300078DFDF91CF910895C0DF8AE072CFAEE428
:10F84000B0E0E5E2FCE70C94A8E270E060E085E45B
:10F850000E949B679AA789A781117CC26EEB70E01A
:10F8600083E50E949B673C0165E070E083E40E94B1
:10F870009B678C0160E085E50E9487678DAF60E043
:10F8800086EC90E20E9494520E94F3C169877A87C5
:10F890008B879C8780916401909165010E97681613
:10F8A000790654F087E790E25DDF0E94B9B8C25B49
:10F8B000DF4FE2E10C94C4E229853A854B855C85F3
:10F8C000205E314B4F4F5F4F2BAB3CAB4DAB5EAB34
:10F8D00083E690E247DF0E9456258FE780938A12E5
:10F8E00081E08093660160E08FE490E20E94945290
:10F8F00089859A85AB85BC85898B9A8BAB8BBC8BB4
:10F900008BA79CA7ADA7BEA7198E1A8E1B8E1C8E27
:10F9100019A21AA21BA21CA219821A821B821C8283
:10F920002FE730E040E050E02D873E874F87588B2F
:10F9300080E090E4ACE1B6E48D839E83AF83B8872A
:10F940001D8A1E8A1F8A188EFFE7CF2ED12CE12C2C
:10F95000F12C2F961FAE2F971FA618AA19AA1AAA24
:10F960001DA21EA21FA218A691E09FAB312C212C34
:10F97000812C912C54019301072C000C440B550B46
:10F9800022962CAF3DAF4EAF5FAF2297402F002E97
:10F99000000C550B5CAF4BAFC3014E969C01092E7A
:10F9A000000C440B550B26962CAF3DAF4EAF5FAF0E
:10F9B0002697CC979C01990F440B550B2A962CAF98
:10F9C0003DAF4EAF5FAF2A9736E0631A7108C301AF
:10F9D000072C000CAA0BBB0B2E968CAF9DAFAEAFC5
:10F9E000BFAF2E9780916601882309F48DC00E94D5
:10F9F000F3C12B013C0110919903112309F473C049
:10FA00000E94C125109299038090841290908512D3
:10FA1000A0908612B0908712A50194016D897E890D
:10FA20008F89988D0E9443E487FF04C08D8A9E8A47
:10FA3000AF8AB88EA50194016D817E818F819885F2
:10FA40000E94C2DB181624F48D829E82AF82B88693
:10FA500022966CAD7DAD8EAD9FAD22970E94C8DB26
:10FA60006D8F7E8F8F8F98A39FA92D8D3E8D4F8D8B
:10FA700058A1992309F472C1C501B4010E9443E45D
:10FA800018168CF5D301C20129893A894B895C8902
:10FA9000821B930BA40BB50BAC01BD01485853411D
:10FAA0006109710977FD1FC04D855E856F85788975
:10FAB0004C195D096E097F097595679557954795AE
:10FAC00040938A128DA39EA3AFA3B8A78D8D9E8D60
:10FAD000AF8DB8A18D8B9E8BAF8BB88F49865A8620
:10FAE0006B867C861FAA26966CAD7DAD8EAD9FADD4
:10FAF00026970E94C8DBA50194010E94C2DB87FF04
:10FB000021C088EC9FE12EDE109266010E945625EE
:10FB1000CCCE4BEEC42ED12CE12CF12C76C124E1BD
:10FB200030E040E050E02D873E874F87588B34E12E
:10FB3000C32ED12CE12CF12C76C1CD86DE86EF864A
:10FB4000F88A71C1D301C2012BA53CA54DA55EA5C4
:10FB5000821B930BA40BB50BB7FD47C089A50E9470
:10FB6000CB248AE0DEDDD301C2018053984FAF4F32
:10FB7000BF4F8BA79CA7ADA7BEA72F969FAD2F9772
:10FB800091116FC02FA538A949A95AA9C501B4017F
:10FB90000E9443E418160CF050C020E030E040E032
:10FBA00050E4C501B4010E94E0E26FA778AB89ABD5
:10FBB0009AABA3019201205E314B4F4F5F4F2BABAD
:10FBC0003CAB4DAB5EAB2E966CAD7DAD8EAD9FADBF
:10FBD0002E970E94C8DBA50194010E94C2DB881FFA
:10FBE0008827881F2F968FAF2F9789859A85AB8599
:10FBF000BC858D8F9E8FAF8FB8A329893A894B8999
:10FC00005C89281739074A075B0720F42D8F3E8F40
:10FC10004F8F58A38D8D9E8DAF8DB8A1481A590A6C
:10FC20006A0A7B0A91E849169FE4590692E169063F
:10FC3000710460F18AEA9FE166CFD301C2012BA96A
:10FC40003CA94DA95EA9821B930BA40BB50B4DE0FB
:10FC500054E16CE174E1B7FDC8CF80E00E946525F6
:10FC6000C4CF2A966CAD7DAD8EAD9FAD2A970E9414
:10FC7000C8DB9B01AC01C501B4010E94C2DB87FF58
:10FC8000B4CF4CE25EE26CE37EE2E7CFABADBCAD5D
:10FC9000A215B3050CF05BC0B3E02B1631040CF4D5
:10FCA00056C08DE49FE15EDD80E39FE15BDD49812D
:10FCB0005A816B817C8189E49FE1BEDD80E39FE115
:10FCC00051DD49A15AA16BA17CA185E49FE1B4DD7E
:10FCD00080E39FE147DD498D5A8D6B8D7C8D81E4FA
:10FCE0009FE1AADD2DAD222309F4DFCD89819A8120
:10FCF000AB81BC8180938B1290938C12A0938D1258
:10FD0000B0938E122CEA35EC47E25EE369A17AA14A
:10FD10008BA19CA10E9427DC60938F12709390129C
:10FD2000809391129093921220E030E543EC50E4DE
:10FD3000698D7A8D8B8D9C8D0E9427DC6093931248
:10FD4000709394128093951290939612AECD0E9468
:10FD5000E26A48CE82EA90E205DDA9CDC501B40190
:10FD60000E94C2DB87FFBFCED301C20129853A853D
:10FD70004B855C85821B930BA40BB50BAC01BD01BD
:10FD8000485853416109710977FDADCE2114310402
:10FD900009F4FCC02DA13EA14FA158A5280F391F81
:10FDA0004A1F5B1F298B3A8B4B8B5C8B2DA13EA18D
:10FDB0004FA158A5281B390B4A0B5B0BC701B60195
:10FDC0000E94E1E129893A894B895C890E946BE2B2
:10FDD000CD84DE84EF84F888C20ED31EE41EF51EA7
:10FDE00034E1C316D104E104F1040CF498CE4CEED6
:10FDF000C416D104E104F1040CF08BCE50E8C51612
:10FE0000D104E104F1040CF498CECD86DE86EF86B1
:10FE1000F88A8EEF90E0A0E0B0E08C199D09AE0961
:10FE2000BF096C017D0187E490E29CDC6D857E85D5
:10FE30008F8598890E94D76F82E490E293DCC70196
:10FE4000B6010E94D76F4D815E816F8178858BE30B
:10FE500090E2B3DC4D895E896F89788D84E390E20E
:10FE6000ACDC33E0231631040CF490C0C701B601BA
:10FE70000E94C8DB20E030E040E850E40E9427DC2C
:10FE800069837A838B839C832D813E814F81588542
:10FE90006D897E898F89988D0E94DFE22BED3FE08E
:10FEA00049EC5FE30E9427DC9B01AC0169817A8108
:10FEB0008B819C810E9457E36FAB78AF89AF9AAF7B
:10FEC00069897A898B899C890E94C8DB2FE632E197
:10FED00043E85AE30E9427DC6D837E838F839887F3
:10FEE0002AE939E949E15FE36FA978AD89AD9AADB7
:10FEF0000E9427DC69837A838B839C839B01AC01FE
:10FF00000E94E0E22D813E814F8158850E9457E397
:10FF100069A37AA38BA39CA320E030E040E05EE3DA
:10FF20006D817E818F8198850E9427DC29813A81AD
:10FF30004B815C810E9427DC698F7A8F8B8F9C8F2D
:10FF40004FA958AD69AD7AAD8EE290E236DC4D81B5
:10FF50005E816F81788588E290E26EDC89E190E2D3
:10FF600001DC49815A816B817C8183E190E225DC4F
:10FF700049A15AA16BA17CA18DE090E21EDC498DC4
:10FF80005A8D6B8D7C8D87E090E256DC8D859E8549
:10FF9000AF85B8898C0D9D1DAE1DBF1DB595A7956C
:10FFA0009795879580938A124CAD4F930F933F920C
:10FFB0002F9283EF9FE19F938F932EEF3FE13F932B
:10FFC0002F931F920E9477525FEF251A350A0FB6C2
:10FFD000F894DEBF0FBECDBF2D8D3E8D4F8D58A145
:10FFE0002D833E834F835887498A5A8A6B8A7C8A3D
:10FFF0001FAB79CD63E678E10E9422B860914F0D86
:020000021000EC
:100000007091500D8091510D9091520D0E94C6DB60
:10001000AB01BC018AE598E1D0DB40917F0D5091A6
:10002000800D6091810D7091820D87E598E1C5DBAF
:100030004091830D5091840D6091850D7091860DD6
:1000400084E598E1BADB40916107509162076091C5
:1000500063077091640781E598E1EECBCF93DF935E
:1000600067E078E10E9422B8CFE3DDE04CA95DA90A
:100070006EA97FA98EEF97E1A0DB48AD59AD6AADBF
:100080007BAD8BEF97E199DB4CAD5DAD6EAD7FAD98
:1000900084E598E1D1DBDF91CF910895CF93DF9391
:1000A00063EE77E10E9422B8CFE3DDE04CA15DA1D1
:1000B0006EA17FA18AED97E180DB48A559A56AA5CD
:1000C0007BA58BEC9CE279DB4CA55DA56EA57FA59D
:1000D00088EC9CE272DB48A959A96AA97BA985EC46
:1000E0009CE2AADBDF91CF910895CF93DF936EEB73
:1000F00077E10E9422B8CFE3DDE0688179818A81CF
:100100009B810E94C6DBAB01BC0185EB97E155DB0F
:100110006C817D818E819F810E94C6DBAB01BC0119
:100120008BEC9CE24ADB688579858A859B850E94F9
:10013000C6DBAB01BC0188EC9CE23FDB6C857D85B6
:100140008E859F850E94C6DBAB01BC0185EC9CE2DD
:1001500073DBDF91CF9108958F929F92AF92BF9200
:10016000EF92FF920F931F93CF93DF9386EE96E16A
:10017000F9DAC0E0D7E0D15019F080E2D2DAFBCF53
:100180008C2F0E94B371CF5FC730A1F78AE0C9DA24
:100190000AEC12E0C0E080E2C4DA8C2F0E94B37156
:1001A0007801D7E080E2BDDAF70180809180A280FB
:1001B000B38020E030E0A901C501B4010E9443E40E
:1001C00087FD02C08BE2ADDA43E0C501B4010E94B5
:1001D000DEA7D150FCE1EF0EF11CD111E3CF8AE094
:1001E000A0DACF5F0C5F1F4FC730A9F68AE099DA1B
:1001F000DF91CF911F910F91FF90EF90BF90AF9043
:100200009F908F900895811105C08FED96E1AADA35
:100210008AE087CA83EE96E1FACF88ED96E1A2CA1A
:1002200082ED96E19FCACF9384E50E948763C0E088
:100230008823D9F00E945D67C82F1816B4F4F0DF48
:100240008DE46FDA80910A0690910B060E946B751F
:1002500080EF98E187DA6C2FCC0F770B880B990B26
:100260000E9494A58AE05DDACFEF8C2FCF9108959C
:10027000CF93C82F67EC78E10E940BB8C11101C081
:10028000CFDF40918B1250918C1260918D12709142
:100290008E128EEB98E191DA20E030E543EC50E4E9
:1002A00060918F12709190128091911290919212A0
:1002B0000E9427DCAB01BC018BEB98E17EDA2CEAD3
:1002C00035EC47E25EE36091931270919412809155
:1002D0009512909196120E9427DCAB01BC0188EB2D
:1002E00098E16BDA8AE01DDACF910895CF93DF931E
:1002F000EB0138DABE01DD0F880B990B0E9494A543
:10030000DF91CF910895EC018B01F42E0E945625C8
:10031000209709F479C084DFCE0124DA8AE001DA7B
:100320000115110511F406E01CE20E9418681F93E4
:100330000F93DF93CF9382EA96E19F938F9381E0AF
:100340008F930E9477520E949043C0913113C695BB
:10035000C6958CE293E10E94AF6ADC2FDD0F1D2F62
:100360001C0F8DB79EB707960FB6F8949EBF0FBEB1
:100370008DBF83E00E94766910926713C093681363
:1003800085E190E10E94CF6E10926713D0936813BD
:100390006FEF7FEF83E996E10E947A6D1092671309
:1003A000109368136FEF7FEF86E896E10E947A6DF5
:1003B00080E393E10E9404C58111DBCF2EDF82EB45
:1003C00096E1D0D989EE93E0019739F000C00000A2
:1003D000EEE5F9E03197F0F7F7CFF89489EE93E086
:1003E000019739F000C00000E6EEF3E03197F0F736
:1003F000F7CF0E945625FF2021F00E94BD27A89527
:10040000FECF0E947827FBCF0115110511F406E0FD
:100410001CE2C9EAD6E189CF8091890D90918A0DBD
:100420002FEF3FEF981751F0E92FF0E0E757F24F29
:10043000228130E09F5F9F7790938A0DC9010895D4
:100440001F920F920FB60F9211240F900FBE0F90B4
:100450001F9018951F920F920FB60F9211240BB692
:100460000F922F938F939F93EF93FF939091C600DA
:1004700020918A0DE091890D81E08E0F8F772817EA
:1004800029F0F0E0E757F24F9283E82FE093890DCF
:10049000FF91EF919F918F912F910F900BBE0F9035
:1004A0000FBE0F901F9018958EBD0DB407FEFDCFA7
:1004B00008958FEF8EBD0DB407FEFDCF8EB5089564
:1004C000909164009B7F90936400982F906A96951A
:1004D0009CBD80FD03C091E0863009F490E09DBD95
:1004E0000895A8E0B0E0E7E7F2E80C94A8E2B82E9F
:1004F0008091720E843008F0F4C131E6D32E8091E1
:10050000720E843008F01FC18091890D90918A0D80
:10051000891B8F7709F417C17FDF97FF09C07DDE44
:1005200082ED95E11FD98091890D80938A0DE7CFE7
:100530008A3019F08D3009F0FDC01092710E809153
:100540000F0E9091100EFC01E55FF14F1682892B82
:1005500019F40E94FA25D3CF1092100E10920F0EAC
:1005600001E11EE0F8018191803209F446C08E3429
:1005700009F09CC06DEC75E1C8010E9441DB7C0173
:10058000892B41F06EE470E0C80104960E94F9E402
:10059000009709F4C8014AE050E070E060E001967D
:1005A0000E94B6D82B013C0180910B0E90910C0E4D
:1005B000A0910D0EB0910E0E0196A11DB11D481611
:1005C00059066A067B0629F060E08AE995E1EF2882
:1005D00051F16AE270E0C8010E9428E59C01009791
:1005E00029F1982F901BF12C992349F09150F80193
:1005F000E90FF11D8081F826F7CF8F01B3CF4AE0D4
:1006000050E070E060E0C90101960E94B6D82F2D3D
:1006100030E050E040E0621773078407950751F01F
:1006200060E08BE795E10E949EB769CF60E081E5CD
:1006300095E1F9CF40920B0E50920C0E60920D0E88
:1006400070920E0E80911F078130D9F467E470E03C
:10065000C8010E94F9E40097A1F04AE050E070E080
:1006600060E001960E94B6D862307105810591055F
:1006700040F480EB94E176D860E086EA94E10E9451
:100680009452F80180818D3481F58381823309F49D
:1006900045C0883301F1803341F58181843329F5E8
:1006A0008281813311F50E94383C1FC080918214F1
:1006B00080FFC8CF6BEA7BE2C8010E9441DB009754
:1006C00031F0FC01838180538A3008F0BBCF60E0B9
:1006D00087E295E1A8CF8281803339F4818181332B
:1006E00021F410926601109292028091110E8B33C8
:1006F00009F405CF8091720E843008F000CF80910C
:10070000740E8D9DC001112461E17EE08B58914FE4
:100710000E9404E580E00E945EB7F1CE82818133C1
:1007200021F78181813309F741E070E060E085E7DE
:100730009AE1E9DD2FE03EE041E15EE061E77EE045
:100740000E949262DCCE8091821483FDCAC082FF37
:10075000C8C087FDC6C01A82198281E6F82E94E0CF
:10076000E92E29E6D22E8091720E843008F0B9C0AD
:100770000E94CA628111B5C041E050E0BE016D5FC8
:100780007F4F89E992E10E9409CB0B8110E001972C
:1007900011F00FEF1FEF8091A1129091A212A09182
:1007A000A312B091A41280937E1490937F14A0930F
:1007B0008014B09381140E94CA620F3F100741F465
:1007C000811106C02ADD8AEE95E10E94B27BCBCF73
:1007D0004091740E242F30E00A3061F00D3051F05A
:1007E000882309F470C089819A81009719F00196D5
:1007F0009A8389831092960589819A81F29EF001ED
:10080000F39EF00D1124EE58F14FDF01A80FB91F30
:1008100013961C92892BA9F50E94FA250E94CA62A0
:10082000882309F4A0CF89E992E10E940D218091EB
:1008300079148823F1F18150809379148D9DC00142
:10084000112462E08959994F0E94C0CEE091791439
:1008500024E0E29FF0011124ED59F94F40815181CC
:100860006281738140937E1450937F14609380144F
:100870007093811489E992E10E940ECA0E9451C6C8
:1008800072CF1A82198283818D3479F48481823304
:1008900061F48581853349F4868180538A3028F05C
:1008A000809182148B7F8093821481E00E945EB7D6
:1008B000B5CF0E9443C680918214886080938214D1
:1008C000E0921F0750CF4F9DA00111244B58514F6C
:1008D0009E012F5F3F4F66E975E0802F0E94926274
:1008E00042CF0E94F3C16B017C01BB2041F0C0925A
:1008F0000D06D0920E06E0920F06F092100680913F
:10090000E4059091E505A091E605B091E705009713
:10091000A105B10529F140910D0650910E06609197
:100920000F0670911006840F951FA61FB71FA70111
:100930009601281B390B4A0B5B0BDA01C901B7FD85
:100940000FC06BDC60915F077091600789EF95E1E4
:100950000E9470CE40E070E060E090E080E0E9CE80
:1009600080914E0190914F01A0915001B0915101A1
:10097000892B8A2B8B2B79F090910413809105138E
:10098000981709F4C4C0C0920D06D0920E06E092EA
:100990000F06F092100680919B0590919C05A09106
:1009A0009D05B0919E0546015701881A990AAA0A29
:1009B000BB0AD501C401B7FDC0C190910413809159
:1009C000051320913D01981709F4D5C0E091051356
:1009D0003BE5E39FF0011124EC51F84F808128178B
:1009E00099F080933D010E94F3C1B0903D010B2D21
:1009F00010E084E00E94BFA70115110509F0BEC0F8
:100A000060E084E00E940BC180919803882309F480
:100A100087C10091060110910701C801029720913A
:100A2000881230918912281739070CF479C1809007
:100A300005138C82812C912C5401809104132C81FC
:100A4000821709F4FDC0822F90E03BE5389FF0014A
:100A5000399FF00D1124E257F84F4589568967896F
:100A6000708D452B462B472B81F4418D528D638D24
:100A7000748D452B462B472B41F4458D568D678D44
:100A800070A1452B462B472BE9F14BE5489F900180
:100A9000499F300D1124C9018257984F1C01FC0158
:100AA00061817281838194810E947CE46D837E8365
:100AB0008F839887F10161A172A183A194A10E9403
:100AC000C6DB2B013C01F10165A176A187A190A5B0
:100AD0000E94C6DB9B01AC01C301B2010E9457E337
:100AE0002D813E814F8158850E9427DC2B013C01DE
:100AF000AC019B01C501B4010E9443E487FF02C021
:100B0000530142018C818F5F8F708C8396CFBB2005
:100B100019F010929F053FCF0E94F3C100910D067E
:100B200010910E0620910F063091100680904E0114
:100B300090904F01A0905001B0905101080D191DE7
:100B40002A1D3B1D601B710B820B930B97FDE1CFA0
:100B500080919F0581111FCF81E080939F0580E0E8
:100B60000E948D2781E00E948D2782E00E948D27C0
:100B70000E94782710CF80917D0731CF0F3F11055C
:100B800011F461E03ECFEAEEFBE2E491E150EA309D
:100B900008F051C0F0E0E153FA470C9487E2D985A0
:100BA000DE85E385ED851B861B86F785FF85078639
:100BB000118684B5806884BDB7BC26CF84B58062B9
:100BC00084BDB8BC21CF8091800080688093800074
:100BD000109389000093880017CF80918000806275
:100BE0008093800010938B0000938A000DCF80913A
:100BF000B00080688093B000B092B30005CF8091C0
:100C0000B00080628093B000B092B400FDCE8091BD
:100C10009000806880939000109399000093980052
:100C2000F3CE8091900080628093900010939B009F
:100C300000939A00E9CE003811050CF0A2CFE0CE67
:100C4000B801110F880B990B0E94C8DB2B013C01E6
:100C50002091000130910101409102015091030166
:100C6000C501B4010E9427DCA30192010E94E0E2C9
:100C70004B015C010091040110910501AC019B0145
:100C8000C301B2010E9443E418168CF0B801012E92
:100C9000000C880B990B0E94C8DB2B013C01A501BD
:100CA00094010E94C2DB181614F4240135018090CF
:100CB000970590909805A0909905B0909A05A3018A
:100CC0009201C501B4010E9443E41816D4F420E057
:100CD00037ED43EA5CE3C301B2010E9427DC2B013C
:100CE0003C0128E431EE4AE75FE3C501B4010E940C
:100CF00027DC9B01AC01C301B2010E94E0E22B01A1
:100D00003C01409297055092980560929905709227
:100D10009A05C301B2010E94BFE3CB010E9434C215
:100D2000F4E6CF0ED11CE11CF11CC0929B05D092C1
:100D30009C05E0929D05F0929E050E94FA25809107
:100D40001F07882309F4D2C010913E01113061F1D0
:100D50008091821480648093821481E080933E01AC
:100D600064EF71E080E090E00E9446750E9413CD30
:100D70008091821484FFCFC0123028F460E086E3B3
:100D800096E10E94945283E0809367010E94F3C130
:100D90006C597F4F8F4F9F4F60935E0670935F0635
:100DA00080936006909361060E94F3C16B017C0101
:100DB00010914D011123F1F08091E9058823D1F0C4
:100DC0004091A0055091A1056091A2057091A305E5
:100DD00046015701841A950AA60AB70AB501A4016B
:100DE00077FD1AC0833009F492C00CF083C08130C3
:100DF0000CF087C0212F30E0A8EEB3E00E941CE287
:100E0000C60ED71EE81EF91EC092A005D092A105FD
:100E1000E092A205F092A3050E94B8410E94E26A06
:100E20008091E305882379F10E94F3C16B017C0175
:100E30008091DF059091E005A091E105B091E20578
:100E4000A7019601281B390B4A0B5B0BDA01C9017C
:100E5000B7FD19C02091E30530E0A8EEB3E00E9491
:100E60001CE2C60ED71EE81EF91EC092DF05D09206
:100E7000E005E092E105F092E20580E00E94CB24DB
:100E80008AE00E94917B8091DE05882379F10E949F
:100E9000F3C16B017C018091DA059091DB05A09193
:100EA000DC05B091DD0546015701881A990AAA0AA6
:100EB000BB0AD501C401B7FD19C02091DE0530E0A1
:100EC000A8EEB3E00E941CE2C60ED71EE81EF91E73
:100ED000C092DA05D092DB05E092DC05F092DD05E8
:100EE0000E944BA886E093E10E94BF262896E2E18B
:100EF0000C94C4E2843009F07DCF92D985E496E168
:100F000003C08ED984E796E10E94B27B73CF88D963
:100F10008DE596E1F9CF112309F446CF34CFA2E154
:100F2000B0E0E5E9F7E80C94A9E290913E0D93FD5D
:100F30007EC0082F78D9182F87FD79C089E40E94D8
:100F40008763882309F48BC00E945D67282F30E0F7
:100F50001216130614F421E030E0220F331F220F83
:100F6000331FF901EE53FD4F80819181198A0E9450
:100F700034C280918812909189128635910574F05F
:100F8000002381F00E943B400DC082E50E948763F0
:100F9000882309F46CC00E949867E9CF0E948340BF
:100FA0000E94B9B86091881270918912072E000CC6
:100FB000880B990B0E94C8DB209184123091851216
:100FC00040918612509187120E9443E4181644F013
:100FD000298980E19FE1222329F049894A8B48C071
:100FE0008BE19FE19F938F9386E29FE19F938F9385
:100FF0001F920E9477520F900F900F900F900F90BA
:1010000031E03A8B35C060E070E0CB014FC0C701E2
:10101000B6010E94C2DB87FF0EC080916601882363
:1010200021F0109266010E94B9B83092980362963E
:10103000E1E10C94C5E24601570100E098C08FE35E
:101040000E94917BCFC020E030E040E450E40E9459
:1010500043E418160CF004C12601370101C183E5F1
:101060000E948763898B811196CF01118ECF1A8AD6
:1010700083E50E948763882331F00E9498679093EC
:1010800007018093060182E40E948763882331F080
:101090000E949867909305018093040186E40E9462
:1010A0001063882309F4AFCF0E94A7676093000103
:1010B00070930101809302019093030133243394D0
:1010C00020E030E0A9010E94C2DB811101C0312C77
:1010D00030929803002309F4AACF5A89552309F4C2
:1010E000A6CF1092980381E0809366011D821E8234
:1010F0001F82188619861A861B861C8680E09CE350
:10110000ACE1B6E48D879E87AF87B88B812C912C9C
:1011100090E8A92E9FEBB92E00E0412C512C320112
:101120006091881270918912072E000C880B990B20
:101130000E94C8DB6B017C01A50194010E94C2DB07
:101140008823A9F020918412309185124091861253
:1011500050918712998991115ACFC701B6010E9407
:10116000C2DB082F001F0027001F460157010E9405
:10117000F3C16B017C01DC01CB0129853A854B85EC
:101180005C85821B930BA40BB50BB7FD2EC0D7015A
:10119000C60188519C4FAF4FBF4F89879A87AB8755
:1011A000BC87812F0E94CB248CE29FE10E94B27BFE
:1011B000411451046104710409F441CFC301B20127
:1011C000605F784D8F4F9F4F6C197D098E099F0985
:1011D00028EE33E040E050E00E94F0E1CA01B9019E
:1011E0000E94D76F8AE00E94917B80E07AD90E94AA
:1011F000F3C160930D0670930E0680930F069093D3
:1012000010062091841230918512409186125091DF
:10121000871229833A834B835C83C501B4010E9402
:10122000DFE29F77411451046104710409F00BCF90
:1012300020E030E040E85FE30E94C2DB87FF10C09F
:101240003A89412C512C3201332331F085E0482E6C
:101250008DE0582E612C712C4C0C5D1C6E1C7F1C7B
:101260000023C1F18D819E81AF81B885892B8A2BA6
:101270008B2B61F0D701C6012D813E814F815885AE
:10128000821B930BA40BB50BB7FD24C029813A81B7
:101290004B815C816D857E858F8598890E94DFE218
:1012A00020E030E040EC5FE30E94C2DB87FDB5CE7A
:1012B000D701C601805A9541AF4FBF4F8D839E83A2
:1012C000AF83B88729813A814B815C812D873E8726
:1012D0004F87588B80916601882309F49ECE411474
:1012E00051046104710461F030E1C31A37E2D30A9A
:1012F000E108F108C418D508E608F708F7FE8DCE16
:101300001A8A0ECFA1E4B0E0E8E8F9E80C94A8E26C
:1013100022968FAF22972091E9052CA781E0809338
:10132000E90580910C068D3409F4F1C4843511F47B
:101330000C940B9E873491F480910A0690910B06D1
:101340008D31910509F462C308F0E5C1843091053F
:1013500009F406C330F4029708F45FC20E9462CE1B
:10136000D7C28531910509F4D3C24C97B9F787E00C
:101370000E945F37811111C080910406909105068B
:10138000A0910606B0910706FEE0B695A795979541
:101390008795FA95D1F780FDBBC20E942329109250
:1013A00013016091B9028CE40E948767382E80E0B7
:1013B0000E9490730E94F3C160930D0670930E0615
:1013C00080930F06909310060E94E53A81E0809387
:1013D000DA060E942A3DC0900406D0900506E090EF
:1013E0000606F0900706E9E1F694E794D794C794CF
:1013F000EA95D1F7C0FE0DC081E00E945F37182F3B
:1014000082E00E945F3711110C94489E11E0811117
:1014100001C010E08091040690910506A091060697
:10142000B091070677E1B695A795979587957A9538
:10143000D1F780FF02C00C942E9E1111CBC2809177
:10144000040690910506A0910606B09107063B2F71
:101450003170A32E3113C0C28C2D8170A12E811347
:10146000BBC211E0AA24A394BB24B39482E50E94DA
:101470008763882309F4B4C20E94A7676C8F7D8FAD
:101480008E8F9F8F20E030E0A9010E94C2DB88236D
:1014900059F0111105C0A11003C0BB2009F428C1E7
:1014A000CE014C960E946BB8112309F489C0AA2082
:1014B00009F483C0109272011092730110927401AA
:1014C00010927501109276011092770110927801B6
:1014D000109279010E94363C8DEE96E00E943571A3
:1014E0006B017C0181EF96E00E9435712B013C017C
:1014F000AC019B01C701B6010E9443E418160CF031
:1015000074C2A7019601C301B2010E9457E39B0177
:10151000AC010E9427DC20E030E040E85FE30E945D
:10152000E0E20E947CE421E030E048E452E40E94E2
:1015300027DC69837A838B839C8380917A019091E5
:101540007B01A0917C01B0917D0188A399A3AAA3FE
:10155000BBA320E030E040EC5FE3C301B2010E9496
:1015600027DC2B013C0177FA709477F8709420E027
:1015700030E040EC5FE3C701B6010E9427DC9058E1
:10158000DE0111966D01E8A0F9A00AA11BA1A3013B
:1015900092010E94043B0E94B83F10927201109287
:1015A00073011092740110927501109276011092DD
:1015B0007701109278011092790180E00E948D3EAF
:1015C000AA2019F081E00E948D3EBB2009F490C052
:1015D00083E00E947A3781118BC00E94363C2091B3
:1015E0007A0130917B0140917C0150917D0128A3CB
:1015F00039A34AA35BA32093A9023093AA02409384
:10160000AB025093AC02A090FF12B0900013D50132
:10161000CD90DD90ED90FC90A701960160E070E028
:1016200080EE92E40E94DFE22B013C0140929D0299
:1016300050929E0260929F027092A002F5018480F7
:101640009580A680B780A501940160E070E080EEEF
:1016500092E40E94DFE26CA37DA38EA39FA360931C
:10166000A1027093A2028093A3029093A4022DE0A2
:1016700030E044EE52E4C501B4010E9443E4181680
:101680000CF4B8C12EE030E042EE52ECC501B401DA
:101690000E94C2DB87FDAEC12DE030E04EEE52E489
:1016A000C701B6010E94C2DB18160CF4A3C12EE0DC
:1016B00030E042EE52ECC701B6010E9443E487FDE0
:1016C00099C119821A821B821C829E012F5F3F4F93
:1016D0006901E8A0F9A00AA11BA12CA13DA14EA17E
:1016E0005FA1C301B2010E94043B82E00E948D3ED3
:1016F0000E94363C8091D9068093DA06332019F097
:1017000081E00E9490730E94CC3A83E0809367014D
:101710000E945C3CFDC08A35910509F4E9C250F590
:101720008E31910509F475C18A9709F017CE809121
:101730001F07833008F4ECC089E40E948763082FF8
:10174000F12C882319F00E949867F82E8AE40E94F1
:101750008763E82E882309F4C9C10E949867182F6F
:101760000111C7C1173008F4CAC181E499E10E9490
:10177000B27BCEC08B35910509F4BDC28C35910585
:1017800009F0ECCD5FE2252E52E0352E62E7E62E21
:1017900061E0F62EC12CD12C10E0D1018D911D01FC
:1017A0000E948763082F882351F10E94A7672B01AD
:1017B0003C01F70120813181428153810E94DFE2A7
:1017C0004B015C012DEB37E346E855EB0E94C2DB91
:1017D00087FD0AC02DEB37E346E855E3C501B401A8
:1017E0000E9443E418165CF4133011F0C02E0D2D46
:1017F000D7014D925D926D927C921397D02E1F5F10
:10180000B4E0EB0EF11C143041F6CC2009F477C2A1
:101810000E94363C0E945C3C7BC080911F07833055
:1018200008F476C0ADE9CA2EA2E0DA2EB2E7EB2EBC
:10183000B1E0FB2E10E088E5810F0E9487638823CA
:1018400009F472C00E94A7674B015C01812F0E94BE
:10185000E962882359F0D7012D913D914D915C911A
:10186000C501B4010E94E0E24B015C01F6018082F7
:101870009182A282B3821F5FF4E0CF0ED11C24E0DC
:10188000E20EF11C1330B9F685E40E9487638823C9
:1018900009F455C00E94A7676B017C0183E00E9498
:1018A000E962882371F020917E0130917F0140919F
:1018B000800150918101C701B6010E94E0E26B01F5
:1018C0007C01C092A902D092AA02E092AB02F092EF
:1018D000AC0240E050E0BA0186E40E94CF6720E00D
:1018E00030E0A9010E9443E4181684F40E94A7671F
:1018F00029E838E848E85CE30E9427DC60930C01A3
:1019000070930D0180930E0190930F010E94BD37DB
:1019100022969FAD2297911102C00E9458B8ACA5A3
:10192000A093E9050C944795F70180819181A281EC
:10193000B381F60180839183A283B3839CCF80918E
:101940007E0190917F01A0918001B09181018093EF
:10195000A9029093AA02A093AB02B093AC02B9CFB4
:1019600080E50E948763C12CD12C7601882321F069
:101970000E943D676B017C0183E50E948763882399
:1019800061F00E94A76720E030E04AE754E40E943B
:1019900027DC0E94C4E36B017C010E942329809113
:1019A0001510811105C060E083E099E10E94945216
:1019B0000E94F3C1C60ED71EE81EF91E0E94F3C195
:1019C0006C197D098E099F0997FFA2CF80E00E94C4
:1019D0007182F4CFA12E10E04C2D4170B42E46CD73
:1019E00060E070E080EA90E449CDA3019201C70174
:1019F000B6018BCD60E08EE199E10E9494520E9485
:101A000010818CE099E10E94B27B72CE0E94A49E6C
:101A10007FCF0091FF1210910013D8012D913D91BD
:101A20004D915C916091720170917301809174018C
:101A3000909175010E94E0E2AB01BC0188E50E9433
:101A4000CF6769837A838B839C83F80124813581F6
:101A5000468157816091760170917701809178017C
:101A6000909179010E94E0E2AB01BC0189E50E94FE
:101A7000CF676D837E838F839887BE016B5F7F4FB7
:101A8000CE0101960E94FBB8882309F441CF80E083
:101A90000E9490730E94E53A61E085E40E948767A6
:101AA00021E0482FBE016B5F7F4FCE0101960E945F
:101AB00031BA6B017C0149815A816B817C8189E358
:101AC00099E10E94DD7B4D815E816F81788584E3A1
:101AD00099E10E94DD7BB701A6018FE299E10E94A6
:101AE0001C7C0E94CC3A0E945C3C12CF10E0002388
:101AF00031F0F6E0FF1508F438CEE11033CE80E186
:101B0000E2E7F1E0ADE9B2E001900D928A95E1F7EC
:101B1000002319F16F2DFF0C770B880B990B0E9496
:101B2000C8DB2091BA023091BB024091BC025091B7
:101B3000BD020E9427DC2091AD023091AE0240919F
:101B4000AF025091B0020E94E0E260939D02709358
:101B50009E0280939F029093A002EE2019F1612FC4
:101B6000110F770B880B990B0E94C8DB2091BE02E6
:101B70003091BF024091C0025091C1020E9427DC07
:101B80002091B1023091B2024091B3025091B4025F
:101B90000E94E0E26093A1027093A2028093A302EC
:101BA0009093A40260E080E50E9487678823C1F1DA
:101BB0000023D1F0E091FF12F091001320813181D8
:101BC0004281538160919D0270919E0280919F029B
:101BD0009091A0020E94DFE260939D0270939E02AA
:101BE00080939F029093A002EE20D1F0E091FF122B
:101BF000F091001324813581468157816091A102C3
:101C00007091A2028091A3029091A4020E94DFE24F
